:100000000C94D1080C94F9080C94F9080C94F90894
:100010000C94F9080C94F9080C94F9080C94F9085C
:100020000C94F9080C94F9080C94F9080C94F9084C
:100030000C94F9080C94464C0C94F9080C94F908AB
:100040000C94F9080C94C25C0C9418250C94F908D3
:100050000C94DA260C94F9080C94F9080C94F9081D
:100060000C94F9080C94F9080C94F9080C94F9080C
:100070000C94F9080C94F9080C94F908084AD73B39
:100080003BCE016E84BCBFFDC12F3D6C74319ABD67
:1000900056833DDA3D00C77F11BED9E4BB4C3E918B
:1000A0006BAAAABE000000803F05A84CCDB2D44E7A
:1000B000B93836A9020C50B9918688083CA6AAAA7C
:1000C0002ABE000000803F6563686F3A00656E716C
:1000D0007565696E67202200220073746172740076
:1000E000506F7765725570002045787465726E6147
:1000F0006C205265736574002042726F776E206FBA
:100100007574205265736574002057617463686468
:100110006F672052657365740020536F6674776152
:100120007265205265736574004D61726C696E2052
:1001300000312E302E302052433200204C61737437
:1001400020557064617465643A2000323031322D7C
:1001500030372D323900207C20417574686F723A37
:10016000200069776A002046726565204D656D6FD5
:1001700072793A20002020506C616E6E6572427573
:100180006666657242797465733A20006F6B00444D
:100190006F6E6520736176696E672066696C652E87
:1001A000004572726F723A004C696E65204E756D33
:1001B000626572206973206E6F74204C61737420C5
:1001C0004C696E65204E756D6265722B312C204C2A
:1001D000617374204C696E653A00636865636B7384
:1001E000756D206D69736D617463682C204C61734B
:1001F00074204C696E653A004E6F20436865636BEE
:1002000073756D2077697468206C696E65206E75F2
:100210006D6265722C204C617374204C696E653A76
:10022000004E6F204C696E65204E756D62657220C0
:100230007769746820636865636B73756D2C204CF7
:10024000617374204C696E653A006F6B005072697F
:100250006E7465722073746F707065642064657568
:1002600020746F206572726F72732E204669782039
:10027000746865206572726F7220616E6420757398
:1002800065204D39393920746F207265737461723D
:1002900074212E202854656D7065726174757265C5
:1002A0002069732072657365742E2053657420690C
:1002B00074206265666F7265207265737461727412
:1002C000696E672900446F6E65207072696E74698B
:1002D0006E672066696C6500426567696E206669B5
:1002E0006C65206C69737400456E642066696C658A
:1002F000206C697374006F6B20543A00202F00202B
:10030000423A00202F0020403A00543A0020453A5B
:100310000020573A00543A0020453A0020423A0063
:100320004649524D574152455F4E414D453A4D6108
:10033000726C696E2056313B20537072696E746521
:10034000722F6772626C206D617368757020666FC2
:10035000722067656E36204649524D574152455FBF
:1003600055524C3A687474703A2F2F7777772E6D08
:10037000656E64656C2D70617274732E636F6D2091
:1003800050524F544F434F4C5F56455253494F4E76
:100390003A312E30204D414348494E455F54595023
:1003A000453A4D656E64656C204558545255444538
:1003B000525F434F554E543A310A00583A00593A69
:1003C000005A3A00453A0020436F756E7420583A3F
:1003D00000593A005A3A00785F6D696E3A00795FC9
:1003E0006D696E3A007A5F6D696E3A00556E6B6E9C
:1003F0006F776E20636F6D6D616E643A220022002C
:10040000526573656E643A006F6B005072696E746A
:1004100065722068616C7465642E206B696C6C2851
:10042000292063616C6C6564202121005072696E23
:100430007465722073746F707065642064657520D4
:10044000746F206572726F72732E20466978207403
:100450006865206572726F7220616E6420757365C5
:10046000204D39393920746F20726573746172744C
:10047000212E202854656D70657261747572652037
:1004800069732072657365742E20536574206974D6
:10049000206265666F72652072657374617274693B
:1004A0006E6729007C3C3E5E2B3D3F2F5B5D3B2C05
:1004B0002A225C006563686F3A0020636F6C6420D9
:1004C000657874727573696F6E2070726576656E8B
:1004D0007465640020746F6F206C6F6E67206578A0
:1004E00074727573696F6E2070726576656E74656F
:1004F00064006563686F3A00656E6473746F70734F
:10050000206869743A200020583A0020593A0020A7
:100510005A3A0024F404D9201BC40C5C0E9804C47D
:10052000095F0265077101F405F900FB04B3004897
:10053000048700C10369005803550003034500BE4A
:10054000023A008402310053022A002902250004E5
:10055000022000E4011C00C8011900AF0117009837
:100560000114008401130071011000610110005199
:10057000010E0043010D0036010B002B010B002082
:10058000010B00150109000C01090003010800FB23
:10059000000800F3000800EB000700E4000600DE9E
:1005A000000600D8000600D2000600CC000500C7F7
:1005B000000500C2000500BD000400B9000400B53C
:1005C000000400B1000400AD000400A9000400A56F
:1005D000000300A20003009F0004009B000300989A
:1005E0000003009500020093000300900003008DBB
:1005F0000002008B000300880002008600020084D5
:10060000000300810002007F0002007D0002007BE9
:1006100000020079000200770001007600020074F9
:1006200000020072000100710002006F0002006D04
:100630000001006C0002006A00010069000200670E
:100640000001006600010065000100640002006214
:1006500000010061000100600001005F0002005D18
:100660000001005C0001005B0001005A000100591C
:10067000000100580001005700010056000100551C
:10068000000100540001005300000053000100521B
:1006900000010051000100500001004F0001004E18
:1006A0000000004E0001004D0001004C0001004B15
:1006B0000000004B0001004A000100490001004811
:1006C000000000480001004700010046000000460D
:1006D0000001004500000045000100440001004306
:1006E0000000004300010042000000420001004100
:1006F00000000041000100400001003F0000003FF9
:100700000001003E0000003E0001003D0000003DF1
:100710000001003C0000003C0000003C0001003BE8
:100720000000003B0001003A0000003A00010039DF
:1007300000000039000100380000003800000038D7
:1007400000010037000000370001003600000036CD
:1007500000000036000100350000003500000035C3
:1007600000010034000000340000003400010033B8
:1007700000000033000000330001003200000032AE
:1007800000000032000100310000003100000031A3
:100790000001003000000030000000300001002F98
:1007A0000000002F0000002F0000002F0001002E8D
:1007B0000000002E0000002E0001002D0000002D82
:1007C0000000002D0000002D0001002C0000002C76
:1007D0000000002C0000002C0001002B0000002B6A
:1007E0000000002B0000002B0001002A0000002A5E
:1007F0000000002A0000002A000100290000002952
:100800000000002900000029000000290001002844
:100810000000002800000028000000280000002838
:10082000000100270000002700000027000000272B
:10083000000000270001002600000026000000261E
:100840000000002600000026000100250000002511
:100850000000002500000025000000250000002504
:1008600000010024000000240000002400000024F7
:1008700000000024000100230000002300000023EA
:1008800000000023000000230000002300000023DC
:1008900000010022000000220000002200000022CF
:1008A00000000022000000220001002100000021C1
:1008B00000000021000000210000002100000021B4
:1008C00000000021000100200000002000000020A6
:1008D0000000002000000020000000200000002098
:1008E000000000200001001F0000001F0000001F8A
:1008F0000000001F0000001F0000001F0000001F7C
:100900000001001E0000001E0000001E0000001E6E
:1009100000000024F4D43050C38E20C2A2401782BD
:100920008B7011127A910D816CD90AA861E108C708
:10093000586607615143061E4B5D05C145A7041A61
:10094000411104093D9803713931034036DB0265DA
:10095000339102D4305402802E1D02632CEE0175B7
:100960002AC501B028A001102781018F2564012B21
:10097000244B01E0223401AC211F018D200D0180A8
:100980001FFC00841EED00971DDF00B81CD200E69E
:100990001BC600201BBC00641AB200B219A8000AD2
:1009A00019A0006A189900D117910040178B00B563
:1009B00016840031167E00B31579003A157300C70E
:1009C000146F0058146A00EE136600881363002544
:1009D000135E00C7125B006C12570015125400C161
:1009E00011510070114F0021114B00D61049008D9C
:1009F0001047004610440002104200C00F40008023
:100A00000F3E00420F3C00060F3B00CB0E38009318
:100A10000E37005C0E3500270E3400F30D3200C196
:100A20000D3100900D3000600D2E00320D2D0005AF
:100A30000D2C00D90C2B00AE0C2900850C29005C74
:100A40000C2700350C27000E0C2600E80B2400C4F0
:100A50000B2400A00B23007D0B23005A0B2100392F
:100A60000B2100180B2000F80A1F00D90A1E00BB3A
:100A70000A1E009D0A1D00800A1D00630A1C004713
:100A80000A1B002C0A1B00110A1A00F7091A00DDC4
:100A9000091900C4091900AB091900920917007B54
:100AA000091800630917004C0916003609160020C2
:100AB0000916000A091500F5081500E0081400CC15
:100AC000081400B8081400A4081400900813007D4E
:100AD0000812006B08130058081200460812003470
:100AE000081100230811001208110001081100F07C
:100AF000071000E0071000D0071000C0071000B07A
:100B0000070F00A107100091070E0083070F007464
:100B1000070F0065070E0057070E0049070E003B40
:100B2000070D002E070E0020070D0013070D00060D
:100B3000070D00F9060C00ED060D00E0060C00D4D0
:100B4000060C00C8060C00BC060C00B0060C00A485
:100B5000060B0099060C008D060B0082060B007731
:100B6000060B006C060B0061060A0057060B004CD2
:100B7000060A0042060A0038060A002E060A002469
:100B8000060A001A060A001006090007060A00FDF8
:100B9000050900F4050900EB050900E2050900D983
:100BA000050900D0050900C7050900BE050900B503
:100BB000050800AD050800A50509009C050800947E
:100BC0000508008C050800840508007C05080074F1
:100BD0000508006C050700650508005D050700565F
:100BE0000508004E050700470507004005080038C6
:100BF000050700310507002A050700230507001C2B
:100C0000050600160507000F050700080506000287
:100C1000050700FB040600F5040700EE040600E8E3
:100C2000040600E2040700DB040600D5040600CF3A
:100C3000040600C9040600C3040600BD040600B78C
:100C4000040600B1040500AC040600A6040600A0DA
:100C50000405009B04060095040500900406008A24
:100C600004050085040500800406007A040500756B
:100C7000040500700405006B0405006604050061AE
:100C80000405005C04050057040500520405004DEE
:100C900004050048040500430405003E0404003A2E
:100CA00004050035040500300404002C0405002769
:100CB000040400230405001E0404001A04040016A2
:100CC000040500110404000D0404000904050004D7
:100CD00004040000040400FC030400F8030400F40E
:100CE000030400F0030400EC030400E8030400E440
:100CF000030400E0030400DC030400D8030400D470
:100D0000030400D0030400CC030400C8030300C59F
:100D100003030020626961733A200020643A2000D6
:100D2000206D696E3A2000206D61783A2000204BDA
:100D3000753A20002054753A200020436C61736995
:100D400063205049442000204B703A2000204B691A
:100D50003A2000204B643A200050494420417574E9
:100D60006F74756E65206661696C656421205465D9
:100D70006D706572617475726520746F2068696743
:100D800068006F6B20543A0020403A0050494420DC
:100D90004175746F74756E65206661696C65642158
:100DA0002074696D656F75740050494420417574F5
:100DB0006F74756E652066696E697368656420215D
:100DC00020506C61636520746865204B702C204B4B
:100DD0006920616E64204B6420636F6E7374616E72
:100DE000747320696E2074686520636F6E6669672E
:100DF00075726174696F6E2E68004572726F723A17
:100E000000202D20496E76616C69642065787472CB
:100E100075646572206E756D626572210070012CBB
:100E20000190012701B0012201C0011D01F001184C
:100E3000011002130130020E016002090190020448
:100E400001C002FF000003FA004003F5008003F038
:100E500000D003EB002004E6007004E100E004DCB5
:100E6000004005D700C005D2004006CD00D006C81E
:100E7000008007C3003008BE00F008B900C009B404
:100E800000B00AAF00B00BAA00D00CA500000EA065
:100E900000500F9B00C01096005012910000148C5F
:100EA00000C0158700B0178200B0197D00D01B78F4
:100EB00000001E730040206E0090226900F0246440
:100EC0000040275F0090295A00E02B5500102E505B
:100ED0000020304B0010324600E033410090353C9A
:100EE000001037370070383200A0392D00B03A2892
:100EF00000A03B2300603C1E00103D1900903D14F3
:100F000000103E0F00703E0A00C03E0500003F008A
:100F100000202D20496E76616C69642065787472BA
:100F200075646572206E756D6265722021003A20CD
:100F30004578747275646572207377697463686547
:100F400064206F66662E204D415854454D502074E4
:100F500072696767657265642021003A204578747C
:100F60007275646572207377697463686564206F55
:100F700066662E204D494E54454D50207472696767
:100F8000676572656420210054656D7065726174D7
:100F9000757265206865617465642062656420739C
:100FA00077697463686564206F66662E204D4158CA
:100FB00054454D50207472696767657265642021DD
:100FC00021006563686F3A00534420696E6974209C
:100FD0006661696C004572726F723A00766F6C756B
:100FE0006D652E696E6974206661696C6564006F59
:100FF00070656E526F6F74206661696C6564005332
:10100000442063617264206F6B006F70656E2066B0
:1010100061696C65642C2046696C653A20002E007D
:1010200046696C65206F70656E65643A002053698F
:101030007A653A0046696C652073656C6563746512
:1010400064006F70656E206661696C65642C204673
:10105000696C653A20002E006F70656E20666169CC
:101060006C65642C2046696C653A20002E0057722E
:101070006974696E6720746F2066696C653A200038
:101080006F70656E206661696C65642C2046696CC2
:10109000653A20002E0046696C652064656C6574B5
:1010A00065643A0044656C6574696F6E20666169B9
:1010B0006C65642C2046696C653A20002E00534410
:1010C000207072696E74696E6720627974652000A1
:1010D0002F004E6F74205344207072696E74696ED5
:1010E00067006572726F722077726974696E67202B
:1010F000746F2066696C650000000001020000004A
:1011000000000000040307060000000000000000CB
:1011100000000000000000000102040810204080D0
:1011200001020408102040800102040810204080C1
:1011300080402010080402010202020202020202A0
:101140000404040404040404030303030303030367
:101150000101010101010101002225282B002124A8
:10116000272A494E46494E4954594E414E000020C7
:10117000410000C84200401C4620BCBE4CCA1B0EA9
:101180005AAEC59D74CDCCCC3D0AD7233C17B7D100
:101190003877CC2B329595E6241FB14F0A001025E5
:1011A000142511241FBECFEFD0E1DEBFCDBF12E06A
:1011B000A0E0B1E0EEE2F7EE02C005900D92AE3C89
:1011C000B107D9F71EE0AEECB2E001C01D92AD321E
:1011D000B107E1F711E1C0EAD1E104C02297FE01B5
:1011E0000E94AB6DCE39D107C9F70E94E2240C945E
:1011F0008A730C940000AF92BF92CF92DF92EF926D
:10120000FF920F931F93CF93DF93CDB7DEB7E09795
:101210000FB6F894DEBF0FBECDBF80E1E3E4F1E08E
:10122000DE01919601900D928A95E1F780E1E3E568
:10123000F1E0DE01519601900D928A95E1F780E18F
:10124000E3E6F1E0DE01119601900D928A95E1F757
:101250006E0181E2C80ED11C8BE5E82E8DE0F82EE0
:101260008E010F5E1F4F6BE67DE0AE014F5F5F4F5B
:101270009BE4A92E9DE0B92E20E030E0F60181919B
:101280009191A191B1916F01F70181939193A193F4
:10129000B1937F01F80181919191A191B1918F0159
:1012A000FB0181939193A193B193BF01FA018191C5
:1012B0009191A191B191AF01F50181939193A19386
:1012C000B1935F012F5F3F4F24303105B9F680E0C5
:1012D00090E0AAE7B4E48093430D9093440DA0936B
:1012E000450DB093460D80933F0D9093400DA09314
:1012F000410DB093420D1092470D1092480D10927F
:10130000490D10924A0D80E29EE4A0E0B0E0809387
:101310007B0D90937C0DA0937D0DB0937E0D10926C
:101320002F0D1092300D1092310D1092320D80E081
:1013300090E0A0E7B1E480933B0D90933C0DA09327
:101340003D0DB0933E0D4DEC5CEC6CEC7EE34093B8
:10135000370D5093380D6093390D70933A0D80938B
:10136000330D9093340DA093350DB093360DE7EC0B
:10137000F0E007C09091C00095FFFCCF8093C600BD
:10138000319684918111F6CFE3E7F1E006C09091A8
:10139000C00095FFFCCF8093C60081918111F7CFEB
:1013A0008091C00085FFFCCF8AE08093C600E09664
:1013B0000FB6F894DEBF0FBECDBFDF91CF911F9166
:1013C0000F91FF90EF90DF90CF90BF90AF90089576
:1013D000CF93DF9300D0CDB7DEB78091270E9091E9
:1013E000280E9E012F5F3F4F009719F42D523E406B
:1013F00002C0281B390B3A83298389819A810F9077
:101400000F90DF91CF9108952091CE033091CF03BB
:10141000243031050CF06AC04091D0035091D103C3
:1014200060E6649F9001659F300D1124BC01C901E5
:101430008E529C4F0E947170E7ECF0E007C09091D3
:10144000C00095FFFCCF8093C60031968491811136
:10145000F6CFEDECF0E007C09091C00095FFFCCF17
:101460008093C600319684918111F6CF8091D0038C
:101470009091D10320E6289FF001299FF00D1124BF
:10148000EE52FC4F06C09091C00095FFFCCF8093B8
:10149000C60081918111F7CFE8EDF0E007C090918F
:1014A000C00095FFFCCF8093C600319684918111D6
:1014B000F6CF8091C00085FFFCCF8AE08093C60004
:1014C0008091D0039091D103019664E070E00E9476
:1014D000376D9093D1038093D0038091CE03909188
:1014E000CF0301969093CF038093CE030895CF92BC
:1014F000DF92EF92FF920F931F93CF93DF9300D071
:1015000000D0CDB7DEB740E052EC61E070E089EA90
:1015100095E00E940F27EAEDF0E007C09091C0002F
:1015200095FFFCCF8093C600319684918111F6CF50
:101530008091C00085FFFCCF8AE08093C60087ECD5
:1015400090E0FC0107C03091C00035FFFCCF209334
:10155000C600319624912111F6CF24B720FF14C084
:10156000E0EEF0E007C04091C00045FFFCCF3093B3
:10157000C600319634913111F6CF3091C00035FF5D
:10158000FCCF3AE03093C60021FF14C0E8EEF0E053
:1015900007C04091C00045FFFCCF3093C600319694
:1015A00034913111F6CF3091C00035FFFCCF3AE0D5
:1015B0003093C60022FF14C0E8EFF0E007C040916E
:1015C000C00045FFFCCF3093C600319634913111F5
:1015D000F6CF3091C00035FFFCCF3AE03093C60023
:1015E00023FF14C0E9E0F1E007C04091C00045FFCF
:1015F000FCCF3093C600319634913111F6CF309143
:10160000C00035FFFCCF3AE03093C60025FF14C080
:10161000E9E1F1E007C03091C00035FFFCCF209335
:10162000C600319624912111F6CF2091C00025FFEC
:10163000FCCF2AE02093C60014BEE9E2F1E007C027
:101640003091C00035FFFCCF2093C6003196249125
:101650002111F6CFE1E3F1E007C03091C00035FF82
:10166000FCCF2093C600319624912111F6CF209112
:10167000C00025FFFCCF2AE02093C600FC01249186
:10168000E7ECF0E008C03091C00035FFFCCF2093BC
:10169000C600319624912111F6CFEBE3F1E007C0AB
:1016A0003091C00035FFFCCF2093C60031962491C5
:1016B0002111F6CFEBE4F1E007C03091C00035FF17
:1016C000FCCF2093C600319624912111F6CFE6E598
:1016D000F1E007C03091C00035FFFCCF2093C60079
:1016E000319624912111F6CFE2E6F1E007C0309166
:1016F000C00035FFFCCF2093C60031962491211104
:10170000F6CF2091C00025FFFCCF2AE02093C60031
:10171000FC018491E7ECF0E008C09091C00095FFD7
:10172000FCCF8093C600319684918111F6CFE6E616
:10173000F1E007C09091C00095FFFCCF8093C600F8
:10174000319684918111F6CF0E94E8094AE050E079
:10175000BC0189EA95E00E942528E5E7F1E007C091
:101760009091C00095FFFCCF8093C6003196849184
:101770008111F6CF4AE050E060ED74E089EA95E02F
:101780000E9425288091C00085FFFCCF8AE08093CD
:10179000C6001092520510925305109254051092F3
:1017A000550580E00E94FB082BE4C22E2DE0D22ECE
:1017B0003BE5E32E3DE0F32E0FE11DE0F6016191E4
:1017C0007191819191916F01F70121913191419135
:1017D00051917F0129833A834B835C830E94196A6C
:1017E00029813A814B815C810E944E6C0E94ED6997
:1017F000F80161937193819391938F01FBE5CF166B
:10180000FDE0DF06D9F60E9479570E94953E0F90C1
:101810000F900F900F90DF91CF911F910F91FF903C
:10182000EF90DF90CF900C94575280915C0590918F
:101830005D0560E070E001960C94AF6D80915C05F1
:1018400090915D054AE050E060E070E001960C94F4
:10185000066F409156055091570590E6949F900170
:10186000959F300D1124682F70E0C9018E529C4F56
:101870000E94667090935D0580935C0521E0892B42
:1018800009F420E0822F08950E94622560936E057E
:1018900070936F058093700590937105E0915605E4
:1018A000F0915705EE5AFA4F8081811114C0E8E09B
:1018B000F4E007C09091C00095FFFCCF8093C60074
:1018C000319684918111F6CF8091C00085FFFCCFC5
:1018D0008AE08093C600089589EA95E00E94632714
:1018E000E0E0F4E007C09091C00095FFFCCF80934A
:1018F000C600319684918111F6CF409162055091D6
:10190000630560916405709165054F5F5F4F6F4F90
:101910007F4F2AE030E089EA95E00E941428809108
:10192000C00085FFFCCF8AE08093C6000C94440C75
:101930002F923F924F925F926F927F928F929F92DF
:10194000AF92BF92CF92DF92EF92FF920F931F93CD
:10195000CF93DF93CDB7DEB76F970FB6F894DEBFA6
:101960000FBECDBFA0E67A2EB4E04B2E512CEDE495
:10197000F2E084901AE0B12EEAE4F2E0A490992417
:10198000939480912A0690912B0620912C063091F9
:101990002D06821B930B8F779927892B09F004C2A0
:1019A00034C38D3051F08A3321F490915905992335
:1019B00021F02F3531050CF4DAC12115310509F478
:1019C0009FC28091D0039091D103789E7001799E3F
:1019D000F00C1124F701E20FF31FEE52FC4F1082BE
:1019E000209159052111BEC110925905FC01EE5AF2
:1019F000FA4F108287010E521C4F6EE470E0C8014E
:101A00000E946670009709F404C190935D0580936D
:101A10005C05801B910B8E0D9F1D4AE050E060E03D
:101A200070E08D529C4F0E94066F60935E0570932C
:101A30005F058093600590936105C0906205D0902A
:101A40006305E0906405F0906505970186010F5FDE
:101A50001F4F2F4F3F4F6017710782079307C1F148
:101A60002091D0033091D103729EC001739E900DDE
:101A700011246BE871E08E529C4F0E949570892B67
:101A800039F5E1EAF1E007C09091C00095FFFCCF85
:101A90008093C600319684918111F6CFE8EAF1E097
:101AA00007C09091C00095FFFCCF8093C60031968F
:101AB00084918111F6CF2AE030E0B701A60189EACE
:101AC00095E00E9414288091C00085FFFCCF8AC059
:101AD0008091D0039091D103789E1001799E300CB3
:101AE000112481010E521C4F6AE270E0C8010E946D
:101AF0006670009721F450C0F3262F5F02C020E0EB
:101B0000F12CF101E20FF11DEE52FC4F30813A321F
:101B100099F790935D0580935C05801B910B820D76
:101B2000931D60E070E08D529C4F0E94AF6D0E944B
:101B3000E8692F2D30E02617370709F459C0E1EA8C
:101B4000F1E007C09091C00095FFFCCF8093C600E4
:101B5000319684918111F6CFEAEDF1E007C09091C2
:101B6000C00095FFFCCF8093C6003196849181110F
:101B7000F6CF4091620550916305609164057091C4
:101B800065052AE030E089EA95E00E9414288091FA
:101B9000C00085FFFCCF26C0E1EAF1E007C09091CC
:101BA000C00095FFFCCF8093C600319684918111CF
:101BB000F6CFE8EFF1E007C09091C00095FFFCCFB1
:101BC0008093C600319684918111F6CF2AE030E0EF
:101BD000B701A60189EA95E00E9414288091C0000F
:101BE00085FFFCCF8AE08093C6000E946C0C47C042
:101BF00080915E0590915F05A0916005B0916105AF
:101C00008093620590936305A0936405B093650586
:101C10003BC06AE270E0C8010E946670892BA1F1A6
:101C2000E1EAF1E007C09091C00095FFFCCF8093FE
:101C3000C600319684918111F6CFE1E2F2E007C04F
:101C40009091C00095FFFCCF8093C600319684919F
:101C50008111F6CF40916205509163056091640552
:101C6000709165052AE030E089EA95E00E94142829
:101C70008091C00085FFFCCF8AE08093C60010925F
:101C80005B0510925A05EFC18091D0039091D1036A
:101C9000789E8001799E100D1124F2EDEF2EF3E075
:101CA000FF2EE00EF11E67E470E0C7010E9466702F
:101CB000009709F442C090935D0580935C058E19EE
:101CC0009F09800F911F60E070E08D529C4F0E9431
:101CD000AF6D0E94E8696430710578F58091CE029D
:101CE000811117C08091F402811127C08A2DEAE486
:101CF000F2E008C09091C00095FFFCCF8093C60031
:101D0000319684918111F6CF8091C00085FFFCCF80
:101D100012C0882DEDE4F2E008C09091C00095FF5C
:101D2000FCCF8093C600319684918111F6CF8091CB
:101D3000C00085FFFCCFB092C6008091D003909187
:101D4000D1030196B2010E94376D9093D103809325
:101D5000D0038091CE039091CF0301969093CF034F
:101D60008093CE0310925B0510925A050ACE8B33F6
:101D700011F49092590590915905911102CE40911C
:101D8000D0035091D103749ED001759EB00D1124E3
:101D9000A20FB31FAE52BC4F8C932F5F3F4F3093B7
:101DA0005B0520935A05EDCD8091CE039091CF0332
:101DB00004970CF42FC129C180915A0590915B05BD
:101DC000892B09F4E8C04FC14D3081F04A3321F42A
:101DD00020915905222351F020915A0530915B053D
:101DE0002F3531051CF4019609F0B8C04091C403A9
:101DF0005091C5036091C6037091C7038091BC03E5
:101E00009091BD03A091BE03B091BF03481759073D
:101E10006A077B0708F46DC08F8DE5ECF2E008C01F
:101E20009091C00095FFFCCF8093C60031968491BD
:101E30008111F6CF8091C00085FFFCCF7092C60063
:101E40000E9462256093660570936705809368051C
:101E50009093690520916A0530916B0540916C055E
:101E600050916D05621B730B840B950BA7019601B6
:101E70000E944B6DCA01B901A50194010E944B6DEE
:101E80007F936F933F932F9380E991E09F938F937C
:101E90003F922F920E94AF70862D0FB6F894DEBF4E
:101EA0000FBECDBFE7ECF0E008C09091C00095FFF9
:101EB000FCCF8093C600319684918111F6CFF10159
:101EC00006C09091C00095FFFCCF8093C600819121
:101ED0008111F7CF8091C00085FFFCCF7092C600C2
:101EE00084EF92E00E94CC6561E084EF92E00E9472
:101EF000C36420915A0530915B052115310519F411
:101F000010925905B0C08091D0039091D103189FD1
:101F1000F001199FF00D1124E20FF31FEE52FC4F58
:101F20001082FC01EE5AFA4F00832091CE033091CB
:101F3000CF032F5F3F4F3093CF032093CE03019603
:101F4000B2010E94376D9093D1038093D003109219
:101F5000590510925B0510925A053BC04B3311F4A2
:101F60000093590580915905811133C08091D003A8
:101F70009091D103189FF001199FF00D1124E20FE9
:101F8000F31FEE52FC4F40832F5F3F4F30935B05B2
:101F900020935A051EC010E601E044E0442E512C67
:101FA000E5ECF2E034913F8F5AE0752E68EEC62ED4
:101FB00063E0D62EE12CF12C7CE3872E912CA12C12
:101FC000B12C22242394312C2C0E3D1EE7ECF0E0A2
:101FD00064904091C4035091C5036091C603709111
:101FE000C7038091BC039091BD03A091BE03B09143
:101FF000BF03481759076A077B07A8F58091CE03EE
:102000009091CF030497A4F02EC08091F502811126
:10201000D3CE29C089EA95E00E94472780935805CE
:1020200020915A0530915B058A3009F0BACCC5CCB5
:102030008091A9039091AA03A091AB03B091AC0346
:102040008093C4039093C503A093C603B093C703C2
:1020500081EA93E00E94AB2B482F809358058A3089
:1020600009F0B2CEC3CE6F960FB6F894DEBF0FBEA6
:10207000CDBFDF91CF911F910F91FF90EF90DF9037
:10208000CF90BF90AF909F908F907F906F905F9018
:102090004F903F902F9008958F929F92AF92BF9252
:1020A000CF92DF92EF92FF920F931F93CF93DF9324
:1020B00008E2A02E02E0B02E0DED12E0C6E7D5E05A
:1020C00080EF882E82E0982EF50181915F010E94B9
:1020D000290C882319F10E94150C6B017C01F40175
:1020E0008081811103C06091860501C061E070E0CC
:1020F00080E090E00E941B6AF801208131814281DA
:1021000053810E944E6C9B01AC01C701B6010E9435
:10211000A068688379838A839B8309C0F8018081E2
:102120009181A281B38188839983AA83BB830C5F49
:102130001F4F2496FFEF8F1A9F0A8CE2A81682E0A9
:10214000B80611F686E40E94290C8823D9F00E9473
:10215000150C6B017C016093900570939105809341
:1021600092059093930520E030E0A9010E947C6BDA
:10217000181644F4C0921401D0921501E092160191
:10218000F0921701DF91CF911F910F91FF90EF9087
:10219000DF90CF90BF90AF909F908F9008950E9456
:1021A0004C1089E40E94290C882359F00E94150CD8
:1021B0006093940570939505809396059093970589
:1021C00008C01092940510929505109296051092F1
:1021D00097058AE40E94290C882359F00E94150C67
:1021E000609398057093990580939A0590939B0549
:1021F0000895109298051092990510929A051092E0
:102200009B050895CF92DF92EF92FF920F931F9359
:1022100020E030E0A901609176057091770580910A
:102220007805909179050E94796987FF08C010921E
:10223000760510927705109278051092790520E0C6
:1022400030E0A90160917A0570917B0580917C0551
:1022500090917D050E94796987FF08C010927A05E8
:1022600010927B0510927C0510927D0520E030E0F5
:10227000A90160917E0570917F0580918005909104
:1022800081050E94796987FF08C010927E0510922F
:102290007F05109280051092810520E030E04BE12F
:1022A00053E460917605709177058091780590915F
:1022B00079050E947C6B181664F480E090E0ABE135
:1022C000B3E48093760590937705A0937805B09357
:1022D000790520E030E046E153E460917A057091A1
:1022E0007B0580917C0590917D050E947C6B181682
:1022F00064F480E090E0A6E1B3E480937A059093E3
:102300007B05A0937C05B0937D0520E030E044EB95
:1023100052E460917E0570917F05809180059091D7
:1023200081050E947C6B181664F480E090E0A4EBB9
:10233000B2E480937E0590937F05A0938005B093CF
:1023400081050E94622560936E0570936F058093EE
:1023500070059093710560910201709103018827C7
:1023600077FD8095982F0E941B6A2091140130916F
:10237000150140911601509117010E944E6C20E00A
:1023800030E040E752E40E94806920E030E048EC11
:1023900052E40E94806920EDC22E22E0D22E7B0101
:1023A0008C0122E835E04EE755E06AE775E086E704
:1023B00095E00E9432408091760590917705A0913A
:1023C0007805B09179058093DD029093DE02A093A9
:1023D000DF02B093E00280917A0590917B05A09195
:1023E0007C05B0917D058093E1029093E202A09379
:1023F000E302B093E40280917E0590917F05A09165
:102400008005B09181058093E5029093E602A09348
:10241000E702B093E8028091820590918305A09134
:102420008405B09185058093E9029093EA02A09318
:10243000EB02B093EC021F910F91FF90EF90DF90B1
:10244000CF900895AF92BF92CF92DF92EF92FF921A
:102450000F931F93CF93DF93182F209198053091FE
:10246000990540919A0550919B0560919405709152
:10247000950580919605909197050E94896BEB01D7
:10248000082FF92E6091020170910301882777FDD2
:102490008095982F0E941B6A20911401309115019C
:1024A00040911601509117010E944E6C20E030E0DF
:1024B00040E752E40E94806920E030E048EC52E4BA
:1024C0000E9480692091D0022F931F93FF920F9357
:1024D000DF93CF935B016C0132E0E32E01E020E05B
:1024E00044E955E066E775E08DED92E00E948B3699
:1024F0008091760590917705A0917805B091790546
:102500008093DD029093DE02A093DF02B093E0029D
:1025100080917A0590917B05A0917C05B0917D0515
:102520008093E1029093E202A093E302B093E4026D
:1025300080917E0590917F05A0918005B0918105E5
:102540008093E5029093E602A093E702B093E8023D
:102550008091820590918305A0918405B0918505B5
:102560008093E9029093EA02A093EB02B093EC020D
:102570000E94622560936E0570936F0580937005CD
:10258000909371050F900F900F900F900F900F90F8
:10259000DF91CF911F910F91FF90EF90DF90CF903F
:1025A000BF90AF900895F8940E94D6575E9A5E9AB5
:1025B000159A5E9AE1EAF1E007C09091C00095FF9C
:1025C000FCCF8093C600319684918111F6CFEBE069
:1025D000F4E007C09091C00095FFFCCF8093C60047
:1025E000319684918111F6CF8091C00085FFFCCF98
:1025F0008AE08093C600FFCFCF92DF92EF92FF92E6
:102600000F931F930E946225009188051091890500
:1026100020918A0530918B05C0906E05D0906F0592
:10262000E0907005F09071056C197D098E099F0985
:10263000061717072807390730F4012B022B032B45
:1026400011F00E94D3128091190190911A01A0916A
:102650001B01B0911C01892B8A2B8B2B09F10E9445
:10266000622500916E0510916F05209170053091E3
:102670007105601B710B820B930B00911901109176
:102680001A0120911B0130911C010617170728071A
:10269000390730F490913D0880913C08981741F03B
:1026A0001F910F91FF90EF90DF90CF900C940E4010
:1026B0005E9A5E9A159A5E9AF3CF2F923F924F924E
:1026C0005F926F927F928F929F92AF92BF92CF92C2
:1026D000DF92EF92FF920F931F93CF93DF93CDB7CB
:1026E000DEB7A6970FB6F894DEBF0FBECDBF87E466
:1026F0000E94290C882309F40EC20E94150C0E9426
:10270000E86964307105D9F144F46230710521F152
:102710005CF577FF17C00C9402216A35710509F446
:10272000A6C134F46C31710511F00C9402216AC019
:102730006B35710509F49FC16C35710511F00C946E
:1027400002219EC18091CE02811106C00E944C10D0
:102750000E9402110C940C248091CE02811104C0BD
:102760000E94CF1081E007C08091CE02811107C086
:102770000E94CF1080E00E9422120C940C2480E56D
:102780000E94290C882339F00E94150C0E94ED69E3
:102790006B017C0103C0C12CD12C760183E50E9422
:1027A000290C882361F00E94150C20E030E04AE7F4
:1027B00054E40E944E6C0E94ED696B017C010E9402
:1027C000A3520E9462254B015C018C0C9D1CAE1C27
:1027D000BF1C0E94622560936E0570936F05809305
:1027E00070059093710505C00E94F45481E00E9429
:1027F000FC120E946225681579058A059B05A0F3E5
:102800000C9402218091140190911501A091160160
:10281000B09117018093720590937305A09374058E
:10282000B093750580910201909103019093EF029E
:102830008093EE0284E690E090930301809302017E
:102840000E94622560936E0570936F0580937005FA
:102850009093710581E00E943D4C8091DD02909142
:10286000DE02A091DF02B091E002809376059093A2
:102870007705A0937805B09379058091E102909156
:10288000E202A091E302B091E40280937A05909372
:102890007B05A0937C05B0937D058091E502909126
:1028A000E602A091E702B091E80280937E05909342
:1028B0007F05A0938005B09381058091E9029091F6
:1028C000EA02A091EB02B091EC0280938205909312
:1028D0008305A0938405B09385051092140110928E
:1028E0001501109216011092170188E50E94290C1B
:1028F000882311F090E00AC089E50E94290C81111B
:10290000F9CF8AE50E94290C91E09827909318014D
:1029100091110C94052188E50E94290C81110C94D9
:1029200005218091180181110C94DD2189E50E9417
:10293000290C81110C94DD218091180181110C94D6
:10294000B5228AE50E94290C81110C94B52288E5F4
:102950000E94290C8823D1F00E941E0C672B682B43
:10296000692BA1F00E94150C2091D1023091D20266
:102970004091D3025091D4020E94A0686093DD027E
:102980007093DE028093DF029093E00289E50E945B
:10299000290C8823D1F00E941E0C672B682B692B11
:1029A000A1F00E94150C2091D5023091D6024091E1
:1029B000D7025091D8020E94A0686093E102709300
:1029C000E2028093E3029093E4028AE50E94290CDC
:1029D0008823D1F00E941E0C672B682B692BA1F075
:1029E0000E94150C2091D9023091DA024091DB024D
:1029F0005091DC020E94A0686093E5027093E602A9
:102A00008093E7029093E80229EE32E045EE52E02F
:102A100061EE72E08DED92E00E94C14A80E00E947A
:102A20003D4C8091720590917305A0917405B09111
:102A300075058093140190931501A0931601B0932E
:102A400017018091EE029091EF0290930301809321
:102A500002010E94622560936E0570936F0580935A
:102A60007005909371050E94364C0C9402211092CF
:102A700086050C94022181E0809386050C94022146
:102A800085E40E94290C811102C00E94A35258E2E1
:102A9000C52E52E0D52E61EDE62E62E0F62E0DED4C
:102AA00012E0B12CF60181916F010E94290C88235C
:102AB00039F1F3E0BF120CC00E94150CF8016083DD
:102AC00071838283938389EE92E00E945D4B18C0EC
:102AD0000E94150CF70120813181428153810E94AF
:102AE000A068F801608371838283938329EE32E0CA
:102AF00045EE52E061EE72E08DED92E00E94C14A37
:102B0000B394F4E0EF0EF11C0C5F1F4F24E0B212FF
:102B1000C9CF0C9402218DE40E94290C882311F462
:102B20000C9455200E94150C0E94E8696D367105C1
:102B300009F4F7C30CF06BC06C31710509F461C185
:102B40009CF56631710509F419C1ACF46231710567
:102B500009F45CC634F46131710511F00C94022162
:102B6000D6C06431710509F4D8C06531710511F022
:102B70000C940221FDC06931710509F428C154F497
:102B80006731710509F400C16831710511F00C94C9
:102B900002210DC16A31710509F41FC16B31710544
:102BA00011F00C94022127C16335710509F42AC67E
:102BB000ACF46F31710509F497C134F46E317105CD
:102BC00011F00C94022152C16A32710509F424C239
:102BD0006235710511F00C94022111C66C35710536
:102BE00009F465C654F46435710509F40FC66535FA
:102BF000710511F00C94022144C66836710509F480
:102C000048C26936710511F00C940221B8C26D3CBE
:102C1000710511F40C94AE1ECCF56937710511F4F1
:102C20000C94D51DBCF46337710509F4D2C634F495
:102C30006237710511F00C940221D9C6673771050E
:102C400011F40C94D91D6837710511F00C94022110
:102C50000C94D31D693C710511F40C94381E54F486
:102C60006C38710509F477C26E3B710511F00C9454
:102C7000022129C56B3C710511F40C94721E6C3C49
:102C8000710511F00C9402210C948E1E6E3231E00D
:102C9000730711F40C942420CCF46C3D710511F4ED
:102CA0000C94281F3CF46E3C710511F00C94022129
:102CB0000C940C1F6D3D710511F40C943A1F6D328C
:102CC000714011F00C9402210C94491F653FE1E022
:102CD0007E0711F40C943A206CF46F3221E07207F5
:102CE00011F40C9428206039714011F00C940221E9
:102CF0000C943720663F81E0780711F40C943C2057
:102D0000673E734011F00C9402210C9440205E98B1
:102D10005E9815985E980C940221E8EDF2E007C0E9
:102D20009091C00095FFFCCF8093C60031968491AE
:102D30008111F6CF8091C00085FFFCCF8AE080939F
:102D4000C60084EF92E00E94BD5FE8EEF2E007C0AB
:102D50009091C00095FFFCCF8093C600319684917E
:102D60008111F6CF8091C00085FFFCCF0C94FF202D
:102D700084EF92E00E94FF5F0C94022184EF92E0C6
:102D80000E94C5600C94022100915C0510915D05C4
:102D90000C5F1F4F6AE270E0C8010E9466700097E6
:102DA00019F0FC013197108241E0B80159C084EF5D
:102DB00092E00E94C9600E94622560936A05709348
:102DC0006B0580936C0590936D050C94022184EF44
:102DD00092E00E94D0600C9402218091F602882338
:102DE00011F40C94022183E50E94290C81110C94AA
:102DF0008D230C94022184EF92E00E9400640C94D5
:102E0000022180915C0590915D056AE270E0049674
:102E10000E9466708C010097E1F020915605309178
:102E2000570540E6429FC001439F900D11246EE478
:102E300070E08E529C4F0E94667060E270E00E94CB
:102E40006670019690935D0580935C05F80131975B
:102E5000108260915C0570915D056C5F7F4F40E072
:102E600084EF92E00E94D5600C9402218091F602DA
:102E7000882311F40C94022184EF92E00E94B7653C
:102E800080915C0590915D056AE270E004960E9475
:102E900066708C010097E1F020915605309157053E
:102EA00040E6429FC001439F900D11246EE470E004
:102EB0008E529C4F0E94667060E270E00E946670C5
:102EC000019690935D0580935C05F801319710821F
:102ED00060915C0570915D056C5F7F4F84EF92E0BF
:102EE0000E94C4620C9402210E94622560936605D0
:102EF00070936705809368059093690500916A0552
:102F000010916B0520916C0530916D05601B710B64
:102F1000820B930B28EE33E040E050E00E944B6DB3
:102F2000CA01B9012CE330E040E050E00E944B6D53
:102F30007F936F933F932F9380E991E09F938F93BB
:102F4000CE0101969F938F930E94AF70E7ECF0E063
:102F500084910FB6F894DEBF0FBECDBFE7ECF0E072
:102F600008C09091C00095FFFCCF8093C6003196B9
:102F700084918111F6CFFE01319606C09091C00078
:102F800095FFFCCF8093C60081918111F7CF80918E
:102F9000C00085FFFCCF8AE08093C60080910E0DB3
:102FA000882311F40C94022110920E0D6091D0022E
:102FB000E62FF0E0EE0FFF1FE851F24F8081918184
:102FC0000E94285420912101309122014091230137
:102FD000509124010E947C6B181614F00C9402216D
:102FE0006091D002062F10E080E090E00E945853DC
:102FF000F801EE0FFF1FE851F24F91838083F80133
:10300000EE0FFF1FEE0FFF1FE252F24F10821182F0
:10301000128213820C94022183E50E94290C8823DA
:1030200011F40C9402210E94150C0E94E8697B01A6
:1030300080E50E94290C882311F40C940221F7FEEC
:1030400002C00C940221FFEFEF16F10409F014F412
:103050000C949E230C9402218191919180179107E9
:1030600011F40C94022122E0E03AF207A9F717FFCD
:1030700002C00C94022161E0802F0E948A266E2DEE
:10308000802F0E94A626B701802F0E94FF250C9456
:1030900002218091D0028093870584E50E94290C4B
:1030A000882379F10E94150C0E94ED6960938705D1
:1030B000662339F1E7ECF0E007C09091C00095FF7E
:1030C000FCCF8093C600319684918111F6CFE5EA5A
:1030D000F1E006C09091C00095FFFCCF8093C60040
:1030E00081918111F7CF40E050E06091870589EA36
:1030F00095E00E940D288091C00085FFFCCF0C94C4
:10310000FF2083E50E94290C882309F1B0908705F0
:103110000E94150C6B017C010B2D10E00E94E869E8
:10312000DC01CB016B2D0E945853F801EE0FFF1FFD
:10313000E851F24F91838083F801EE0FFF1FEE0FED
:10314000FF1FE252F24FC082D182E282F3820E94DC
:10315000D5570C94022183E50E94290C882311F491
:103160000C9402210E94150C0E94E869CB010E9478
:10317000DC539093E70D8093E60D0C94022180912F
:10318000D0028093870584E50E94290C882379F179
:103190000E94150C0E94ED6960938705662339F142
:1031A000E7ECF0E007C09091C00095FFFCCF809362
:1031B000C600319684918111F6CFECEBF1E006C0A8
:1031C0009091C00095FFFCCF8093C6008191811142
:1031D000F7CF40E050E06091870589EA95E00E94D2
:1031E0000D288091C00085FFFCCF0C94FF20E6EFF6
:1031F000F2E007C09091C00095FFFCCF8093C6001D
:10320000319684918111F6CF60918705E62FF0E029
:10321000EE0FFF1FEC51F24F808191810E942854E4
:10322000AB01BC0121E030E089EA95E00E941E2953
:10323000ECEFF2E007C09091C00095FFFCCF8093C7
:10324000C600319684918111F6CF60918705E62FF3
:10325000F0E0EE0FFF1FE851F24F808191810E9454
:103260002854AB01BC0121E030E089EA95E00E94DE
:103270001E29EFEFF2E007C09091C00095FFFCCF50
:103280008093C600319684918111F6CF8091E20D32
:103290009091E30D0E94E256AB01BC0121E030E0C9
:1032A00089EA95E00E941E29E3E0F3E007C09091CF
:1032B000C00095FFFCCF8093C600319684918111A8
:1032C000F6CF8091E60D9091E70D0E94E256AB019A
:1032D000BC0121E030E089EA95E00E941E29E6E089
:1032E000F3E007C09091C00095FFFCCF8093C6002B
:1032F000319684918111F6CF8091870590E00E94EC
:1033000052534AE050E0BC0189EA95E00E9425282A
:103310008091C00085FFFCCF8AE08093C6000C94AA
:103320000C248091D0028093870584E50E94290CAB
:10333000882371F10E94150C0E94ED696093870546
:10334000662331F1E7ECF0E007C09091C00095FFF3
:10335000FCCF8093C600319684918111F6CFE3EDC6
:10336000F1E006C09091C00095FFFCCF8093C600AD
:1033700081918111F7CF40E050E06091870589EAA3
:1033800095E00E940D288091C00085FFFCCF37C7D3
:1033900010920E0D83E50E94290C882309F1B0904C
:1033A00087050E94150C6B017C010B2D10E00E941B
:1033B000E869DC01CB016B2D0E945853F801EE0F38
:1033C000FF1FE851F24F91838083F801EE0FFF1F3A
:1033D000EE0FFF1FE252F24FC082D182E282F382EF
:1033E00083E50E94290C882351F00E94150C6093FC
:1033F000210170932201809323019093240182E4A0
:103400000E94290C882351F00E94150C609325011D
:1034100070932601809327019093280186E40E94EF
:10342000290C882369F00E94150C60931D0170938C
:103430001E0180931F019093200181E080930E0D67
:103440000E94D5570E9462254B015C01809187053F
:1034500090E0880F991FFC01E851F24F20813181E3
:1034600038A32F8FFC01EC51F24F808191819EA3F4
:103470008DA3CC24CA94DC2C7601EAE0F3E02490FE
:10348000EDE0F3E03490E1E1F3E0049148EE442E06
:1034900043E0542E612C712C1AE00C94C223822D2F
:1034A000EAE0F3E008C09091C00095FFFCCF809364
:1034B000C600319684918111F6CF60918705E62F81
:1034C000F0E0EE0FFF1FEC51F24F808191810E94DE
:1034D0002854AB01BC0121E030E089EA95E00E946C
:1034E0001E29832DEDE0F3E008C09091C00095FF08
:1034F000FCCF8093C600319684918111F6CF609104
:1035000087054AE050E070E089EA95E00E942528AE
:10351000802FE1E1F3E008C09091C00095FFFCCF5F
:103520008093C600319684918111F6CFF7FE03C0D7
:10353000EAEEF1E027C00E9462254B015C01C70161
:10354000B601605F784D8F4F9F4F681979098A09DE
:103550009B09A30192010E944B6D49015A012AE087
:1035600030E0B501A40189EA95E00E94012880912C
:10357000C00085FFFCCF0DC09091C00095FFFCCF2F
:103580008093C60081918111F7CF8091C00085FFA3
:10359000FCCF1093C6000E9462254B015C010E9483
:1035A000F45481E00E94FC129FEFC916D906E90687
:1035B000F906C1F560918705EF8DF8A12DA13EA117
:1035C0002E173F0714F00C94DF23E62FF0E0EE0FE8
:1035D000FF1FEC51F24F808191810E94285469A312
:1035E0007AA38BA39CA360918705E62FF0E0EE0FF2
:1035F000FF1FE851F24F808191810E94285420E002
:1036000030E040E85FE30E949F689B01AC0169A144
:103610007AA18BA19CA10E947C6B87FD02C00C94B7
:10362000A7233AC0F7FC38C060918705E62FF0E089
:10363000EE0FFF1FEC51F24F808191810E942854C0
:1036400069A37AA38BA39CA360918705E62FF0E082
:10365000EE0FFF1FE851F24F808191810E942854A4
:103660009B01AC0169A17AA18BA19CA10E949F68DA
:103670000E94E869AB01BC0177FF07C070956095B7
:10368000509541955F4F6F4F7F4F44305105610515
:10369000710514F00C94A7233FEFC316D306E3067D
:1036A000F30611F40C94C223F7FE02C00C94AD2370
:1036B0000E9462256C197D096031774210F40C94E8
:1036C000C2230C94AD2383E50E94290C882359F072
:1036D0000E94150C0E94E869CB010E94DC53909374
:1036E000E70D8093E60D0E9462256B017C01E5E108
:1036F000F3E0A490E8E1F3E0B490ECE1F3E014919E
:103700000AE070C00E9462256C197D098E099F092C
:10371000693E73408105910508F45FC06091D00255
:10372000A62FB0E0AA0FBB1FAC51B24F8D919C9158
:103730000E942854AB01BC018A2DE5E1F3E008C0EA
:103740009091C00095FFFCCF8093C6003196849184
:103750008111F6CF22E030E089EA95E00E941E292F
:103760008B2DE8E1F3E008C09091C00095FFFCCFFD
:103770008093C600319684918111F6CF6091D0027A
:103780004AE050E070E089EA95E00E942528812F08
:10379000ECE1F3E008C09091C00095FFFCCF80936E
:1037A000C600319684918111F6CF8091E20D9091FF
:1037B000E30D0E94E256AB01BC0121E030E089EA52
:1037C00095E00E941E298091C00085FFFCCF0093E8
:1037D000C6000E9462256B017C010E94F45481E0C6
:1037E0000E94FC122091E60D3091E70D8091E20DD0
:1037F0009091E30D821793070CF484CFB8C7109211
:10380000F30200C581E08093F302FCC483E50E94CB
:10381000290C882399F00E94150C20E030E04AE73B
:1038200054E40E944E6C0E94ED69609319017093FC
:103830001A0180931B0190931C01E4C488E50E9447
:10384000290C8111B4C789E50E94290C8111AFC7E9
:103850008AE50E94290C8111AAC785E40E94290CDF
:103860008111A5C79EC75E9A89E50E94290C811126
:103870005E9A8AE50E94290C882309F4C3C4159A2C
:10388000C1C483E50E94290C0E94150C20E030E0A1
:103890004AE754E40E944E6C0E94ED6960938805EB
:1038A0007093890580938A0590938B05ABC428E2B9
:1038B00032E03EA32DA35BE5252E5DE0352E8BE6A1
:1038C0009DE098A38F8F6FE1862E6DE0962E10E01D
:1038D000EDA1FEA18191FEA3EDA30E94290C8823F6
:1038E00009F466C0133009F05CC00E94150C6B012E
:1038F0007C0120E030E040EA51E40E94796987FFD2
:103900004AC0A7019601F101608171818281938192
:103910000E948069762EA72EB82E092F762F272F8A
:103920003A2D4B2D502F6091330D7091340D8091B5
:10393000350D9091360D0E944E6C6093330D70934F
:10394000340D8093350D9093360D272D3A2D4B2D48
:10395000502FEF8DF8A160817181828193810E9447
:103960004E6CEF8DF8A16083718382839383F401A1
:1039700060817181828193810E94196A272D3A2D7D
:103980004B2D502F0E944E6C0E94ED69F401608314
:10399000718382839383F101C082D182E282F382B8
:1039A00007C00E94150CF1016083718382839383A9
:1039B0001F5FF4E02F0E311C2F8D38A12C5F3F4F7D
:1039C00038A32F8F34E0830E911C143009F080CF80
:1039D00019C4E0E2F3E007C09091C00095FFFCCF6E
:1039E0008093C600319684918111F6CF0BC4EBEB26
:1039F000F3E007C09091C00095FFFCCF8093C60014
:103A0000319684918111F6CF4091DD025091DE0212
:103A10006091DF027091E00222E030E089EA95E0F7
:103A20000E941E29EEEBF3E007C09091C00095FFC5
:103A3000FCCF8093C600319684918111F6CF4091DE
:103A4000E1025091E2026091E3027091E40222E00F
:103A500030E089EA95E00E941E29E1ECF3E007C01E
:103A60009091C00095FFFCCF8093C6003196849161
:103A70008111F6CF4091E5025091E6026091E70294
:103A80007091E80222E030E089EA95E00E941E2968
:103A9000E4ECF3E007C09091C00095FFFCCF809369
:103AA000C600319684918111F6CF4091E902509180
:103AB000EA026091EB027091EC0222E030E089EAC8
:103AC00095E00E941E29E7ECF3E007C09091C0004A
:103AD00095FFFCCF8093C600319684918111F6CF7B
:103AE0000E94FD520E941B6A20915B0D30915C0D7B
:103AF00040915D0D50915E0D0E948069AB01BC014B
:103B000022E030E089EA95E00E941E29E1EDF3E031
:103B100007C09091C00095FFFCCF8093C6003196FE
:103B200084918111F6CF81E00E94FD520E941B6AB0
:103B300020915F0D3091600D4091610D5091620DAB
:103B40000E948069AB01BC0122E030E089EA95E087
:103B50000E941E29E4EDF3E007C09091C00095FF9C
:103B6000FCCF8093C600319684918111F6CF82E01C
:103B70000E94FD520E941B6A2091630D3091640DDA
:103B80004091650D5091660D0E948069AB01BC01AA
:103B900022E030E089EA95E00E941E298091C00071
:103BA00085FFFCCF2CC380E001C081E00E943D4C2A
:103BB00029C3E7EDF3E007C09091C00095FFFCCF6B
:103BC0008093C600319684918111F6CF329B03C059
:103BD000EFE9F1E009C0E2EAF1E006C09091C0002F
:103BE00095FFFCCF8093C60081918111F7CFEEED58
:103BF000F3E007C09091C00095FFFCCF8093C60012
:103C0000319684918111F6CF339B03C0EFE9F1E047
:103C100009C0E2EAF1E006C09091C00095FFFCCF38
:103C20008093C60081918111F7CFE5EEF3E007C0E4
:103C30009091C00095FFFCCF8093C600319684918F
:103C40008111F6CF349B03C0EFE9F1E009C0E2EA4D
:103C5000F1E006C09091C00095FFFCCF8093C600B4
:103C600081918111F7CF8091C00085FFFCCFC7C241
:103C700048E2E42E42E0F42E00E010E0F7018191EA
:103C80007F010E94290C882339F10E94150C2BE436
:103C9000C22E2DE0D22EC00ED11E0E94ED69F6017B
:103CA00060837183828393830E94150C3FE1C32E4E
:103CB0003DE0D32EC00ED11EF801E55AF24F20810F
:103CC0003181428153810E944E6C0E94ED69F60160
:103CD00060837183828393830C5F1F4F00311105D2
:103CE00069F690C208E212E08BE6E82E8DE0F82E2D
:103CF000F80181918F010E94290C882339F00E94DC
:103D0000150CF7016083718382839383F4E0EF0ED7
:103D1000F11C22E00C32120759F774C283E50E94AD
:103D2000290C882351F00E94150C6093430D709369
:103D3000440D8093450D9093460D84E50E94290C17
:103D4000882309F45FC20E94150C60933F0D7093A5
:103D5000400D8093410D9093420D54C283E50E9423
:103D6000290C882351F00E94150C6093470D709325
:103D7000480D8093490D90934A0D84E50E94290CCB
:103D8000882351F00E94150C60932F0D7093300D15
:103D90008093310D9093320D82E40E94290C882388
:103DA00061F00E94150C0E94ED6960937B0D709389
:103DB0007C0D80937D0D90937E0D88E50E94290CEB
:103DC000882351F00E94150C60933B0D70933C0DBD
:103DD00080933D0D90933E0D8AE50E94290C882327
:103DE00051F00E94150C6093370D7093380D80933D
:103DF000390D90933A0D85E40E94290C882309F42B
:103E000001C20E94150C6093330D7093340D8093A2
:103E1000350D9093360DF6C108E212E0B1EDEB2EB0
:103E2000B2E0FB2EF80181918F010E94290C8823BA
:103E300039F00E94150CF7016083718382839383AC
:103E4000F4E0EF0EF11C22E00B32120759F7DAC151
:103E500083E50E94290C882309F4D4C10E94150C23
:103E60000E94E869709303016093020181E08093EE
:103E7000ED02C8C183E50E94290C882309F4C2C160
:103E80000E94150C0E94E869709301016093000183
:103E9000B9C180E50E94290C882351F00E94150CBD
:103EA00060933A0170933B0180933C0190933D01F4
:103EB00089E40E94290C882381F00E94150C2DEBC7
:103EC00037E346E05EE30E944E6C609336017093E8
:103ED0003701809338019093390184E40E94290CC2
:103EE000882381F00E94150C2DEB37E346E05EE35A
:103EF0000E94806960933201709333018093340192
:103F00009093350183E40E94290C882351F00E948C
:103F1000150C60932E0170932F01809330019093C4
:103F200031010E943B53ECEEF1E006C09091C000DD
:103F300095FFFCCF8093C60081918111F7CFEFEE02
:103F4000F1E006C09091C00095FFFCCF8093C600C1
:103F500081918111F7CF40913A0150913B016091DD
:103F60003C0170913D0122E030E089EA95E00E9439
:103F70001E29E3EFF1E006C09091C00095FFFCCF51
:103F80008093C60081918111F7CF2DEB37E346E096
:103F90005EE3609136017091370180913801909114
:103FA00039010E948069AB01BC0122E030E089EA5E
:103FB00095E00E941E29E7EFF1E006C09091C00055
:103FC00095FFFCCF8093C60081918111F7CF2DEB37
:103FD00037E346E05EE360913201709133018091F6
:103FE0003401909135010E944E6CAB01BC0122E07E
:103FF00030E089EA95E00E941E29EBEFF1E006C06F
:104000009091C00095FFFCCF8093C60081918111F3
:10401000F7CF2DEB37E346E05EE360912E01709120
:104020002F0180913001909131010E944E6CAB01C3
:10403000BC0122E030E089EA95E00E941E298091CF
:10404000C00085FFFCCFDBC081E00E94774BDAC067
:1040500083E50E94290C882319F00E94150C04C0E6
:1040600060E070E086E193E40E94F857CBC00E94C4
:10407000A352C8C080E001C081E00E94FB08C2C01A
:104080001092CE0280918C0590918D05A0918E05A5
:10409000B0918F058093620590936305A0936405AA
:1040A000B09365050E946C0CADC084E50E94290C9C
:1040B000882309F463C00E94150C0E94ED69609387
:1040C0008705662391F1E7ECF0E007C09091C0000E
:1040D00095FFFCCF8093C600319684918111F6CF75
:1040E000EFEFF1E006C09091C00095FFFCCF809308
:1040F000C60081918111F7CF40E050E060918705C3
:1041000089EA95E00E940D28E1E0F2E006C0909176
:10411000C00095FFFCCF8093C60081918111F7CF3D
:104120008091C00085FFFCCF6AC01092D002E7ECFE
:10413000F0E007C09091C00095FFFCCF8093C600CF
:10414000319684918111F6CFE2E1F2E006C09091C0
:10415000C00095FFFCCF8093C60081918111F7CFFD
:104160006091D0024AE050E070E089EA95E00E9458
:1041700025288091C00085FFFCCF41C0E7ECF0E02E
:1041800007C09091C00095FFFCCF8093C600319688
:1041900084918111F6CFECEEF3E007C09091C0005E
:1041A00095FFFCCF8093C600319684918111F6CFA4
:1041B000809156059091570520E6289FF001299F90
:1041C000F00D1124EE52FC4F06C09091C00095FFF7
:1041D000FCCF8093C60081918111F7CFEEEFF3E021
:1041E00007C09091C00095FFFCCF8093C600319628
:1041F00084918111F6CF8091C00085FFFCCF8AE0C9
:104200008093C6000E94440C07C31092DD021092F6
:10421000DE021092DF021092E00229EE32E045EE5B
:1042200052E061EE72E08DED92E00E94C14A80E0C2
:1042300090E8A8E6B3EC8093760590937705A09379
:104240007805B09379056091040170910501809122
:1042500006019091070160931401709315018093FA
:1042600016019093170120E030E040E752E40E94ED
:104270008069A0EDCA2EA2E0DA2E7B018C0122E833
:1042800035E04EE755E06AE775E086E795E00E9485
:1042900032400E94A3521092DD021092DE02109270
:1042A000DF021092E00229EE32E045EE52E061EECC
:1042B00072E08DED92E00E94C14A80E090E0A0EAB9
:1042C000B0E48093760590937705A0937805B0933A
:1042D000790520E030E040E752E4609114017091EC
:1042E000150180911601909117010E9480697B0150
:1042F0008C0122E835E04EE755E06AE775E086E795
:1043000095E00E9432400E94A35280E090E0A0E23B
:10431000B1EC8093760590937705A0937805B093E0
:10432000790520E030E040E05FE3609104017091A6
:10433000050180910601909107010E944E6CFB01DE
:10434000462F5F2F682F792F40931401509315014A
:10435000609316017093170120E030E040E752E4CB
:10436000BF010E9480697B018C0122E835E04EE7A5
:1043700055E06AE775E086E795E00E9432400E94CA
:10438000A3521092DD021092DE021092DF02109210
:10439000E00210927605109277051092780510923F
:1043A00079051092140110921501109216011092C5
:1043B00017010E94364C0C9491141092E102109255
:1043C000E2021092E3021092E40229EE32E045EE9E
:1043D00052E061EE72E08DED92E00E94C14A80E011
:1043E00090E0A1E6B3EC80937A0590937B05A093CF
:1043F0007C05B0937D056091080170910901809161
:104400000A0190910B016093140170931501809340
:1044100016019093170120E030E040E752E40E943B
:104420008069F0EDCF2EF2E0DF2E7B018C0122E8D7
:1044300035E04EE755E06AE775E086E795E00E94D3
:1044400032400E94A3521092E1021092E2021092B6
:10445000E3021092E40229EE32E045EE52E061EE12
:1044600072E08DED92E00E94C14A80E090E0A0EA07
:10447000B0E480937A0590937B05A0937C05B0937C
:104480007D0520E030E040E752E460911401709136
:10449000150180911601909117010E9480697B019E
:1044A0008C0122E835E04EE755E06AE775E086E7E3
:1044B00095E00E9432400E94A35280E090E0A0E28A
:1044C000B1EC80937A0590937B05A0937C05B09323
:1044D0007D0520E030E040E05FE3609108017091ED
:1044E000090180910A0190910B010E944E6CFB0121
:1044F000462F5F2F682F792F409314015093150199
:10450000609316017093170120E030E040E752E419
:10451000BF010E9480697B018C0122E835E04EE7F3
:1045200055E06AE775E086E795E00E9432400E9418
:10453000A3521092E1021092E2021092E302109252
:10454000E40210927A0510927B0510927C0510927D
:104550007D0510921401109215011092160110920F
:1045600017010E94364C0C949C141092E502109294
:10457000E6021092E7021092E80229EE32E045EEE0
:1045800052E061EE72E08DED92E00E94C14A80E05F
:1045900090E0A7E0B3EC80937E0590937F05A09315
:1045A0008005B093810560910C0170910D0180919F
:1045B0000E0190910F016093140170931501809387
:1045C00016019093170120E030E040E752E40E948A
:1045D0008069E0EDCE2EE2E0DE2E7B018C0122E848
:1045E00035E04EE755E06AE775E086E795E00E9422
:1045F00032400E94A3521092E5021092E6021092FD
:10460000E7021092E80229EE32E045EE52E061EE58
:1046100072E08DED92E00E94C14A80E090E0A0E857
:10462000BFE380937E0590937F05A0938005B093B0
:10463000810520E030E040E752E460911401709180
:10464000150180911601909117010E9480697B01EC
:104650008C0122E835E04EE755E06AE775E086E731
:1046600095E00E9432400E94A35280E090E0A0E0DA
:10467000B0EC80937E0590937F05A0938005B09366
:10468000810520E030E040E05FE360910C01709133
:104690000D0180910E0190910F010E944E6CFB0163
:1046A000462F5F2F682F792F4093140150931501E7
:1046B000609316017093170120E030E040E752E468
:1046C000BF010E9480697B018C0122E835E04EE742
:1046D00055E06AE775E086E795E00E9432400E9467
:1046E000A3521092E5021092E6021092E702109295
:1046F000E80210927E0510927F05109280051092BC
:104700008105109214011092150110921601109259
:1047100017010E94364C0C94A7140E941E0CAB018A
:104720006093C4035093C5038093C6039093C7035B
:10473000BC0181EA93E00E94362C64CD0E94150CE6
:104740000E94E8698B01ECE2F2E00C942C180E94C4
:1047500062256B017C010C944C1B0E9462256093C6
:104760006A0570936B0580936C0590936D050E94AC
:10477000622560936E0570936F058093700590932A
:10478000710540CD0E946225681979098A099B0943
:10479000693E73408105910510F00C944F1A0C94FA
:1047A000CF1A0E94A3525E9A0E9411532BCD0E94F1
:1047B000A35288E50E94290C811155C855C8E62FDF
:1047C000F0E0EE0FFF1FEC51F24F808191810E94CB
:1047D000285469A37AA38BA39CA360918705E62F35
:1047E000F0E0EE0FFF1FE851F24F808191810E94AF
:1047F000285420E030E040E85FE30E94A0689B017D
:10480000AC0169A17AA18BA19CA10E9479691816BB
:104810000CF09DCF0C944C1BA6960FB6F894DEBFFF
:104820000FBECDBFDF91CF911F910F91FF90EF9001
:10483000DF90CF90BF90AF909F908F907F906F90C0
:104840005F904F903F902F900895CF93DF9380918A
:10485000CE039091CF03039714F40E94980C60E06C
:1048600084EF92E00E94C3648091CE039091CF03C5
:10487000892B09F460C08091F402882309F443C0B5
:10488000809156059091570520E6289FE001299FC9
:10489000D00D1124CE52DC4F64E272E0CE010E94B2
:1048A0009570892BB9F4BE0184EF92E00E945564A3
:1048B000ECE8F1E007C09091C00095FFFCCF809339
:1048C000C600319684918111F6CF8091C00085FF9A
:1048D000FCCF15C084EF92E00E94B765EFE8F1E0ED
:1048E00007C09091C00095FFFCCF8093C600319621
:1048F00084918111F6CF8091C00085FFFCCF8AE0C2
:104900008093C60002C00E945D138091CE039091F7
:10491000CF0301979093CF038093CE0380915605E8
:1049200090915705019664E070E00E94376D909376
:104930005705809356050E94F45481E00E94FC12B2
:10494000DF91CF910C947A4B0E94D6578091CE0282
:10495000811134C081E08093CE02809162059091F4
:104960006305A0916405B091650580938C059093D3
:104970008D05A0938E05B0938F05E1EAF1E007C0A5
:104980009091C00095FFFCCF8093C6003196849132
:104990008111F6CFECE2F4E007C09091C00095FFE2
:1049A000FCCF8093C600319684918111F6CF80911F
:1049B000C00085FFFCCF8AE08093C60008958091F7
:1049C000CE0208950E94C4250E94770A0E942524E1
:1049D000FDCF2CE632E0FC013183208325812223A8
:1049E00019F002960C941D2D0895CF93DF93EC01DE
:1049F00085559F4F0E94E924CE0185599F4F0E9403
:104A0000E924CE01825B9F4F0E94E924CE01C1962A
:104A10000E94E924CE014296DF91CF910C94E924C3
:104A200084EF92E00C94E15D84EF92E00C94F52425
:104A30001F920F920FB60F9211242F933F938F93D3
:104A40009F93AF93BF938091A0059091A105A091F2
:104A5000A205B091A3053091A805232F2D5F2D3716
:104A600020F40196A11DB11D05C0232F2A570296DF
:104A7000A11DB11D2093A8058093A0059093A105C9
:104A8000A093A205B093A3058091A4059091A505DC
:104A9000A091A605B091A7050196A11DB11D809317
:104AA000A4059093A505A093A605B093A705BF9173
:104AB000AF919F918F913F912F910F900FBE0F90CB
:104AC0001F9018950F931F938FB7F8940091A0052E
:104AD0001091A1052091A2053091A3058FBFB801C7
:104AE000C9011F910F9108950F931F939FB7F894D9
:104AF0000091A4051091A5052091A6053091A70568
:104B000086B5A89B06C08F3F21F00F5F1F4F2F4F28
:104B10003F4F9FBF322F212F102F0027080F111D4D
:104B2000211D311D42E0000F111F221F331F4A9526
:104B3000D1F7B801C9011F910F910895CF92DF926B
:104B4000EF92FF92CF93DF936B017C010E9474255B
:104B5000EB010EC00E9474256C1B7D0B683E7340F8
:104B600038F081E0C81AD108E108F108C851DC4FDB
:104B7000C114D104E104F10469F7DF91CF91FF90F2
:104B8000EF90DF90CF900895789484B5826084BDD3
:104B900084B5816084BD85B5826085BD85B5816041
:104BA00085BDEEE6F0E0808181608083E1E8F0E0A1
:104BB0001082808182608083808181608083E0E8D0
:104BC000F0E0808181608083E1EBF0E080818460AF
:104BD0008083E0EBF0E0808181608083EAE7F0E0B1
:104BE0008081846080838081826080838081816015
:104BF00080838081806880831092C10008951F9314
:104C0000CF93DF93182FEB0161E00E948A26209753
:104C100011F460E004C0CF3FD10539F461E0812F89
:104C2000DF91CF911F910C94A626E12FF0E0E85080
:104C3000FF4EE491E330B9F028F4E13051F0E23076
:104C4000B1F50CC0E63019F1E73049F1E43079F5FF
:104C500014C084B5806884BDC7BD2EC084B5806291
:104C600084BDC8BD29C08091800080688093800089
:104C7000D0938900C09388001FC08091800080621B
:104C800080938000D0938B00C0938A0015C08091E0
:104C9000B00080688093B000C093B3000DC08091D5
:104CA000B00080628093B000C093B40005C0C038EB
:104CB000D1050CF0B3CFADCFDF91CF911F91089507
:104CC000833069F028F48130A1F0823011F514C0EE
:104CD0008630B1F08730C1F08430D9F404C08091BF
:104CE00080008F7703C0809180008F7D809380004B
:104CF000089584B58F7702C084B58F7D84BD0895F3
:104D00008091B0008F7703C08091B0008F7D809339
:104D1000B000089590E0FC01E85EFE4E2491FC0195
:104D2000E85CFE4EE491EE2381F0F0E0E35AFE4EA3
:104D3000A491B0E09FB7F8948C91611103C02095C5
:104D4000822301C0822B8C939FBF08950F931F93E2
:104D5000CF93DF931F92CDB7DEB7A82FB0E0FD0150
:104D6000E850FF4E8491FD01E85EFE4E1491FD0176
:104D7000E85CFE4E04910023B9F0882321F069839A
:104D80000E9460266981E02FF0E0E85AFE4EA4916F
:104D9000B0E09FB7F8948C91611103C01095812306
:104DA00001C0812B8C939FBF0F90DF91CF911F91FA
:104DB0000F9108951F920F920FB60F9211242F9307
:104DC0003F934F935F936F938F939F93EF93FF93D3
:104DD0006091C60020912A0630912B06C9010196E8
:104DE0008F77992740912C0650912D0684179507AF
:104DF00041F0F901E655FA4F608390932B068093BA
:104E00002A06FF91EF919F918F916F915F914F9142
:104E10003F912F910F900FBE0F901F9018959A0100
:104E2000AB01211581EE380741055105A9F42AC0CF
:104E30003093C5002093C4008091C10080618093AD
:104E4000C1008091C10088608093C1008091C10041
:104E500080688093C100089582E08093C00060E084
:104E600079E08DE390E00E946D6D21503109410998
:104E70005109CA01B90122E030E040E050E00E944F
:104E80006D6DD6CF1092C00020E130E0D1CF80917F
:104E90002C0690912D0620912A0630912B0628177A
:104EA000390769F0FC01E655FA4F208101968F77AA
:104EB000992790932D0680932C0630E002C02FEFA7
:104EC0003FEFC901089580912C0690912D06909393
:104ED0002B0680932A0608956F927F928F929F925D
:104EE000AF92BF92CF92DF92EF92FF920F931F93F8
:104EF000CF93DF93CDB7DEB7A0970FB6F894DEBFA0
:104F00000FBECDBF8C014115510561057105E1F45E
:104F100020E030E040E350E060E070E0A0960FB6A3
:104F2000F894DEBF0FBECDBFDF91CF911F910F91DF
:104F3000FF90EF90DF90CF90BF90AF909F908F90B9
:104F40007F906F900C94142866246394712C6C0EDF
:104F50007D1EC12CD12C7601822E912CA12CB12C3E
:104F6000CB01BA01A50194010E944B6DFA01D30156
:104F70006D933D01BFEFCB1ADB0AEB0AFB0AA901D7
:104F8000BF01411551056105710551F781E0C81A4E
:104F9000D108E108F1081AC0E1E0F0E0EC0FFD1FD4
:104FA000EC0DFD1D8081482F8A3010F4405D01C05A
:104FB000495C50E060E070E020E030E0C8010E9411
:104FC0001428A1E0CA1AD108E108F108BFEFCB16F6
:104FD000DB06EB06FB0601F7A0960FB6F894DEBFE2
:104FE0000FBECDBFDF91CF911F910F91FF90EF903A
:104FF000DF90CF90BF90AF909F908F907F906F90F9
:1050000008952115310539F48091C00085FFFCCF4A
:105010004093C60008950C946C279A01462F50E0E7
:1050200060E070E00C9401282115310539F480917D
:10503000C00085FFFCCF4093C60008952A3031059B
:1050400011F40C9451280C946C279A01AB0166273B
:1050500057FD6095762F0C941428CF93DF93EC01C5
:1050600020E030E04DE050E060E070E00E94142865
:1050700020E030E04AE050E060E070E0CE01DF91F7
:10508000CF910C941428CF93DF93EC019A01AB01DC
:1050900060E070E00E940128CE01DF91CF910C9476
:1050A0002D28CF92DF92EF92FF92CF93DF93EC0106
:1050B0006A017B0177FF10C020E030E04DE250E054
:1050C00060E070E00E941428F094E094D094C094C2
:1050D000C11CD11CE11CF11C2AE0B701A601CE01C4
:1050E000DF91CF91FF90EF90DF90CF900C946C27E1
:1050F0008F929F92AF92BF92CF92DF92EF92FF92E8
:105100000F931F93CF93DF938C014A015B01C22F52
:1051100020E030E0A901C501B4010E94796987FF50
:105120000DC020E030E04DE250E060E070E0C801EA
:105130000E941428B7FAB094B7F8B094D0E060E0B9
:1051400070E080E09FE307C020E030E040E251E4FF
:105150000E948069DF5FDC13F7CF262F372F482F9F
:10516000592FC501B4010E94A068D62EE72EF82E53
:10517000D92F0E94ED69962EA72EB82EC92E0E9417
:10518000196A9B01AC016D2D7E2D8F2D9D2F0E94E4
:105190009F68D62FF72EE82ED92E2AE0492D5A2DBA
:1051A0006B2D7C2DC8010E946C27CC23C1F1E6E653
:1051B000F2E006C09091C00095FFFCCF8093C6003E
:1051C00081918111F7CF2BC020E030E040E251E423
:1051D0006D2F7F2D8E2D9D2D0E944E6C4B015C01FD
:1051E000792D9B2D0E94E8696B01EE24D7FCE09499
:1051F000FE2CB701A601C8010E945128C701B601C3
:105200000E941B6A9B01AC01682D792D8A2D9B2D74
:105210000E949F68D62FF72EE82ED92EC150C111BB
:10522000D3CFDF91CF911F910F91FF90EF90DF903F
:10523000CF90BF90AF909F908F9008950C94782856
:10524000CF93DF93EC019C012C5F3F4F41E050E096
:1052500060E070E0898D9A8D0E94E9338823A1F087
:105260004D895E896F89788D452B462B472B71F4CC
:105270004C815D816E817F814D8B5E8B6F8B788FD2
:1052800089818068898302C080E001C081E0DF916C
:10529000CF910895CF92DF92EF92FF921F93CF9319
:1052A000DF93EC0149895A896B897C89403E5F4FC5
:1052B0006F41710508F06DC00E942029882309F410
:1052C00068C00E94F431882309F463C0E98DFA8D27
:1052D000CC80DD80EE80FF8032E0C31AD108E10887
:1052E000F108058404C0CC0CDD1CEE1CFF1C0A94E4
:1052F000D2F74685578560897189C40ED51EE61E92
:10530000F71E81E080933406C0923708D0923808A7
:10531000E0923908F0923A0880E092E0E7E3F6E0A4
:10532000DF019C011D9221503040E1F711E011C0D6
:10533000B701A601410F511D611D711D27E336E024
:1053400080913506909136060E945568882309F1B0
:105350001F5FE98DFA8D8481181750F3C12C82E00C
:10536000D82EE12CF12C058404C0CC0CDD1CEE1CE5
:10537000FF1C0A94D2F749895A896B897C894C0DA4
:105380005D1D6E1D7F1D498B5A8B6B8B7C8B81E065
:1053900001C080E0DF91CF911F91FF90EF90DF90EF
:1053A000CF900895CF93DF93EC0141E0611101C0EC
:1053B00040E06C857D858E859F850E942F328823F5
:1053C00041F0288980E2289F90011124295C394FFF
:1053D00002C020E030E0C901DF91CF910895CF9362
:1053E000FB0120E030E231932F5F2B30E1F7DC014D
:1053F00030E0C7E01CC0CA3051F138E0CAE017C045
:10540000E21729F1FC010196E491E111F9CFC317EC
:10541000F0F02132E0F02F37D0F4FB01E30FF11D63
:10542000822F81568A3108F4205220833F5FCD01BC
:105430002D91211109C0FA018083918381E0FB0144
:105440009081903259F403C02F3219F4F4CF80E0E8
:1054500005C02E3281F284EA94E0D4CFCF91089532
:105460000F931F93CF93DF93EC018B018B818823E4
:1054700011F080E044C0FB018789803131F528C0FC
:1054800083E08B83F801428D538D648D758D4D8B38
:105490005E8B6F8B788F9E012F5E3F4FC8010E94FD
:1054A000E932882331F31A8F098F81E089831C82C6
:1054B0001D821E821F82188619861A861B861C86EC
:1054C0001D861E861F86188A1AC0803291F6D8CF94
:1054D00082E08B831D8A1E8A1F8A188EFB01408DF5
:1054E000518D60E070E095E0440F551F661F771FF7
:1054F0009A95D1F7498B5A8B6B8B7C8BD4CFDF91EC
:10550000CF911F910F9108952F923F924F925F92EA
:105510006F927F928F929F92AF92BF92CF92DF92C3
:10552000EF92FF920F931F93CF93DF9300D000D0A1
:10553000CDB7DEB79C838B831A01DC0113968C9167
:10554000811103C02FEF3FEFEEC0EB81FC81818121
:1055500080FFF8CFBCC01601201A310A21015B017F
:105560008B819C8104969A838983ABC0AB81BC817B
:1055700018960D911D912D913C911B97D901C80151
:105580009170AA27BB273C01EB81FC814381680114
:10559000790159E0F694E794D794C7945A95D1F7D6
:1055A000818D928D423061F4DC015A966D917D912E
:1055B0008D919C915D976C0D7D1D8E1D9F1D4BC027
:1055C000FC0194809A949C206114710401F591105F
:1055D0001EC0012B022B032B59F4EB81FC81858922
:1055E0009689A789B08D84839583A683B7830FC0DE
:1055F000AB81BC8114964D915D916D917C91179713
:1056000029813A810E946832882309F49BCFAB81BB
:10561000BC815996ED91FC915A9714966D917D91AC
:105620008D919C91179762507109810991090584A8
:1056300004C0660F771F881F991F0A94D2F706854A
:10564000178520893189600F711F821F931F690D93
:10565000711D811D911D20E032E02619370972016C
:105660002415350508F47901E114B2E0FB0609F0D0
:1056700054C00091370810913808209139083091B2
:105680003A086017710782079307D9F546C0C3012E
:10569000895C994FA701BC01C5010E945270AE0CF4
:1056A000BF1CEB81FC8100851185228533850E0DA1
:1056B0001F1D211D311D00871187228733874E183A
:1056C0005F084114510409F051CF91012CC0EB81C6
:1056D000FC81C188D288E388F48800851185228501
:1056E00033852A01612C712C46015701801A910AD9
:1056F000A20AB30A481459046A047B0408F02BCFA9
:105700002DCF9501AB01BC018091350690913606F5
:105710000E9432678111C3CF15CF40E00E942F3223
:105720008111B5CF0FCFC9010F900F900F900F903F
:10573000DF91CF911F910F91FF90EF90DF90CF906D
:10574000BF90AF909F908F907F906F905F904F90A1
:105750003F902F900895CF93DF931F92CDB7DEB780
:1057600041E050E0BE016F5F7F4F0E94842A0197A5
:1057700019F4298130E002C02FEF3FEFC9010F90EB
:10578000DF91CF9108950F931F93CF93DF938C01F7
:10579000EB01FC018381823028F1408551856285CF
:1057A00073854F71552766277727452B462B472B47
:1057B000C9F440E250E0BE01C8010E94842A803250
:1057C000910521F0892B71F480E00DC08881882338
:1057D000D9F3853E71F38E3261F38B8583FDE9CF7A
:1057E00080E201C08FEFDF91CF911F910F9108955B
:1057F000CF92DF92EF92FF92CF93DF93EC018B81F8
:10580000823018F420E030E029C0C884D984EA84CA
:10581000FB8475E0F694E794D794C7947A95D1F712
:105820008FE0C822DD24EE24FF24CE010E94AB2BA2
:1058300097FDE8CF488559856A857B85415E5F4F36
:105840006F4F7F4F488759876A877B87960165E04E
:10585000220F331F6A95E1F7295C394FC901DF91A7
:10586000CF91FF90EF90DF90CF9008958F929F920D
:10587000AF92BF92CF92DF92EF92FF920F931F935E
:10588000CF93DF93EC014A015B012B81222309F4C2
:1058900075C089899A89AB89BC8984179507A60741
:1058A000B70708F46BC06CC081149104A104B10463
:1058B00049F41C821D821E821F82188619861A8650
:1058C0001B865AC0088519852A853B85E98DFA8D86
:1058D000858590E00996B901A801415051096109F7
:1058E0007109082E04C076956795579547950A94D7
:1058F000D2F7CC24CA94DC2C7601C80CD91CEA1C43
:10590000FB1C04C0F694E794D794C7948A95D2F709
:10591000C416D506E606F70620F0012B022B032B52
:1059200049F44D895E896F89788D4C835D836E83E0
:105930007F8316C0C41AD50AE60AF70A11C04C8143
:105940005D816E817F819801898D9A8D0E94683278
:1059500091E0C91AD108E108F108811104C014C00E
:105960008E010C5F1F4FC114D104E104F10439F71B
:1059700088869986AA86BB8681E006C080E004C03E
:10598000223009F091CFF4CFDF91CF911F910F9189
:10599000FF90EF90DF90CF90BF90AF909F908F904F
:1059A00008950F931F93CF93DF93EC018B8188238E
:1059B000E1F1898187FF33C061E0CE010E94D229E5
:1059C0008C01009791F1FC018081853E71F18B8102
:1059D000823040F449895A896B897C89448F558F7C
:1059E000668F778F4D895E896F89788DF801538F27
:1059F000428F758B648BE0912E06F0912F063097C5
:105A000059F0B8016A5E7F4FC80148960995F801C0
:105A1000808D918D938B828B89818F778983DF91A4
:105A2000CF911F910F910C94F43181E0888380E035
:105A3000DF91CF911F910F910895CF93DF93EC01E8
:105A40000E94D12C1B82DF91CF910895FC0123810C
:105A500021110C941D2D08956F927F928F929F9229
:105A6000AF92BF92CF92DF92EF92FF920F931F936C
:105A7000CF93DF9300D000D0CDB7DEB73C016A01F1
:105A80007B01FC018381813009F083C0818181FF2A
:105A900080C081C0452B462B472B09F478C0F30109
:105AA00080849184A284B384B701A601C3010E94BB
:105AB000362C811101C06DC0F301818D928DC1140E
:105AC000D104E104F10479F4458956896789708D20
:105AD0000E94FA34882309F45CC0F301158A168AFF
:105AE000178A108E3AC0F30144815581668177810F
:105AF0009E012F5F3F4F0E946832882309F449C0FE
:105B000049815A816B817C81F301818D928DFC01E9
:105B10002789203139F4483FFFEF5F0761057105A0
:105B2000E0F407C0483F2FEF520762072FE07207EB
:105B3000A0F40E94FA34882361F1F3014481558175
:105B4000668177810FEF1FEF2FEF3FE0818D928D00
:105B50000E945133811101C01CC0F301C18AD28A55
:105B6000E38AF48A818180688183C3010E94D12CF9
:105B7000882379F0B701A6018C149D04AE04BF04FC
:105B800010F4B501A401C3010E94362C10C081E0BD
:105B90000EC080E00CC0F301418952896389748989
:105BA0004C155D056E057F0508F074CFF2CF0F90A0
:105BB0000F900F900F90DF91CF911F910F91FF9059
:105BC000EF90DF90CF90BF90AF909F908F907F909D
:105BD0006F900895CF93DF93EC0140E050E0BA015D
:105BE0000E942C2D882371F061E0CE010E94D22901
:105BF000009741F025EEFC0120831B82DF91CF91BD
:105C00000C94F43180E0DF91CF910895FF920F93CF
:105C10001F93CF93DF93EC01F42E80E2689FF00195
:105C20001124E95CF94F8385817121F0842F827101
:105C300009F05CC0009137081091380820913908AC
:105C400030913A080C871D872E873F87688B4489DF
:105C5000558960E070E0BA0155274427028D138D05
:105C600020E030E0402B512B622B732B4D8B5E8B51
:105C70006F8B788F8385887151F4048D158D268DF7
:105C8000378D098B1A8B2B8B3C8B81E00CC08031BC
:105C900069F59E012F5E3F4F898D9A8D0E94E932F2
:105CA000882321F184E08B838F2D8F7089831C8260
:105CB0001D821E821F82188619861A861B86F4FE94
:105CC00018C040E050E0BA01CE010E942C2D811195
:105CD00010C012C049895A896B897C89CE01DF9135
:105CE000CF911F910F91FF900C94362C1B8280E076
:105CF00003C0F5FCEFCF81E0DF91CF911F910F91B1
:105D0000FF9008956F927F928F929F92AF92BF9271
:105D1000CF92DF92EF92FF920F931F93CF93DF9377
:105D20005C01EB014A01722E898D9A8DF501928FEB
:105D3000818F40E050E0BA01CE010E94362C612CE8
:105D400033C045E036952795179507954A95D1F7C5
:105D50000F70CE010E94F82BDC01009709F495C06A
:105D60008C91882311F0853EB1F4611010C0C09071
:105D70003708D0903808E0903908F0903A08F501DB
:105D8000C486D586E686F786008B662463948C915C
:105D900081110AC075C04BE050E0BD01C4010E94F2
:105DA0004570009709F46FC0088519852A853B85E1
:105DB000C988DA88EB88FC880C151D052E053F057F
:105DC00008F4BFCF5DC071FE60C0662051F0F501E0
:105DD000008961E0C5010E94D229EC01009771F4AD
:105DE00054C08B81823009F450C0CE010E944A29F0
:105DF000882309F44AC0C7E3D6E000E080E2FE0150
:105E000011928A95E9F78BE0F401DE0101900D9281
:105E10008A95E1F7E0912E06F0912F06309739F040
:105E2000BE01625F7F4FCE014096099508C081E2B6
:105E300098E2998B888B80E098E09F878E8788898D
:105E400099899B8B8A8B998F888F8E859F859F8B55
:105E50008E8B0E94F4318823C1F0472D602FC5013D
:105E6000DF91CF911F910F91FF90EF90DF90CF9036
:105E7000BF90AF909F908F907F906F900C94062E64
:105E800076FCA1CF02C077FEE8CF80E0DF91CF9112
:105E90001F910F91FF90EF90DF90CF90BF90AF9048
:105EA0009F908F907F906F9008955F926F927F92F6
:105EB0008F929F92AF92BF92CF92DF92EF92FF921A
:105EC0000F931F93CF93DF93CDB7DEB7C354D109A0
:105ED0000FB6F894DEBF0FBECDBF5C016B012496F8
:105EE0005FAF4EAF2497522E1C8E1F8E19821C82DC
:105EF0006115710511F410E075C0FC0183818111F9
:105F0000FACF2496EEADFFAD249780818F3239F021
:105F1000760117C031962496FFAFEEAF24972496F2
:105F2000EEADFFAD249780818F32A1F3F60183811E
:105F30008250823060F4ECCFEE24E394F12CEC0E2E
:105F4000FD1E8E01045E1F4F480138010CC0F60192
:105F5000618D728DCE0101960E94302A8111ECCFA5
:105F6000CACF78018301AE014E5B5F4FBE01695C11
:105F70007F4F24968EAD9FAD24970E94EF2981110B
:105F800006C0B9CF31962496FFAFEEAF2497249682
:105F9000EEADFFAD249780818F32A1F38823C9F045
:105FA00021E0AE01495C5F4FB701C8010E94822E1B
:105FB000882309F4A0CFEC14FD0419F0C7010E9456
:105FC0001D2D0815190569F68E010F5F1F4F73010E
:105FD000CACF252DAE01495C5F4FB701C5010E94B4
:105FE000822E182FCE0101960E94262DCE014C96AE
:105FF0000E94262D812FCD5BDF4F0FB6F894DEBFB8
:106000000FBECDBFDF91CF911F910F91FF90EF9009
:10601000DF90CF90BF90AF909F908F907F906F90C8
:106020005F9008951F93CF93DF93CDB7DEB76B9743
:106030000FB6F894DEBF0FBECDBFAB0119821C8234
:1060400022E0BC01CE0101960E94552F882331F039
:10605000CE0101960E94EA2D182F01C010E0CE015A
:1060600001960E94262D812F6B960FB6F894DEBF05
:106070000FBECDBFDF91CF911F9108952F923F9218
:106080004F925F927F928F929F92AF92BF92CF92E8
:10609000DF92EF92FF920F931F93CF93DF9300D085
:1060A00000D000D0CDB7DEB71C01162F072F5E83BE
:1060B0004D83DC0113968C911397813009F054C104
:1060C00011968C9181FF50C155C1F10141895289CE
:1060D0006389748980859185A285B3858417950726
:1060E000A607B70729F4AD80BE80812E902E07C188
:1060F000C1010E94362C8111F6CF36C1D1015996CB
:106100008D919C915A97FC0174807A94B701A601F5
:10611000E9E07695679557954795EA95D1F774220A
:10612000F1E0DF22EE24FF24260171104AC0C114E1
:10613000D10409F046C014964D915D916D917C910A
:106140001797411551056105710561F455960D913B
:106150001D912D913C91589701151105210531058F
:1061600049F522C09E012F5F3F4F0E94683288236D
:1061700009F4FAC009811A812B813C81D101599619
:10618000ED91FC915A978789803139F4083FBFEF30
:106190001B072105310540F40DC0083FEFEF1E0736
:1061A0002E07EFE03E0730F0C1010E942029811147
:1061B00008C0DAC0D10114960D931D932D933C9322
:1061C000179780E092E08419950985018A159B054F
:1061D00008F48C01D1015996ED91FC915A971496CF
:1061E000CD90DD90ED90FC901797B2E0CB1AD108DE
:1061F000E108F108058404C0CC0CDD1CEE1CFF1C7A
:106200000A94D2F786859785A089B189C80ED91ED0
:10621000EA1EFB1EC70CD11CE11CF11C0115E2E0BB
:106220001E0731F58091370890913808A091390800
:10623000B0913A088C159D05AE05BF0569F4109222
:1062400034068FEF9FEFDC01809337089093380876
:10625000A0933908B0933A089401B701A601809140
:106260003506909136060E945568811137C07CC072
:106270004114510419F5D10118964D915D916D911C
:106280007C911B9751968D919D910D90BC91A02D65
:10629000481759076A077B0788F00E94F431882362
:1062A00009F462C081E080933406C0923708D0922E
:1062B0003808E0923908F0923A0808C041E0C70176
:1062C000B6010E942F32882309F44EC09201295C46
:1062D000394FA801B401C9010E945270F101C08474
:1062E000D184E284F384C00ED11EE11CF11CC0866F
:1062F000D186E286F386800E911EA01AB10AF101C2
:10630000C084D184E284F384A114B10409F0F6CEF0
:1063100001891289238934890C151D052E053F0535
:1063200030F4D101C18AD28AE38AF48A0BC0809109
:106330002E0690912F06892B59F0ED81FE81EF2BCF
:1063400039F0D10111968C911197806811968C9338
:10635000F101818183FD03C02D813E810EC0C10109
:106360000E94D12C8111F8CF81E0D1018C932FEFC5
:106370003FEF03C082FDA9CEB6CEC90126960FB667
:10638000F894DEBF0FBECDBFDF91CF911F910F916B
:10639000FF90EF90DF90CF90BF90AF909F908F9045
:1063A0007F905F904F903F902F900895DB010D906C
:1063B0000020E9F7AD0141505109461B570B0296E9
:1063C0000C943E30CF93DF931F92CDB7DEB7698335
:1063D00041E050E0BE016F5F7F4F02960E943E3069
:1063E0000F90DF91CF910895809134068823A9F111
:1063F00040913708509138086091390870913A08F7
:1064000027E336E080913506909136060E94556864
:10641000811102C080E0089540913006509131060C
:106420006091320670913306411551056105710581
:1064300091F027E336E080913506909136060E9470
:106440005568882339F31092300610923106109265
:106450003206109233061092340681E00895CF92EE
:10646000DF92EF92FF92CF936B017C01C42F80915A
:10647000370890913808A0913908B0913A088C15E6
:106480009D05AE05BF05D1F00E94F431811102C017
:1064900080E018C027E336E0B701A60180913506F9
:1064A000909136060E943267882391F3C092370894
:1064B000D0923808E0923908F0923A0881E0C11190
:1064C00080933406CF91FF90EF90DF90CF900895A6
:1064D000AF92BF92CF92DF92EF92FF920F931F93F2
:1064E000CF93DF935C016A017B01E901FC014185E7
:1064F0005285638574854F5F5F4F6F4F7F4F4C159B
:106500005D056E057F0510F480E058C0FC018789A9
:10651000803129F499278F2D7E2D6D2D0CC080326E
:1065200099F7C701B60127E0969587957795679506
:106530002A95D1F7F5010389148925893689600FD9
:10654000711F821F931F0091370810913808209106
:10655000390830913A08601771078207930729F4C8
:10656000F50187898031A1F406C040E00E942F32F6
:106570008111F6CFC9CFDD24EE24FF24F601EE0F02
:10658000FF1FE95CF94F80819181A0E0B0E011C06C
:10659000E894C7F8DD24EE24FF24F601EE0FFF1F78
:1065A000EE0FFF1FE95CF94F80819181A281B381D9
:1065B000BF7088839983AA83BB8381E0DF91CF91E9
:1065C0001F910F91FF90EF90DF90CF90BF90AF9011
:1065D00008956F927F928F929F92AF92BF92CF92C7
:1065E000DF92EF92FF920F931F93CF93DF9300D030
:1065F00000D0CDB7DEB78C0149835A836B837C838F
:106600003901C12CD12C7601812C42E0942EA12C91
:10661000B12C49815A816B817C819E012F5F3F4F54
:10662000C8010E946832882341F1D501C401F801F4
:10663000058404C0880F991FAA1FBB1F0A94D2F7B4
:10664000C80ED91EEA1EFB1E49815A816B817C81CE
:106650008789803131F4483F5F4F6105710530F41F
:10666000D8CF483F5F4F6F4F7F4098F2F301C08211
:10667000D182E282F38281E001C080E00F900F902E
:106680000F900F90DF91CF911F910F91FF90EF909E
:10669000DF90CF90BF90AF909F908F907F906F9042
:1066A00008956F927F928F929F92AF92BF92CF92F6
:1066B000DF92EF92FF920F931F93CF93DF9300D05F
:1066C000CDB7DEB73C014A015B014230510561059F
:1066D000710508F46CC0F3014185528563857485AA
:1066E0004F5F5F4F6F4F7F4F481559056A057B0518
:1066F00008F45DC08789803129F4FF24EB2CDA2C63
:10670000C92C0DC0803209F052C07501640177E0D8
:10671000F694E794D794C7947A95D1F7F3018389D7
:106720009489A589B689C80ED91EEA1EFB1E41E0D0
:10673000C701B60129833A830E942F3229813A8109
:106740008823A9F1F3018789803159F49924AA2477
:10675000BB24F401EE0FFF1FE95CF94F11830083A6
:1067600010C0E89487F89924AA24BB24F401EE0F02
:10677000FF1FEE0FFF1FE95CF94F00831183228397
:106780003383F3018289823080F085819681A781ED
:10679000B0858C0D9D1DAE1DBF1D8093300690935E
:1067A0003106A0933206B093330681E001C080E049
:1067B0000F900F90DF91CF911F910F91FF90EF906D
:1067C000DF90CF90BF90AF909F908F907F906F9011
:1067D00008952F923F924F925F926F927F928F9285
:1067E0009F92AF92BF92CF92DF92EF92FF920F9360
:1067F0001F93CF93DF93CDB7DEB72F970FB6F894E3
:10680000DEBF0FBECDBF1C014C875D876E877F87C3
:106810003B872A87DC0119964D905D906D907C90A6
:106820001C97BFEF4B1A5B0A6B0A7B0AF901808049
:106830009180A280B38081149104A104B10431F04D
:10684000FFEF8F1A9F0AAF0ABF0A10C0DC018D90BC
:106850009D90AD90BC90B1E0BD832C853D854E856B
:106860005F85213031054105510509F01D82750113
:1068700064011E821F8218861986F1018185928526
:10688000A385B4852E813F8148855985281739070E
:106890004A075B0708F052C04C145D046E047F0485
:1068A00050F4B2E0CB2ED12CE12CF12C12E0812E51
:1068B000912CA12CB12C9E012F5F3F4FB701A60157
:1068C000C1010E9468328823C9F149815A816B81D4
:1068D0007C81D701C6010196A11DB11D452B462B18
:1068E000472B19F04C015D010DC088199909AA09BF
:1068F000BB092C853D854E855F8582179307A407CC
:10690000B50789F08E819F81A885B9850196A11D63
:10691000B11D8E839F83A887B9879FEFC91AD90AB3
:10692000E90AF90AAACF0FEF1FEF2FEF3FE0A60108
:10693000B701C1010E945133811115C080E041C0EF
:1069400044244A94542C32014C0C5D1C6E1C7F1C58
:1069500097018601B301A201C1010E94513388232E
:1069600069F3730162018C149D04AE04BF0440F30B
:10697000AA85BB854D915D916D917C914115510525
:106980006105710551F4EA85FB8580829182A282BE
:10699000B382FD81F11109C013C095018401C101C9
:1069A0000E9451338111EFCFC9CF2FEF821A920A83
:1069B000A20AB20AD1018D929D92AD92BC92139718
:1069C00081E02F960FB6F894DEBF0FBECDBFDF91EA
:1069D000CF911F910F91FF90EF90DF90CF90BF90DC
:1069E000AF909F908F907F906F905F904F903F906F
:1069F0002F900895AF92BF92CF92DF92EF92FF92C5
:106A00000F931F93CF93DF9300D000D0CDB7DEB7A5
:106A10005C016A017B0142E050E060E070E0FC0153
:106A200040835183628373839E012F5F3F4FB70181
:106A3000A601C5010E946832811102C080E023C016
:106A400000E010E09801B701A601C5010E94513392
:106A50008823A1F3C980DA80EB80FC80F501878967
:106A6000803141F4F8EFCF16FFEFDF06E104F104C7
:106A700048F4DACF88EFC8168FEFD806E8068FE023
:106A8000F80690F281E00F900F900F900F90DF9139
:106A9000CF911F910F91FF90EF90DF90CF90BF901B
:106AA000AF9008958F929F92AF92BF92CF92DF9254
:106AB000EF92FF920F931F93CF93DF93EC01142F6C
:106AC00070933606609335061F8A52E0C52ED12C8E
:106AD000E12CF12CC882D982EA82FB821092340622
:106AE0001092300610923106109232061092330640
:106AF000CC24CA94DC2C7601C0923708D092380896
:106B0000E0923908F0923A08442359F1453008F0F0
:106B1000DDC040E060E070E0CB010E942F328823AE
:106B200009F4D4C020E1129FF0011124EB51F84F79
:106B300080818F7709F0CAC0C484D584E684F78445
:106B400034E6C316D104E104F10408F4BFC0C084E4
:106B5000D184E284F384C114D104E104F10421F46A
:106B6000B5C0C12CD12C760140E0C701B6010E940E
:106B70002F32882309F4AAC08091420690914306DF
:106B80008115924009F0A2C020914706222309F402
:106B90009DC08091450690914606009709F496C0E5
:106BA00040914406442309F491C02A8B4C831D86EE
:106BB00050E061E070E006C02E2F2F5F2D87E83097
:106BC00008F084C0ED859B010E2E02C0220F331FFA
:106BD0000A94E2F74217530779F720914D06309156
:106BE0004E062115310519F040E050E008C0209113
:106BF0005B0630915C0640915D0650915E062D83E8
:106C00003E834F83588746015701880E991EA11C69
:106C1000B11C8B8A9C8AAD8ABE8A0091480610916D
:106C20004906198F088FA0914706B0E00E94146DA5
:106C3000680D791D8A1D9B1D6A8F7B8F8C8F9D8FA0
:106C4000980105E0220F331F0A95E1F721503E4FCE
:106C5000232F33272695DC01CB01820F931FA11D23
:106C6000B11D8E879F87A88BB98B80904A06909024
:106C70004B068114910419F0A12CB12C08C080900E
:106C8000570690905806A0905906B0905A06A70152
:106C90009601281B390B4A0B5B0BDA01C901880DE1
:106CA000991DAA1DBB1D04C0B695A79597958795FC
:106CB000EA95D2F789879A87AB87BC87853F3FE003
:106CC0009307A105B10520F48CE08F8B80E016C0FE
:106CD000853F9F4FA105B10510F480E10DC04091A3
:106CE00063065091640660916506709166064A8F4E
:106CF0005B8F6C8F7D8F80E28F8B81E0DF91CF91F6
:106D00001F910F91FF90EF90DF90CF90BF90AF90C9
:106D10009F908F9008952F923F924F925F926F9223
:106D20007F928F929F92AF92BF92CF92DF92EF921B
:106D3000FF920F931F93CF93DF93CDB7DEB7CA5463
:106D4000D1090FB6F894DEBF0FBECDBF1C017E8BFC
:106D50006D8B3A012BA30EA3E8A6AEAABFAAC8AEBC
:106D6000D9AE34E0239F80011124400F511F5BAB4B
:106D70004AABDA018D909D90AD90BC90FC01E00F84
:106D8000F11F2081318142815381C501B4010E94EC
:106D9000A0686AAF7BAF8CAF9DAFEEA1B4E0EB9F74
:106DA0007001112493012E0D3F1D3DAB2CABD90179
:106DB0004D905D906D907C90F101EE0DFF1D208156
:106DC000318142815381C301B2010E94A0686EAF3C
:106DD0007FAF21968FAF219722969FAF2297E8A58C
:106DE000B4E0EB9FC0011124F101E80FF91F2081ED
:106DF0003181428153812B8F3C8F4D8F5E8FED8986
:106E0000FE89E80FF91F60817181828193810E9460
:106E10009F68462F572F682F792F498B5A8B6B8B82
:106E20007C8BAD89BE891C968D919D910D90BC91F6
:106E3000A02D8AA79BA7ACA7BDA7D1011C962D9119
:106E40003D914D915C911F972F8F38A349A35AA371
:106E5000B7FAB094B7F8B09477FA709477F8709462
:106E6000ED89FE89E00FF11F7AAD6BAD9CAD8DAD64
:106E7000272F362F492F582F60817181828193816E
:106E80000E949F686F8B788F898F9DA3ED89FE8903
:106E9000EE0DFF1D7EAD6FAD21969FAD2197229621
:106EA0008FAD2297272F362F492F582F6081718160
:106EB000828193810E949F68162F072F382E292EDA
:106EC0007F89688D998D8DA1272F362F492F582FB7
:106ED000C501B4010E944E6C6B017C01B801C10177
:106EE000272F362F492F582FC301B2010E944E6C15
:106EF0009B01AC01C701B6010E94A0686B017C0137
:106F0000B801C101272F362F492F582FC501B401D1
:106F10000E944E6C6EA77FA788AB99AB7F89688D66
:106F2000998D8DA1272F362F492F582FC301B201DC
:106F30000E944E6C9B01AC016EA57FA588A999A902
:106F40000E949F68A70196010E941369362E272E82
:106F5000182F092F20E030E0A901D101F8016B2F93
:106F60007A2F8F2F9E2F0E94796987FF10C02BEDFB
:106F70003FE049EC50E4D101F8016B2F7A2F8F2FBD
:106F80009E2F0E94A068362E272E182F092FA49618
:106F90008FADA497882381F02BED3FE049EC50E4BE
:106FA000D101F8016B2F722D8F2F902F0E949F68B7
:106FB000362E272E182F092FC988DA88EB88FC88EF
:106FC000E894F7F8A3962CAD3DAD4EAD5FADA39719
:106FD000D101F8016B2F722D8F2F902F0E944E6CD4
:106FE000A70196010E94896B6B017C012FE632E1BB
:106FF00043E85AE30E94796987FD7BC2C701B60165
:107000000E94566A0E94ED697A8F698FFB01EF2B0F
:1070100021F421E030E03A8F298F498D5A8DBA0151
:1070200080E090E00E94196A6B017C019B01AC0139
:10703000D101F8016B2F722D8F2F902F0E94806944
:107040006F8B788F1C01A701960169897A898B89DA
:107050009C890E94806924966FAF249725967FAF04
:10706000259726968FAF269727969FAF27972F8D28
:1070700038A149A15AA16AA57BA58CA59DA50E940E
:107080009F68A70196010E94806928966FAF289794
:1070900029967FAF29972A968FAF2A972B969FAF75
:1070A0002B9720E030E040E05FE3BF89A88D6B2F95
:1070B0007A2F822D932D0E944E6CBF89A88D2B2F85
:1070C0003A2F422D532D0E944E6C9B01AC0160E083
:1070D00070E080E89FE30E949F686DA37AA78EA767
:1070E00023969FAF2397CE010196FC01A8A554E0FB
:1070F000A59FE00DF11D11242B8D3C8D4D8D5E8DD6
:1071000020833183428353832F8D38A149A15AA113
:107110002D873E874F87588B198A41E050E05C8F5E
:107120004B8F81E090E08C0F9D1FBBA1A4E0BA9F24
:10713000800D911D112499A788A721E030E02C0F24
:107140003D1F5EA144E0549F200D311D11243FA33B
:107150002EA3FCA3EBA3ACC1898989310CF050C0EC
:107160007F89688D272F362F422D532DC501B401FD
:107170000E944E6C6B017C017DA16AA59EA52396A1
:107180008FAD2397272F362F492F582FC301B201D8
:107190000E944E6C9B01AC01C701B6010E94A06821
:1071A0007B018C017DA16AA59EA523968FAD2397B7
:1071B000272F362F492F582FC501B4010E944E6C3E
:1071C0005B016C017F89688D272F362F422D532D4F
:1071D000C301B2010E944E6C9B01AC016A2D7B2D54
:1071E0008C2D9D2D0E949F68862E972EA82EB92E3D
:1071F00099899F5F998B4E2C5F2C602E712E72C0E7
:10720000AB8DBC8DBD0180E090E00E94196ABF8902
:10721000A88D2B2F3A2F422D532D0E944E6C7B01AF
:107220008C017F2D802F912F0E947D692B013C01C5
:107230006E2D7F2D802F912F0E94B16C698B7A8BE0
:107240008B8B9C8BEAA9FBA980819181A281B38160
:107250009C01AD0150582F8F38A349A35AA3ACA964
:10726000BDA9CD90DD90ED90FC90A30192016F8DB2
:1072700078A189A19AA10E944E6C4B015C012989D9
:107280003A894B895C89C701B6010E944E6C9B010B
:10729000AC01C501B4010E94A068862E972EA82ECD
:1072A000B92E29893A894B895C896F8D78A189A18A
:1072B0009AA10E944E6C698B7A8B8B8B9C8BA3015D
:1072C0009201C701B6010E944E6C9B01AC01698915
:1072D0007A898B899C890E949F68462E572E682E3A
:1072E000792E198AA5019401BAADABADFCADEDAD17
:1072F0006B2F7A2F8F2F9E2F0E94A068E8A5F9A5EB
:107300006083718382839383A3019201BEADAFAD8D
:107310002196FFAD21972296EFAD22976B2F7A2F02
:107320008F2F9E2F0E94A068AEA1BFA16D937D9369
:107330008D939C93139724967FAD249725966FADDC
:10734000259726969FAD269727968FAD2797272FAF
:10735000362F492F582FEBA1FCA1608171818281CA
:1073600093810E94A068ABA1BCA16D937D938D9386
:107370009C93139728967FAD289729966FAD2997F0
:107380002A969FAD2A972B968FAD2B97272F362FB6
:10739000492F582F6D857E858F8598890E94A0681A
:1073A0006D877E878F87988B20E030E0A901698107
:1073B0007A818B819C810E94796987FF04C0198240
:1073C0001A821B821C8220E030E0A9016D817E813F
:1073D0008F8198850E94796987FF04C01D821E8273
:1073E0001F82188620E030E0A90169857A858B85A7
:1073F0009C850E94796987FF04C019861A861B86BE
:107400001C8620E030E04BE153E469817A818B8176
:107410009C810E947C6B181644F480E090E0ABE104
:10742000B3E489839A83AB83BC8320E030E046E1F8
:1074300053E46D817E818F8198850E947C6B181644
:1074400044F480E090E0A6E1B3E48D839E83AF83B3
:10745000B88720E030E044EB52E469857A858B857B
:107460009C850E947C6B181644F480E090E0A4EBAD
:10747000B2E489879A87AB87BC8794E6C92ED12C62
:10748000CC0EDD1EEEA8FFA808AD19AD9E01235F4E
:107490003F4FAE01475F5F4FBE016B5F7F4FCE0135
:1074A00001960E943240EB8DFC8D3196FC8FEB8F64
:1074B0002B8D3C8D498D5A8D2417350708F44CCE01
:1074C0002D893E89245F3F4F4D895E89485F5F4F1C
:1074D0006D897E896C5F7F4F84E6C82ED12CCC0EDF
:1074E000DD1EEEA8FFA808AD19AD8D899E890E940A
:1074F0003240C65BDF4F0FB6F894DEBF0FBECDBF84
:10750000DF91CF911F910F91FF90EF90DF90CF907F
:10751000BF90AF909F908F907F906F905F904F90B3
:107520003F902F9008952F923F924F925F926F92CB
:107530007F928F929F92AF92BF92CF92DF92EF9203
:10754000FF920F931F93CF93DF93CDB7DEB768976A
:107550000FB6F894DEBF0FBECDBF1C014A015B0120
:1075600068017901DC01D8966D917D918D919C9196
:10757000DB970E94196A69837A838B839C83A501B8
:1075800094010E944E6C0E9466690E94ED696D83B1
:107590007E838F839887A701960169817A818B8189
:1075A0009C810E944E6C0E9466690E94ED69698709
:1075B0007A878B879C872D813E814F81588528371C
:1075C00031054105510540F488E790E0A0E0B0E0C6
:1075D0008D839E83AF83B88729853A854B855C85EB
:1075E000283731054105510540F488E790E0A0E0D7
:1075F000B0E089879A87AB87BC87F101EC5BFF4FCE
:107600004080518062807380C301B2010E941B6A76
:107610006B017C01D101DC966D917D918D919C91E6
:10762000DF970E94196A6D877E878F87988B20E08D
:1076300030E0A901C701B6010E947969882339F1B8
:1076400029813A814B815C81CA01B9010E944E6C4B
:107650004B015C012D853E854F855889CA01B901D2
:107660000E944E6C9B01AC01C501B4010E949F6851
:107670004B015C01A7019601C701B6010E94A068F9
:107680009B01AC01C501B4010E94806904C060E0A7
:1076900070E080E090E00E9466690E94E8694B011A
:1076A0005C0166277727CB0164197509860997095C
:1076B0000E941B6A2B013C01F101E05CFF4F6081DD
:1076C0007181828193810E94196A698B7A8B8B8B7D
:1076D0009C8B20E030E0A901C301B2010E947969CE
:1076E000882379F129893A894B895C89CA01B901D2
:1076F0000E944E6C6D8B7E8B8F8B988F29813A8187
:107700004B815C81CA01B9010E944E6C9B01AC01A6
:107710006D897E898F89988D0E949F6869837A839D
:107720008B839C83A3019201C301B2010E94A068D4
:107730009B01AC0169817A818B819C810E94806967
:1077400004C060E070E080E090E00E94566AD101E1
:1077500050962D913D914D915C91539729833A8399
:107760004B835C8329013A01481859086A087B0851
:107770000E94E869461A570A680A790A77FE6CC0BF
:1077800020E030E0A901C701B6010E947969882391
:1077900009F445C0A7019601C701B6010E94A0687F
:1077A0002B013C0169817A818B819C810E94196A3D
:1077B0009B01AC01C301B2010E944E6C2B013C0144
:1077C0002D853E854F855889CA01B9010E944E6CAE
:1077D0009B01AC01C301B2010E949F682B013C01D7
:1077E00029893A894B895C89CA01B9010E944E6C8A
:1077F0009B01AC01C301B2010E94A0684B015C0176
:1078000020E030E040E850E4C701B6010E944E6C31
:107810009B01AC01C501B4010E94806904C060E015
:1078200070E080E090E00E9466690E94E8694B0188
:107830005C01B7FE03C0812C912C540129813A814F
:107840004B815C8182169306A406B50610F04901AF
:107850005A01412C512C32018FB7F894F101E45BAD
:10786000FF4F9081911125C0D10154968D929D9228
:10787000AD92BC925797480C591C6A1C7B1CF101B5
:10788000408E518E628E738E2D813E814F81588540
:10789000DC962D933D934D935C93DF97A05CBF4F97
:1078A00029853A854B855C852D933D934D935C935B
:1078B00013978FBF68960FB6F894DEBF0FBECDBF8B
:1078C000DF91CF911F910F91FF90EF90DF90CF90BC
:1078D000BF90AF909F908F907F906F905F904F90F0
:1078E0003F902F900895AF92BF92CF92DF92EF9288
:1078F000FF920F931F93CF93DF935B017A01611582
:10790000710509F475C04115510509F471C0FB01F9
:1079100002A513A5D4A5C5A5CE01202F312F492F2F
:10792000582F66A177A180A591A50E947969882327
:1079300009F45EC0F50187A981114BC0F701C6A00B
:10794000D7A0E0A4F1A4A7019601DE01602F712F5A
:107950008B2F9A2F0E947C6B1816DCF5A7019601DD
:10796000C701B6010E944E6C6B017C01F50182A932
:1079700093A9A4A9B5A9BC01CD0190589B01AC0164
:107980000E94A068F50126A537A540A951A90E942B
:107990004E6C9B01AC01C701B6010E949F680E941A
:1079A000BB6C6B017C01762F272F3D2D4E2D5F2D5B
:1079B000FE01602F712F8F2F9E2F0E94796987FF04
:1079C00003C06801ED2EFC2E5C2D4D2D3E2D2F2D7C
:1079D00003C0502F412F9E01852F942FA32FB22F2C
:1079E000F50186A397A3A0A7B1A781E0F50186AB17
:1079F000DF91CF911F910F91FF90EF90DF90CF908B
:107A0000BF90AF900895CF92DF92EF92FF920F93C5
:107A10001F93CF93DF931F92CDB7DEB780913D08C0
:107A20008FB7F894F0903C088FBF80913D0890E0AC
:107A30008F1991098F709927049704F120913D08BF
:107A400023502F7040E050E000E010E08DE4E82E7D
:107A500013C0211101C020E12150E29E60011124D8
:107A60008EE398E0C80ED91EB801C60129830E9492
:107A7000733CA801860129812F11EBCF0F90DF9174
:107A8000CF911F910F91FF90EF90DF90CF900895CD
:107A90002F923F924F925F926F927F928F929F921E
:107AA000AF92BF92CF92DF92EF92FF920F931F930C
:107AB000CF93DF93EC011B01009709F464C08FA9F9
:107AC000811161C08EA09FA0A8A4B9A4FB01C6A08B
:107AD000D7A0E0A4F1A42C2D3D2D4E2D5F2DC50186
:107AE000B4010E94796987FF4EC0A5019401C501C8
:107AF000B4010E944E6C2B013C018AA89BA8ACA843
:107B0000BDA8C501B40190589B01AC010E94A068BA
:107B10002EA53FA548A959A90E944E6C9B01AC0116
:107B2000C301B2010E949F680E94BB6C8B01D82FD9
:107B3000C92F762FCE01272F312F492F582F6C2D8B
:107B40007D2D8E2D9F2D0E94796987FF03C08601B0
:107B5000DE2DCF2DCE01202F312F492F5C2F6C2D04
:107B60007D2D8E2D9F2D0E947969882361F09E01C5
:107B7000802F912FA32FBC2FF10186A397A3A0A73D
:107B8000B1A781E086ABDF91CF911F910F91FF905C
:107B9000EF90DF90CF90BF90AF909F908F907F90AD
:107BA0006F905F904F903F902F900895EF92FF92CB
:107BB0000F931F93CF93DF93F0903C08C0E0D0E089
:107BC00080E090E02DE4E22E11C0EF9C80011124B2
:107BD000025C174FA801BE010E94483D8F2D8F5FA8
:107BE000803109F480E0F82ECE01E80120913D08B3
:107BF000F212EBCF40E050E0BE01DF91CF911F9138
:107C00000F91FF90EF900C94483D4F925F926F92CE
:107C10007F928F929F92AF92BF92CF92DF92EF921C
:107C2000FF920F931F93CF93DF9350903C08C0E0D7
:107C3000D0E03DE4432E37C0489E3001499E700C91
:107C400011248EE398E0680E791E209731F18EA9F9
:107C5000811104C0F30186A98823F9F0CAA0DBA032
:107C6000ECA0FDA0A7019601F30166A177A180A574
:107C700091A50E9480694B015C01A70196016EA14C
:107C80007FA188A599A50E948069AB01BC019501DF
:107C90008401CE010E94933A1EAA5394F0E15F1230
:107CA00001C0512CE301852D992787FD90952091E6
:107CB0003D0830E08217930709F0BECF2097F1F01E
:107CC000CAA0DBA0ECA0FDA0A70196016DEC7CECA6
:107CD0008CE49DE30E9480694B015C01A701960141
:107CE0006EA17FA188A599A50E948069AB01BC0106
:107CF00095018401CE010E94933A1EAADF91CF9193
:107D00001F910F91FF90EF90DF90CF90BF90AF90B9
:107D10009F908F907F906F905F904F9008950E94FA
:107D2000033D0E94D63D0C94053E10923D081092F2
:107D30003C0880E1EFE0FDE0DF011D928A95E9F764
:107D400010927F0D1092800D1092810D1092820D75
:107D50001092830D1092840D1092850D1092860D55
:107D60001092870D1092880D1092890D10928A0D35
:107D700010928B0D10928C0D10928D0D10928E0D15
:107D800010928F0D1092900D1092910D1092920DF5
:107D900008954F925F926F927F928F929F92AF92CF
:107DA000BF92CF92DF92EF92FF920F931F93CF93E8
:107DB000DF9380910E0D882309F41FC160E080914C
:107DC000E80D9091E90D0E94285400912101109135
:107DD0002201D0912301C091240120E030E040E055
:107DE00050E40E94A068FE01202F312F4F2F5E2FFC
:107DF0000E94796987FD01C1F0903C08B12CC12C2B
:107E0000D12CE12C4DE4A42E5CC02F2D30E0A29E9D
:107E1000F001A39EF00D1124E25CF74F8081918167
:107E2000A281B381892B8A2B8B2B81F4848195814C
:107E3000A681B781892B8A2B8B2B41F48085918574
:107E4000A285B385892B8A2B8B2BC1F1A29E400181
:107E5000A39E900C11248EE398E0880E991EF401E5
:107E600064857585868597850E941B6A2B013C0178
:107E7000F40160897189828993890E94196A9B0142
:107E8000AC01C301B2010E948069F40122A133A1B7
:107E900044A155A10E944E6C3B014C012B2D3C2D61
:107EA0004D2D5E2D662D772D882D992D0E947C6B92
:107EB000181624F4B62CC72CD82CE92CF394FFE028
:107EC000FF2280913D08F812A0CF20911D01309132
:107ED0001E0140911F01509120016B2D7C2D8D2D95
:107EE0009E2D0E944E6C9B01AC01FE01602F712FF4
:107EF0008F2F9C2F0E94A0686B017C01CE01202F48
:107F0000312F492F5C2F6C2D7D2D8E2D9F2D0E94A2
:107F1000796987FD03C08601DE2DCF2DC090250134
:107F2000D0902601E0902701F09028012C2D3D2DC6
:107F30004E2D5F2DFE01602F712F8F2F9C2F0E94E1
:107F40007C6B18161CF06801ED2EFC2E8090930DB2
:107F50009090940DA090950DB090960D2C2D3D2DE8
:107F60004E2D5F2DC501B4010E947C6B1816F4F4F0
:107F700020E037ED43EA5CE36C2D7D2D8E2D9F2DA7
:107F80000E944E6C8B01D82FC92F28E431EE4AE7AE
:107F90005FE3C501B4010E944E6CFE01202F312F1A
:107FA0004F2F5E2F0E94A0686B017C018C2D9D2DB0
:107FB000AE2DBF2D8093930D9093940DA093950DAE
:107FC000B093960D6C2D7D2D8E2D9F2D0E94E8690E
:107FD000DC01CB0160E00E9458539093E90D80933F
:107FE000E80D8C2D9D2DAE2DBF2D8093DE0D909331
:107FF000DF0DA093E00DB093E10DDF91CF911F91C4
:108000000F91FF90EF90DF90CF90BF90AF909F9037
:108010008F907F906F905F904F90089590913C0863
:1080200080913D089817D9F020913C0830E04DE44C
:1080300010C0429FF0011124E25CF74F80859185CA
:10804000A285B385892B8A2B8B2B09F03F5F2F5F8D
:108050002F7080913D082813ECCF311101C0159A83
:108060000C94C93E2F923F924F925F926F927F92F3
:108070008F929F92AF92BF92CF92DF92EF92FF9238
:108080000F931F93CF93DF93CDB7DEB7C357D109BB
:108090000FB6F894DEBF0FBECDBF2C013B014A01E5
:1080A00059013E2CF9AA0AAB212EDDAACCAA2091B7
:1080B0003D082F5F63962FAF6397203119F46396C5
:1080C0001FAE639763963FAD6397032F112707FD9C
:1080D000109505C00E94F45481E00E94FC1280912A
:1080E0003C0890E080179107A9F320915B0D309137
:1080F0005C0D40915D0D50915E0DD2016D917D91B1
:108100008D919C910E944E6C0E941E6C23966FAFC5
:10811000239724967FAF249725968FAF2597269691
:108120009FAF269720915F0D3091600D4091610DBA
:108130005091620DF30160817181828193810E946F
:108140004E6C0E941E6C27966FAF279728967FAFC4
:10815000289729968FAF29972A969FAF2A97209123
:10816000630D3091640D4091650D5091660DD40101
:108170006D917D918D919C910E944E6C0E941E6C20
:108180002B966FAF2B972C967FAF2C972D968FAF9A
:108190002D972E969FAF2E972091670D3091680DE9
:1081A0004091690D50916A0DF50160817181828164
:1081B00093810E944E6C0E941E6C6AAF7BAF8CAFA5
:1081C0009DAF80911B0D90911C0DA0911D0DB09144
:1081D0001E0D2AAD3BAD4CAD5DAD281739074A07E2
:1081E0005B07C1F16091D002E62FF0E0EE0FFF1FB8
:1081F000EC51F24F808191810E94285420E030E0C0
:108200004AE253E40E94796987FF24C080913B08C9
:10821000811120C00C94974A9091C00095FFFCCF2B
:108220008093C600319684918111F6CFEAEBF4E099
:1082300007C09091C00095FFFCCF8093C600319697
:1082400084918111F6CF8091C00085FFFCCF8AE038
:108250008093C60080911B0D90911C0DA0911D0D67
:10826000B0911E0D2AAD3BAD4CAD5DAD281B390B59
:108270004A0B5B0BCA01B90157FF07C09095809567
:10828000709561957F4F8F4F9F4F0E941B6A4B01E6
:108290005C0120E030E848E953E46091670D70919B
:1082A000680D8091690D90916A0D0E944E6C9B0142
:1082B000AC01C501B4010E947C6B18166CF58AAD47
:1082C0009BADACADBDAD80931B0D90931C0DA093E9
:1082D0001D0DB0931E0DE4EBF4E007C09091C000BB
:1082E00095FFFCCF8093C600319684918111F6CF23
:1082F000E4EDF4E007C09091C00095FFFCCF8093BF
:10830000C600319684918111F6CF8091C00085FF1F
:10831000FCCF8AE08093C60080913D08EDE48E9FFB
:10832000D0011124A25CB74FBCA3ABA3FD01E45B59
:10833000FF4F108220910F0D3091100D4091110DC3
:108340005091120D2DA33EA34FA358A726964CACD7
:108350005DAC6EAC7FAC2697421A530A640A750A6C
:1083600077FE08C07094609450944094411C511C56
:10837000611C711CABA1BCA14D925D926D927C926F
:1083800013972091130D3091140D4091150D5091BC
:10839000160D29A73AA74BA75CA72A968CAC9DACD3
:1083A000AEACBFAC2A97821A930AA40AB50AB7FEEC
:1083B00008C0B094A09490948094811C911CA11C3E
:1083C000B11CABA1BCA114968D929D92AD92BC92B2
:1083D00017972091170D3091180D4091190D50915C
:1083E0001A0D2DA73EA74FA758AB2E964CAD5DADED
:1083F0006EAD7FAD2E978DA59EA5AFA5B8A9481BE4
:10840000590B6A0B7B0B77FF07C0709560955095F1
:1084100041955F4F6F4F7F4F142F052F6EAB78AF95
:10842000ABA1BCA118964C93189719965C93199719
:108430001A966C931A971B967C93C0901B0DD09044
:108440001C0DE0901D0DF0901E0DA0910001B0914B
:1084500001012AAD3BAD4CAD5DAD2C193D094E0976
:108460005F0957FF07C050954095309521953F4FC4
:108470004F4F5F4F0E941F6D24E630E040E050E018
:108480000E946D6DEBA1FCA1248735874687578735
:10849000812F902FAEA9B8AD88159905AA05BB0507
:1084A00014F4D501C40182179307A407B50714F487
:1084B000DA01C90193018201481659066A067B0652
:1084C00014F48C019D01ABA1BCA150960D931D939A
:1084D0002D933C935397063011052105310510F477
:1084E0000C94A74AFD01E85BFF4F8091CF0290E01A
:1084F000A0E0B0E080839183A283B38326962CAD65
:108500003DAD4EAD5FAD26978DA19EA1AFA1B8A5A3
:10851000281739074A075B072CF0ABA1BCA190963E
:108520001C9204C081E0EBA1FCA180A32A962CAD93
:108530003DAD4EAD5FAD2A9789A59AA5ABA5BCA56B
:10854000281739074A075B0744F4ABA1BCA19096F2
:108550008C919097826090968C932E962CAD3DAD29
:108560004EAD5FAD2E978DA59EA5AFA5B8A92817D6
:1085700039074A075B0744F4ABA1BCA190968C91E4
:108580009097846090968C932AAD3BAD4CAD5DADD9
:108590002C153D054E055F0544F4ABA1BCA190969A
:1085A0008C919097886090968C93ECA9FDA980811E
:1085B000ABA1BCA191968C9345284628472809F089
:1085C0005E98EBA1FCA184819581A681B781892B5E
:1085D0008A2B8B2B09F05E98EBA1FCA180859185FD
:1085E000A285B385892B8A2B8B2B09F01598EBA1DB
:1085F000FCA184859585A685B785892B8A2B8B2B35
:1086000009F05E98ABA1BCA11C962D913D914D91B6
:108610005C911F9722962CAF3DAF4EAF5FAF229774
:10862000232B242B252BD9F440902F0D5090300D67
:108630006090310D7090320D242D352D462D572D23
:10864000A9A9FAA9632D7A2F8F2F922D0E947969FB
:1086500087FD0EC0432C59A86AA8722C09C040900F
:10866000470D5090480D6090490D70904A0DE4CF31
:1086700026966CAD7DAD8EAD9FAD26972DA13EA10A
:108680004FA158A5621B730B840B950B0E941B6AAC
:1086900020915B0D30915C0D40915D0D50915E0D10
:1086A0000E9480696DA379AB8AAB9CAB362F272FD4
:1086B000982F8CA9432F522F692F782F498B5A8BD3
:1086C0006B8B7C8B2A966CAD7DAD8EAD9FAD2A9762
:1086D00029A53AA54BA55CA5621B730B840B950BD2
:1086E0000E941B6A20915F0D3091600D4091610DD9
:1086F0005091620D0E948069162F072F89A79EABAB
:108700009801982F8EA9432F522F692F782F4D8BC8
:108710005E8B6F8B788F2E966CAD7DAD8EAD9FADE1
:108720002E972DA53EA54FA558A9621B730B840B50
:10873000950B0E941B6A2091630D3091640D40914E
:10874000650D5091660D0E9480696DA778AF382E37
:10875000292E362F272FC101432F522F692F782F13
:10876000498F5A8F6B8F7C8FA0900001B0900101D0
:108770006AAD7BAD8CAD9DAD6C197D098E099F09ED
:108780000E941B6A2091670D3091680D4091690D20
:1087900050916A0D0E9480696B017C01B5018827A8
:1087A00077FD8095982F0E941B6A9B01AC01C70141
:1087B000B6010E944E6C20E030E048EC52E40E948A
:1087C0008069462F572F682F792FDB01CA014D8F03
:1087D0005E8F6F8F78A3EBA1FCA180809180A28037
:1087E000B380F6E08F169104A104B104E4F4EBA188
:1087F000FCA1448155816681778146305105610530
:1088000071058CF44085518562857385463051052C
:108810006105710544F4AC01BD017F7746A757A7F8
:1088200060AB71AB3AC05DA149A93AA92CA9652FEB
:10883000742F832F922F0E94F96C6B017C01A80189
:1088400039A52EA9652F702F832F922F0E94F96CC6
:108850009B01AC01C701B6010E94A068162F072F2B
:10886000F82EE92E5DA548AD9101652F742F832F59
:10887000922D0E94F96C9B01AC01D801F7016B2F7E
:108880007A2F8F2F9E2F0E94A0680E94BB6CEBA1B5
:10889000FCA166A777A780AB91ABABA1BCA19E96CC
:1088A0002D913D914D915C91D197AA962CAF3DAF02
:1088B0004EAF5FAFAA9760E070E080E89FE30E9450
:1088C00080699B01AC01642D752D862D972D0E942A
:1088D0004E6C69A77DA789AB9CAB90913D088091B8
:1088E0003C08E92FF0E0E81BF109EF70FF27FBAB34
:1088F000EAAB762F6DA599A98CA9272F362F492F82
:10890000582F60E074E284E799E40E9480690E9435
:108910001E6C1B018C012AA93BA9223031050CF4E5
:108920004AC06901EE24D7FCE094FE2CC701B601D1
:108930000E941B6A20E030E040E051E40E94796927
:1089400087FF39C02101380180917B0D90917C0D0A
:10895000A0917D0DB0917E0D481659066A067B06E2
:1089600050F5BC01CD016419750986099709660F98
:10897000771F881F991FA70196010E944B6DCA019E
:10898000B9010E94196A0E941E6CAB01BC01CB01A7
:10899000BA01640D751D861D971D0E94196A9B0101
:1089A000AC0160E074E284E799E40E94806969A701
:1089B0007DA789AB9CAB79A56DA599A98CA9272F1B
:1089C000362F492F582FAA966CAD7DAD8EAD9FAD39
:1089D000AA970E944E6C6E966FAF6E97A2967FAF6D
:1089E000A2972F968FAF2F97A6969FAFA697362F59
:1089F000272F982FA6968FADA697432F522F692F1A
:108A0000782FABA1BCA192964D935D936D937C930F
:108A1000959750966D917D918D919C9153970E9461
:108A2000196A6B017C0179A56DA599A98CA9272FDD
:108A3000362F492F582FC701B6010E944E6C0E9455
:108A400066690E94ED6967966CAF7DAF8EAF9FAF90
:108A50006797EBA1FCA160AF71AF82AF93AF9E01AE
:108A60002F5E3F4F3FAB2EABAE014F5F5F4F5EA31C
:108A70004DA38BE69DE06D969FAF8EAF6D97DE01A7
:108A80009196BAA3A9A359AF48AF212C312C00E885
:108A90001FE3EEA9FFA96191719181919191FFABC3
:108AA000EEABB9A5ADA5F9A9ECA92B2F3A2F4F2F05
:108AB0005E2F0E944E6CAB01BC01A8ADB9AD4D93C9
:108AC0005D936D937D93B9AFA8AFDB01CA01BF770A
:108AD0006B968CAF9DAFAEAFBFAF6B976D96AEADE3
:108AE000BFAD6D974D905D906D907D906D96BFAFD1
:108AF000AEAF6D97A30192016B966CAD7DAD8EAD5F
:108B00009FAD6B970E947C6B1816F4F46B962CAD9E
:108B10003DAD4EAD5FAD6B97C301B2010E94806960
:108B20002B01782E692E762FC301272F352D492F43
:108B3000582F622D732D802F912F0E94796987FD08
:108B400003C01201072D162DEEA9FFA929A13AA1F4
:108B5000E217F30709F09DCF20E030E040E85FE343
:108B6000622D732D802F912F0E94796987FF4FC04E
:108B70003E0131E1630E711C222D332D402F512F08
:108B8000ADA1BEA16D917D918D919C910E944E6C85
:108B9000EDA1FEA16193719381939193FEA3EDA347
:108BA000E615F70549F7222D332D402F512F6E96EC
:108BB000BFAD6E97A296AFADA2972F96FFAD2F9740
:108BC000A696EFADA6976B2F7A2F8F2F9E2F0E9420
:108BD0004E6CABA1BCA192966D937D938D939C93AB
:108BE000959767966CAD7DAD8EAD9FAD67970E94F2
:108BF000196A222D332D402F512F0E944E6C0E9456
:108C0000ED69EBA1FCA160AF71AF82AF93AFAA9603
:108C10002CAD3DAD4EAD5FADAA97C701B6010E9428
:108C20008069162F072F382E292E81149104A10454
:108C3000B10491F5EBA1FCA184819581A681B78156
:108C4000892B8A2B8B2B41F580859185A285B38555
:108C5000892B8A2B8B2B01F520913F0D3091400DF4
:108C60004091410D5091420DD801F1016B2F7A2FA7
:108C70008F2F9E2F0E944E6C0E946669EBA0FCA075
:108C8000F4E4EF0EF11C0E94ED69D7016D937D9322
:108C90008D939C93139700C12091430D3091440D07
:108CA0004091450D5091460DD801F1016B2F702F69
:108CB0008F2F922D0E944E6C0E9466690E94ED6972
:108CC000EBA1FCA1EC5BFF4FFEA3EDA360837183DE
:108CD0008283938340901F0D5090200D6090210D52
:108CE0007090220D0E94196A69A77AA78BA79CA78A
:108CF000C501B4010E941B6A9B01AC0169A57AA55C
:108D00008BA59CA50E944E6CA70196010E948069CC
:108D10004B015C01C301B2010E94196A9B01AC01C5
:108D2000C501B4010E947C6B181634F4EDA1FEA1BC
:108D300040825182628273824090230D5090240DB4
:108D40006090250D7090260DADA1BEA16D917D9115
:108D50008D919C910E94196A4B015C01EBA1FCA1D1
:108D600064817581868197810E941B6A9B01AC0199
:108D7000C501B4010E944E6CA70196010E94806952
:108D80004B015C01C301B2010E94196A9B01AC0155
:108D9000C501B4010E947C6B18163CF4ADA1BEA1C4
:108DA0004D925D926D927C92139740902B0D509056
:108DB0002C0D60902D0D70902E0DEBA1FCA1EC5BA5
:108DC000FF4FFEA3EDA360817181828193810E9498
:108DD000196A4B015C0122966CAD7DAD8EAD9FADE5
:108DE00022970E941B6A9B01AC01C501B4010E943D
:108DF0004E6CA70196010E9480694B015C01C30182
:108E0000B2010E94196A9B01AC01C501B4010E9424
:108E10007C6B18163CF4ADA1BEA14D925D926D9293
:108E20007C9213974090270D5090280D6090290D4B
:108E300070902A0DEDA1FEA16081718182819381E4
:108E40000E94196A4B015C01ABA1BCA118966D91FF
:108E50007D918D919C911B970E941B6A9B01AC0197
:108E6000C501B4010E944E6CA70196010E94806961
:108E70006B017C01C301B2010E94196A9B01AC0124
:108E8000C701B6010E947C6B181634F4EDA1FEA157
:108E90004082518262827382EBA1FCA1EC5BFF4FA6
:108EA00060817181828193810E94196A6B017C01CA
:108EB000B801C101272F302F492F522DC701B6010C
:108EC0000E948069462F572F682F792FE0964CAF6C
:108ED0005DAF6EAF7FAFE097ABA1BCA1D2964D93D3
:108EE0005D936D937C93D5972DEB37E346E051E48A
:108EF000C701B6010E944E6C0E94E869EBA1FCA17B
:108F0000648F758F868F978F40903B0D50903C0DEE
:108F100060903D0D70903E0D20E030E040E05FE35A
:108F2000C301B2010E944E6C6DA379A78DA799ABC6
:108F300029853A854B855C85A1962CAF3DAF4EAF18
:108F40005FAFA1978090370D9090380DA090390DAC
:108F5000B0903A0D20E030E040E05FE3C501B4019D
:108F60000E944E6C162F072FF82EE92EA1966CAD9D
:108F70007DAD8EAD9FADA1979F77D801F7012B2FC7
:108F80003A2F4F2F5E2F0E947C6B1816B4F4B80155
:108F9000C701272F362F492F582FBDA1A9A5FDA501
:108FA000E9A96B2F7A2F8F2F9E2F0E94796987FD59
:108FB00004C01DA309A7FDA6E9AA8D859E85AF85DE
:108FC000B889A5968CAF9DAFAEAFBFAFA597C09047
:108FD000330DD090340DE090350DF090360D20E03B
:108FE00030E040E05FE3C701B6010E944E6C162FEF
:108FF000072F382E292EA5966CAD7DAD8EAD9FAD79
:10900000A5979F77D801F1012B2F3A2F4F2F5E2F75
:109010000E947C6B1816B4F4B801C101272F362FBB
:10902000492F582FBDA1A9A5FDA5E9A96B2F7A2F1E
:109030008F2F9E2F0E94796987FD04C01DA309A769
:109040003DA629AAABA1BCA19296BC91BCABEBA159
:10905000FCA1F3A1FEABABA1BCA19496BC91B8AFAF
:10906000EBA1FCA1F5A1FEAF7CA96EA9272F362F9D
:109070004B2F5F2FBDA1A9A5FDA5E9A96B2F7A2FC5
:109080008F2F9E2F0E94796987FD08C02CA92DA3E0
:109090003EA939A748AD4DA75EAD59AB8AA99BA99A
:1090A00002970CF443C190918F0D9AABA091900D53
:1090B0006496AFAF6497B091910D6896BFAF689713
:1090C000E091920D6C96EFAF6C9727E137EB41ED95
:1090D00058E36896FFAD6897692F7A2F8F2F9E2FE0
:1090E0000E947C6B18160CF021C120917F0D3091ED
:1090F000800D4091810D5091820D69817A818B8123
:109100009C810E949F68162F072F382E292E2091B0
:10911000830D3091840D4091850D5091860D6D81A8
:109120007E818F8198850E949F682F966FAF2F97C1
:10913000A6967FAFA697AB968FAFAB97AC969FAF37
:10914000AC97B801C101272F362F492F582FD801CE
:10915000F1016B2F7A2F8F2F9E2F0E944E6CE49679
:109160006CAF7DAF8EAF9FAFE4972F967FAD2F97FB
:10917000A6966FADA697AB969FADAB97AC968FAD0D
:10918000AC97272F362F492F582FDB01FC016B2F6F
:109190007A2F8F2F9E2F0E944E6C9B01AC01E4967C
:1091A0006CAD7DAD8EAD9FADE4970E94A0680E942E
:1091B000BB6C62966CAF7DAF8EAF9FAF6297A30121
:1091C00092010E947C6B18166CF462962CAD3DAD3A
:1091D0004EAD5FAD6297C301B2010E9480698B0101
:1091E0001C0106C000E010E050E8252E6FE3362E8B
:1091F0002091870D3091880D4091890D50918A0DF5
:10920000A1966CAD7DAD8EAD9FADA1970E949F687C
:109210002B013C01E89477F8A5019401C301B20148
:109220000E947C6B1816D4F4A3019201C501B4010D
:109230000E9480694B01B82EA92E762FC501272FD9
:10924000392D492F582F602F712F822D932D0E9479
:10925000796987FD03C084012B2C3A2C20918B0D5A
:1092600030918C0D40918D0D50918E0DA5966CAD69
:109270007DAD8EAD9FADA5970E949F684B015C01AF
:10928000E894B7F8A7019601C501B4010E947C6B70
:109290001816D4F4A5019401C701B6010E94806993
:1092A0006B01F82EE92E762FC701272F3D2D492F70
:1092B000582F602F712F822D932D0E94796987FD81
:1092C00003C086012F2C3E2C202F312F422D532DF1
:1092D000BCA9AEA9F8ADEEAD6B2F7A2F8F2F9E2FC4
:1092E0000E944E6C4B015C01762F272F392D4A2DA1
:1092F0005B2DBAA96496AFAD64976896FFAD689789
:109300006C96EFAD6C976B2F7A2F8F2F9E2F0E944C
:10931000796987FF0FC08AA864969FAC64976896A6
:10932000AFAC68976C96BFAC6C9704C08DA099A445
:10933000ADA4B9A8482D592D6A2D7B2DABA1BCA198
:109340009A964D935D936D937C939D97E0966CAD4B
:109350007DAD8EAD9FADE09790589B01AC010E9412
:10936000A068AA962CAD3DAD4EAD5FADAA970E9408
:109370004E6C9B01AC016BE077ED83E29BE30E94B6
:109380009F680E94BB6C8B01F82EE92E762FC701D7
:10939000272F312F492F582F682D792D8A2D9B2D5E
:1093A0000E94796987FD03C04801AF2CBE2C482D6F
:1093B000592D6A2D7B2DEBA1FCA146A357A360A7D5
:1093C00071A7C701202F312F492F5E2DBCA9AEA94F
:1093D000F8ADEEAD6B2F7A2F8F2F9E2F0E947969FB
:1093E000181634F081E0ABA1BCA1D7968C9303C0D2
:1093F000EBA1FCA117AA81E0ABA1BCA1D6968C93EE
:1094000080E1FE013196AFE7BDE001900D928A95B3
:10941000E1F73CA92EA998AD8EAD432F522F692FAD
:10942000782F40938F0D5093900D6093910D709312
:10943000920D232F352F492F582FBDA1A9A5FDA58A
:10944000E9A96B2F7A2F8F2F9E2F0E9480696B01C5
:109450007C017CA96EA998AD8EAD272F362F492FA0
:10946000582F682D792D8A2D9B2D0E948069AB0184
:10947000BC01970186018BA19CA10E94933A63963F
:10948000BFAD6397B0933D0826962CAD3DAD4EAD74
:109490005FAD269720930F0D3093100D4093110D63
:1094A0005093120D2A968CAD9DADAEADBFAD2A97EF
:1094B0008093130D9093140DA093150DB093160D7A
:1094C0002E962CAD3DAD4EAD5FAD2E972093170D72
:1094D0003093180D4093190D50931A0D8AAD9BAD22
:1094E000ACADBDAD80931B0D90931C0DA0931D0DD5
:1094F000B0931E0D0E948F3ECD58DF4F0FB6F894EB
:10950000DEBF0FBECDBFDF91CF911F910F91FF90B6
:10951000EF90DF90CF90BF90AF909F908F907F9013
:109520006F905F904F903F902F900C94404C2AADDD
:109530003BAD4CAD5DAD20931B0D30931C0D4093A6
:109540001D0D50931E0DE4EBF4E00C941341CD5827
:10955000DF4F0FB6F894DEBF0FBECDBFDF91CF91C6
:109560001F910F91FF90EF90DF90CF90BF90AF9041
:109570009F908F907F906F905F904F903F902F9033
:109580000895EF92FF920F931F93CF93DF937B0188
:109590008A01E90120915B0D30915C0D40915D0DD8
:1095A00050915E0DFC0160817181828193810E94E6
:1095B0004E6C0E941E6CEFE0FDE06083718382833D
:1095C000938320915F0D3091600D4091610D50911A
:1095D000620DF70160817181828193810E944E6CDE
:1095E0000E941E6CE3E1FDE06083718382839383BC
:1095F0002091630D3091640D4091650D5091660D81
:10960000F80160817181828193810E944E6C0E9479
:109610001E6CE7E1FDE06083718382839383209178
:10962000670D3091680D4091690D50916A0D688108
:1096300079818A819B810E944E6C0E941E6CEBE1B5
:10964000FDE060837183828393839F0147E15DE046
:1096500063E17DE08FE09DE00E94B05210928F0D9B
:109660001092900D1092910D1092920D10927F0D0C
:109670001092800D1092810D1092820D1092830D28
:109680001092840D1092850D1092860D1092870D08
:109690001092880D1092890D10928A0D10928B0DE8
:1096A00010928C0D10928D0D10928E0DDF91CF9136
:1096B0001F910F91FF90EF9008952091670D3091C9
:1096C000680D4091690D50916A0DFC0160817181B6
:1096D000828193810E944E6C0E941E6CEBE1FDE042
:1096E0006083718382839383CF010C94EC528093C7
:1096F0003B0808958091A90D8111B5C08091A80DF6
:109700008111B1C08091A70D8111ADC008959091D4
:10971000C00095FFFCCF8093C600319684918111E3
:10972000F6CFE8EFF4E007C09091C00095FFFCCFC2
:109730008093C600319684918111F6CF8091A90D56
:10974000882349F1E7E0F5E007C09091C00095FF5C
:10975000FCCF8093C600319684918111F6CF609141
:10976000AA0D7091AB0D8091AC0D9091AD0D0E9442
:109770001B6A20915B0D30915C0D40915D0D509105
:109780005E0D0E948069AB01BC0122E030E089EAF5
:1097900095E00E941E298091A80D882349F1EBE0F5
:1097A000F5E007C09091C00095FFFCCF8093C60004
:1097B000319684918111F6CF6091AE0D7091AF0D0D
:1097C0008091B00D9091B10D0E941B6A20915F0DA8
:1097D0003091600D4091610D5091620D0E94806941
:1097E000AB01BC0122E030E089EA95E00E941E292D
:1097F0008091A70D882349F1EFE0F5E007C0909133
:10980000C00095FFFCCF8093C600319684918111F2
:10981000F6CF6091B20D7091B30D8091B40D90911F
:10982000B50D0E941B6A2091630D3091640D40912B
:10983000650D5091660D0E948069AB01BC0122E06C
:1098400030E089EA95E00E941E298091C00085FFE2
:10985000FCCF8AE08093C6001092A90D1092A80D4B
:109860001092A70D0895E2EFF4E058CF1092A90DE1
:109870001092A80D1092A70D089580932D010895C0
:10988000EFE6F0E080818260808308951F920F925E
:109890000FB60F9211240F931F932F933F934F9363
:1098A0005F936F937F938F939F93AF93BF93EF9348
:1098B000FF938091BA0D9091BB0D892B09F07DC16A
:1098C00090913D0880913C08981771F0E0913C0818
:1098D0008DE4E89FF0011124E25CF74FDF01A45B07
:1098E000BF4F81E08C9302C0E0E0F0E0F093BB0D4D
:1098F000E093BA0D309709F45AC1DF01A45BBF4F62
:1099000081E08C931092BC0D1092BD0D1092BE0D93
:109910001092BF0D60AD71AD61349CE9790728F4F8
:1099200061329EE4790748F002C060E47CE97695F4
:1099300067957695679584E007C0613197E279076E
:1099400030F07695679582E08093C00D07C08093D4
:10995000C00D6032710510F460E270E06052710970
:10996000611588E07807D0F0872F9927880F991F15
:10997000880F991F8D5E9A4FFC0132964591549144
:10998000AA27659F9001649F210D3A1F06942A1F04
:109990003A1F1124FC01859194911DC09B013695BD
:1099A00027952C7F2D5E364FF901859194912E5F7E
:1099B0003F4FF90145915491FB01E770FF274E9FFE
:1099C00090014F9F300D5E9F300D112413E03695AE
:1099D00027951A95E1F7821B930B84369105A0F425
:1099E000E2E7F2E006C09091C00095FFFCCF8093C3
:1099F000C60081918111F7CF4AE050E089EA95E0F5
:109A00000E94432884E690E09093C20D8093C10D9C
:109A1000E091BA0DF091BB0D64AD75AD7093C40DBE
:109A20006093C30D61349CE9790728F461328EE4B8
:109A3000780748F002C060E47CE9769567957695F2
:109A4000679584E007C0613197E2790730F0769539
:109A5000679582E08093C00D08C081E08093C00DBF
:109A60006032710510F460E270E0605271096115B6
:109A700088E07807E0F0872F9927880F991F880FD3
:109A8000991F8D5E9A4FFC01329625913491AA2739
:109A9000639FA001629F410D5A1F06944A1F5A1FDF
:109AA0001124FC0125913491241B350B1EC0CB01E0
:109AB000969587958C7F8D5E964FFC01259134910C
:109AC0000296FC0145915491FB01E770FF274E9FE0
:109AD000C0014F9F900D5E9F900D112443E096951D
:109AE00087954A95E1F7281B390B24363105A0F4F8
:109AF000E2E7F2E006C09091C00095FFFCCF8093B2
:109B0000C60081918111F7CF4AE050E089EA95E0E3
:109B10000E94432824E630E0C901A0E0B0E0809331
:109B2000C50D9093C60DA093C70DB093C80D30938B
:109B3000890020938800E091BA0DF091BB0D8089D7
:109B40009189A289B389B695A79597958795B09580
:109B5000A095909581959F4FAF4FBF4F8093C90DB2
:109B60009093CA0DA093CB0DB093CC0D8093CD0DE7
:109B70009093CE0DA093CF0DB093D00D8093D10DC7
:109B80009093D20DA093D30DB093D40D8093D50DA7
:109B90009093D60DA093D70DB093D80D1092B60D1B
:109BA0001092B70D1092B80D1092B90D06C080ED4D
:109BB00097E09093890080938800E091BA0DF0912E
:109BC000BB0D309709F460C480A18093D90D80FF4C
:109BD00038C0459A8FEF8093290180912D01882309
:109BE000A1F1329942C480E029C080819181A28193
:109BF000B381181619061A061B06FCF48091970DFE
:109C00009091980DA091990DB0919A0D8093AA0D05
:109C10009093AB0DA093AC0DB093AD0D81E080930C
:109C2000A90D80899189A289B3898093B60D9093FB
:109C3000B70DA093B80DB093B90D81E08093DA0D04
:109C400004C0459881E0809329018091D90D81FF5E
:109C50003CC047988FEF80932A0180912D01882383
:109C6000C1F1339907C480E02DC0E091BA0DF091A5
:109C7000BB0D84819581A681B781181619061A0635
:109C80001B06FCF480919B0D90919C0DA0919D0D65
:109C9000B0919E0D8093AE0D9093AF0DA093B00D3B
:109CA000B093B10D81E08093A80D80899189A2893C
:109CB000B3898093B60D9093B70DA093B80DB09370
:109CC000B90D81E08093DB0D04C0479A81E0809359
:109CD0002A018091D90D82FF3CC02A988FEF809392
:109CE0002B0180912D018823C1F13499C8C380E0F4
:109CF0002DC0E091BA0DF091BB0D80859185A285B4
:109D0000B385181619061A061B06FCF480919F0DE0
:109D10009091A00DA091A10DB091A20D8093B20DD4
:109D20009093B30DA093B40DB093B50D81E08093E3
:109D3000A70D80899189A289B3898093B60D9093EC
:109D4000B70DA093B80DB093B90D81E08093DC0DF1
:109D500004C02A9A81E080932B018091D90D83FF62
:109D600003C0289A8FEF02C0289881E080932C01CD
:109D700020E030E081C18091C00087FF19C0E091F0
:109D8000C60040912A0650912B06CA0101968F7792
:109D9000992760912C0670912D068617970741F040
:109DA000DA01A655BA4FEC9390932B0680932A06BE
:109DB000E091BA0DF091BB0D8091C90D9091CA0D43
:109DC000A091CB0DB091CC0D408151816281738106
:109DD000840F951FA61FB71F8093C90D9093CA0DBE
:109DE000A093CB0DB093CC0D181619061A061B06BE
:109DF00044F55F9A4089518962897389841B950B68
:109E0000A60BB70B8093C90D9093CA0DA093CB0DF1
:109E1000B093CC0D409129018091970D9091980DB0
:109E2000A091990DB0919A0D840F911DA11DB11DA6
:109E30008093970D9093980DA093990DB0939A0DE0
:109E40005F98E091BA0DF091BB0D8091CD0D90918E
:109E5000CE0DA091CF0DB091D00D4481558166817A
:109E60007781840F951FA61FB71F8093CD0D909308
:109E7000CE0DA093CF0DB093D00D181619061A066B
:109E80001B0644F5469A4089518962897389841B6F
:109E9000950BA60BB70B8093CD0D9093CE0DA09391
:109EA000CF0DB093D00D40912A0180919B0D9091E0
:109EB0009C0DA0919D0DB0919E0D840F911DA11D33
:109EC000B11D80939B0D90939C0DA0939D0DB0931D
:109ED0009E0D4698E091BA0DF091BB0D8091D10D89
:109EE0009091D20DA091D30DB091D40D40855185A4
:109EF00062857385840F951FA61FB71F8093D10DB0
:109F00009093D20DA093D30DB093D40D18161906CB
:109F10001A061B0644F52B9A408951896289738978
:109F2000841B950BA60BB70B8093D10D9093D20D8C
:109F3000A093D30DB093D40D40912B0180919F0D30
:109F40009091A00DA091A10DB091A20D840F911D33
:109F5000A11DB11D80939F0D9093A00DA093A10D05
:109F6000B093A20D2B98E091BA0DF091BB0D8091AA
:109F7000D50D9091D60DA091D70DB091D80D4485F7
:109F8000558566857785840F951FA61FB71F80931B
:109F9000D50D9093D60DA093D70DB093D80D18166C
:109FA00019061A061B0644F5299A408951896289C7
:109FB0007389841B950BA60BB70B8093D50D9093DB
:109FC000D60DA093D70DB093D80D40912C01809160
:109FD000A30D9091A40DA091A50DB091A60D840F95
:109FE000911DA11DB11D8093A30D9093A40DA0936D
:109FF000A50DB093A60D29988091B60D9091B70D3F
:10A00000A091B80DB091B90D0196A11DB11D80931D
:10A01000B60D9093B70DA093B80DB093B90D4091C4
:10A02000B60D5091B70D6091B80D7091B90D2F5FBD
:10A030003F4FE091BA0DF091BB0D80899189A289C3
:10A04000B389481759076A077B07B0F04091B60DEE
:10A050005091B70D6091B80D7091B90DE091BA0DA6
:10A06000F091BB0D84899589A689B78984179507D6
:10A07000A607B70748F4E0C08091C00D90E028170C
:10A0800039070CF478CEE2CF4091C50D5091C60D42
:10A090006091C70D7091C80D048D158D268D378D7B
:10A0A000AA27419FB12D529FC001629F900D619FD1
:10A0B000800D911D429FB00D811D9A1F519FB00DC3
:10A0C000811D9A1F609FB00D811D9A1F509FB10D79
:10A0D0008A1F9A1FB6958A1F9A1F112444AD55AD49
:10A0E000480F591F5093C40D4093C30D80AD91ADDF
:10A0F000A2ADB3AD60E070E084179507A607B7077F
:10A1000020F49093C40D8093C30D6091C30D7091A2
:10A11000C40D61349CE9790728F461328EE4780734
:10A1200048F002C060E47CE976956795769567957E
:10A1300084E007C0613197E2790730F07695679542
:10A1400082E08093C00D08C081E08093C00D603232
:10A15000710510F460E270E060527109611588E0E9
:10A160007807E0F0872F9927880F991F880F991F8C
:10A170008D5E9A4FFC01329625913491AA27639FF8
:10A18000A001629F410D5A1F06944A1F5A1F1124B5
:10A19000FC0125913491241B350B1EC0CB019695F3
:10A1A00087958C7F8D5E964FFC01259134910296A8
:10A1B000FC0145915491FB01E770FF274E9FC001C0
:10A1C0004F9F900D5E9F900D1124F3E0969587951B
:10A1D000FA95E1F7281B390B24363105A0F4E2E7A4
:10A1E000F2E006C09091C00095FFFCCF8093C600BE
:10A1F00081918111F7CF4AE050E089EA95E00E9411
:10A20000432824E630E03093890020938800809131
:10A21000C50D9091C60DA091C70DB091C80D820FCC
:10A22000931FA11DB11D8093C50D9093C60DA093E2
:10A23000C70DB093C80DF3C04091B60D5091B70D46
:10A240006091B80D7091B90D808D918DA28DB38DF7
:10A2500084179507A607B70708F0D9C04091BC0D31
:10A260005091BD0D6091BE0D7091BF0D048D158D87
:10A27000268D378DAA27419FB12D529FC001629F25
:10A28000900D619F800D911D429FB00D811D9A1F01
:10A29000519FB00D811D9A1F609FB00D811D9A1FA7
:10A2A000509FB10D8A1F9A1FB6958A1F9A1F1124BD
:10A2B0002091C30D3091C40DE05CFF4F2817390782
:10A2C00018F42081318102C0281B390B80819181D3
:10A2D000A281B381A90160E070E0481759076A07BD
:10A2E0007B0708F49C0121349CE9390728F42132CA
:10A2F0008EE4380748F002C020E43CE93695279503
:10A300003695279584E007C0213197E2390730F070
:10A310003695279582E08093C00D08C081E0809338
:10A32000C00D2032310510F420E230E0B901605256
:10A330007109611588E07807E0F0872F9927880F69
:10A34000991F880F991F8D5E9A4FFC013296459197
:10A350005491AA27659F9001649F210D3A1F06948E
:10A360002A1F3A1F1124FC0145915491421B530BA3
:10A370001EC0CB01969587958C7F8D5E964FFC0114
:10A38000459154910296FC0125913491FB01E770AF
:10A39000FF272E9FC0012F9F900D3E9F900D1124EF
:10A3A00033E0969587953A95E1F7481B590B44366B
:10A3B0005105A0F4E2E7F2E006C09091C00095FFDD
:10A3C000FCCF8093C60081918111F7CF4AE050E025
:10A3D00089EA95E00E94432844E650E050938900C2
:10A3E000409388008091BC0D9091BD0DA091BE0D51
:10A3F000B091BF0D840F951FA11DB11D8093BC0DA1
:10A400009093BD0DA093BE0DB093BF0D08C0809179
:10A41000C10D9091C20D9093890080938800409166
:10A42000B60D5091B70D6091B80D7091B90DE091D6
:10A43000BA0DF091BB0D80899189A289B389481723
:10A4400059076A077B0700F11092BB0D1092BA0DF5
:10A4500090913D0880913C089817B1F080913C089C
:10A460008F5F8F7080933C080FC08091DA0D81114F
:10A47000BCCBE3CB8091DB0D8111F7CB22CC80915B
:10A48000DC0D811136CC61CCFF91EF91BF91AF9182
:10A490009F918F917F916F915F914F913F912F91FC
:10A4A0001F910F910F900FBE0F901F9018953D9A1E
:10A4B0003F9A229A209A569A5E9A569A5E9A0D9AD6
:10A4C000159A569A5E9A3A98429A3B98439A3C98C3
:10A4D000449A579A5F985E9A3E9A46985E9A239A53
:10A4E0002B98159A219A29985E9AA1E8B0E08C9150
:10A4F0008F7E8C938C9188608C93E0E8F0E0808173
:10A500008D7F808380818E7F808380818F73808325
:10A5100080818F7C80838C91887F82608C9380E0A7
:10A5200090E49093890080938800109285001092A7
:10A530008400EFE6F0E080818260808381E0809398
:10A540002D017894089590913D0880913C089817CA
:10A5500031F00E94F45481E00E94FC12F4CF08957F
:10A56000CF93DF93EFB7F894EC0188819981AA81AA
:10A57000BB818093970D9093980DA093990DB09304
:10A580009A0DEB0188819981AA81BB8180939B0DF3
:10A5900090939C0DA0939D0DB0939E0DEA01888130
:10A5A0009981AA81BB8180939F0D9093A00DA09368
:10A5B000A10DB093A20DE90188819981AA81BB8187
:10A5C0008093A30D9093A40DA093A50DB093A60D19
:10A5D000EFBFDF91CF9108952FB7F894FC018081F0
:10A5E0009181A281B3818093A30D9093A40DA09338
:10A5F000A50DB093A60D2FBF08950F931F939FB77E
:10A60000F89424E0829FF0011124E956F24F008172
:10A610001181228133819FBFB801C9011F910F9120
:10A6200008950E94A3525E9A5E9A159A5E9A0895C2
:10A6300080916F008D7F80936F0006C080913C08F1
:10A640008F5F8F7080933C0890913D0880913C080B
:10A6500098130AC01092BB0D1092BA0D80916F0032
:10A66000826080936F00089590913D0880913C082E
:10A67000981751F3E3CF2091360130913701409183
:10A6800038015091390160E070E08FE793E40E9457
:10A6900080696093EB0D7093EC0D8093ED0D9093BA
:10A6A000EE0D08958651924FFC01808190E008954F
:10A6B0000F931F93CF93DF93EC01662309F461C0DE
:10A6C000EAEFFDE007C09091C00095FFFCCF8093BA
:10A6D000C600319684918111F6CF4AE050E070E0D7
:10A6E00089EA95E00E942528E1E0FEE007C090910C
:10A6F000C00095FFFCCF8093C600319684918111F4
:10A70000F6CF8091C00085FFFCCF8AE08093C60021
:10A710000E94D31236C0C901880F991F880F991F54
:10A72000FC01E15EF14F659174916C177D073CF57A
:10A7300021503109220F331F220F331FF901E35E2D
:10A74000F14F05911491215E314FF90145915491DA
:10A75000FC01E35EF14F25913491C41BD50B201B06
:10A76000310BC29FC001C39F900DD29F900D112449
:10A77000641B750B0E94376D600F711F13C04F5F14
:10A7800001C041E0242F30E04D3309F0C4CF2D3318
:10A79000310531F4EDE0FFE085919491BC0102C0F8
:10A7A00060E070E020EF3FE3261B370BC901DF912B
:10A7B000CF911F910F910895CF93DF9321E030E067
:10A7C000D901AA0FBB1FAA0FBB1FFD01E15EF14F0C
:10A7D000659174916817790744F521503109220F6A
:10A7E000331F220F331FF901E35EF14FC591D4915E
:10A7F000215E314FF90145915491FD01E35EF14F26
:10A8000025913491FC01E41BF50B2C1B3D0BE29FC1
:10A81000C001E39F900DF29F900D1124641B750BF6
:10A820000E94376D6C0F7D1F0BC02F5F3F4F2D3384
:10A83000310509F0C5CFEDE0FFE085919491BC01B1
:10A8400020EF3FE3261B370BC901DF91CF9108951D
:10A850002F923F924F925F926F927F928F929F9230
:10A86000AF92BF92CF92DF92EF92FF920F931F931E
:10A87000CF93DF938C01662351F1EAEFFDE007C02F
:10A880009091C00095FFFCCF8093C60031968491D3
:10A890008111F6CF4AE050E070E089EA95E00E942D
:10A8A0002528E1E1FFE007C09091C00095FFFCCFB3
:10A8B0008093C600319684918111F6CF8091C000BB
:10A8C00085FFFCCF8AE08093C6000E94D312C0EFC0
:10A8D000DFE3C01BD10B41E05EC09C01220F331FA0
:10A8E000220F331FF901E35EF14F65907490C61596
:10A8F000D7050CF04FC00197880F991F880F991F3B
:10A90000FC01E15EF14F25903490835E914FFC0194
:10A9100005911491F901E15EF14F45905490B10118
:10A92000882777FD8095982F0E941B6A6B017C0118
:10A93000BE01601B710B882777FD8095982F0E94C0
:10A940001B6A4B015C01B20162197309882777FD0C
:10A950008095982F0E941B6A9B01AC01C501B40130
:10A960000E944E6C4B015C01B301601B710B882788
:10A9700077FD8095982F0E941B6A9B01AC01C50151
:10A98000B4010E9480699B01AC01C701B6010E941D
:10A99000A06817C04F5F842F90E04D3309F09DCF22
:10A9A000CD9759F4EFE0FFE065917491882777FD2A
:10A9B0008095982F0E941B6A04C060E070E080E0E0
:10A9C00090E0DF91CF911F910F91FF90EF90DF907A
:10A9D000CF90BF90AF909F908F907F906F905F903F
:10A9E0004F903F902F9008952F923F924F925F92F9
:10A9F0006F927F928F929F92AF92BF92CF92DF928F
:10AA0000EF92FF920F931F93CF93DF9300D0CDB7B8
:10AA1000DEB78091DD0D882309F4BFC18FB7F894AC
:10AA20001092DD0D8FBF60E08091E40D9091E50DF7
:10AA30000E9428546B017C019B01AC016091DE0DEA
:10AA40007091DF0D8091E00D9091E10D0E949F6863
:10AA5000B62EA72E182F092FA5019801852F942F08
:10AA6000A32FB22F8093EF0D9093F00DA093F10DD3
:10AA7000B093F20D20E030E040E251E4D501F8015E
:10AA80006B2F7A2F8F2F9E2F0E947C6B18160CF441
:10AA90001DC120E030E040E251ECD501F8016B2F00
:10AAA0007A2F8F2F9E2F0E94796987FD0BC180918D
:10AAB000F30D8111FCC020913A0130913B0140918E
:10AAC0003C0150913D01D501F8016B2F7A2D8F2F5C
:10AAD000902F0E944E6C762E672E89839A83A30155
:10AAE000382F292F852F942FA32FB22F8093F80D65
:10AAF0009093F90DA093FA0DB093FB0D2091F40DF6
:10AB00003091F50D4091F60D5091F70DD501F801FA
:10AB10006B2F7A2D8F2F902F0E94A0688B012C0114
:10AB20008090FC0D9090FD0DA090FE0DB090FF0D5B
:10AB3000282D392D4A2D5B2D602F712F842D952DB9
:10AB40000E94796987FF9DC084012501802F912F84
:10AB5000A42DB52D8093F40D9093F50DA093F60DD3
:10AB6000B093F70D209136013091370140913801B3
:10AB700050913901602F712F842D952D0E944E6CBC
:10AB80004B015C01862F992DAA2DBB2D8093000EC1
:10AB90009093010EA093020EB093030E2091040E29
:10ABA0003091050E4091060E5091070EC701B60177
:10ABB0000E949F682091320130913301409134010D
:10ABC000509135010E944E6C20ED3CEC4CE45DE36D
:10ABD0000E944E6C1B012C0123E333E343E75FE348
:10ABE0006091080E7091090E80910A0E90910B0EE3
:10ABF0000E944E6C9B01AC01C201B1010E94A06891
:10AC00008B012C01862F912FA42DB52D8093080E3A
:10AC10009093090EA0930A0EB0930B0EC092040EEF
:10AC2000D092050EE092060EF092070E282D392DD7
:10AC30004A2D5B2DD301F980EA806B2F762D8F2D65
:10AC40009E2D0E94A068202F312F442D552D0E944B
:10AC50009F688B017C0120E030E0A901712F9F2DBE
:10AC60000E94796987FD3CC020E030E04FE753E463
:10AC7000602F712F8E2D9F2D0E947C6B1816A4F5CE
:10AC800028C08090EB0D9090EC0DA090ED0DB09051
:10AC9000EE0D282D392D4A2D5B2D602F712F842D1F
:10ACA000952D0E947C6B18160CF050CF4DCF109252
:10ACB000F40D1092F50D1092F60D1092F70D109202
:10ACC000F30DF9CE81E08093F30D0AC081E080930B
:10ACD000F30D00E010E08FE7E82E93E4F92E04C0B6
:10ACE00000E010E0E12CF12C2091E40D3091E50D15
:10ACF00040910C0E50910D0E421753071CF010920C
:10AD0000EA0D11C040913E0150913F0124173507D3
:10AD1000B4F7602F712F8E2D9F2D0E94E8697595D5
:10AD200067956093EA0D0E94622500910E0E1091C6
:10AD30000F0E2091100E3091110E601B710B820BC3
:10AD4000930B683873418105910538F10E946225A3
:10AD500060930E0E70930F0E8093100E9093110E51
:10AD60008091E20D9091E30D2091120E3091130E1F
:10AD7000281739078CF42091400130914101821746
:10AD8000930754F42091E60D3091E70D8217930755
:10AD90000CF002C05A9A01C05A980F900F90DF91A0
:10ADA000CF911F910F91FF90EF90DF90CF90BF90C8
:10ADB000AF909F908F907F906F905F904F903F905B
:10ADC0002F9008952F923F924F925F926F927F92B1
:10ADD0008F929F92AF92BF92CF92DF92EF92FF92AB
:10ADE0000F931F93CF93DF93C0EFDFE3C81BD90B03
:10ADF00081E090E09C01220F331F220F331FF901E5
:10AE0000E35EF14F65907490C615D7050CF04FC006
:10AE10000197880F991F880F991FFC01E15EF14F80
:10AE200025903490835E914FFC0105911491F901B6
:10AE3000E15EF14F45905490B101882777FD8095F0
:10AE4000982F0E941B6A6B017C01BE01601B710B75
:10AE5000882777FD8095982F0E941B6A4B015C0123
:10AE6000B20162197309882777FD8095982F0E9497
:10AE70001B6A9B01AC01C501B4010E944E6C4B01E1
:10AE80005C01B301601B710B882777FD8095982FBB
:10AE90000E941B6A9B01AC01C501B4010E9480693C
:10AEA0009B01AC01C701B6010E94A0680FC00196CA
:10AEB0008D33910509F09ECFEFE0FFE0659174912D
:10AEC000882777FD8095982F0E941B6ADF91CF918C
:10AED0001F910F91FF90EF90DF90CF90BF90AF90B8
:10AEE0009F908F907F906F905F904F903F902F90AA
:10AEF00008951092FC0D1092FD0D1092FE0D10920F
:10AF0000FF0D209136013091370140913801509169
:10AF1000390160E070E08FE793E40E9480696093FC
:10AF2000EB0D7093EC0D8093ED0D9093EE0D559A13
:10AF3000529A87ED80937A00EEE7F0E010828081EC
:10AF40008068808380818064808380E888BDEEE6AD
:10AF5000F0E08081846080836AEF70E080E090E0C0
:10AF60000E949E2560E085E090E00E9458539093F7
:10AF70000D0E80930C0E60E083E191E00E94585327
:10AF800090933F0180933E0185E090E00E94DC5366
:10AF90009093130E8093120E86E990E00E94DC538A
:10AFA00090934101809340010895089560E080E00E
:10AFB00090E00E9458531092DE0D1092DF0D109217
:10AFC000E00D1092E10D80E090E00E94DC53909340
:10AFD000E70D8093E60D1092E90D1092E80D1092A6
:10AFE000EA0D5D981092E70D1092E60D5A980895BB
:10AFF0002F923F924F925F926F927F928F929F9289
:10B00000AF92BF92CF92DF92EF92FF920F931F9376
:10B01000CF93DF93CDB7DEB7E1970FB6F894DEBFDD
:10B020000FBECDBF688B798B8A8B9B8B0E9462256C
:10B030006C8B7D8B8E8B9F8BE6E8F2E006C0909147
:10B04000C00095FFFCCF8093C60081918111F7CF9E
:10B050008091C00085FFFCCF8AE08093C6000E94EB
:10B06000D6578FE78093EA0D4C885D886E887F887D
:10B070004C865D866E867F86AFE7CA2ED12CE12C8A
:10B08000F12CBFE78B2E912CA12CB12C8EA69FA664
:10B09000A8AAB9AA11E01B861A86E3E1FDE0949004
:10B0A0009FA2EBE1FDE0A490A8A6E0E2FDE0B49051
:10B0B000B9A6E7E2FDE084908AA6EEE2FDE0949076
:10B0C0009BA6E4E3FDE0A490ACA68091DD0D88236F
:10B0D00009F4BBC28FB7F8941092DD0D8FBF60E00A
:10B0E0008091E40D9091E50D0E9428546E837F833A
:10B0F00088879987762F6F81982F8985272F362FFC
:10B10000492F582FB88DA98DEA8DFB8D6B2F7A2F83
:10B11000CF010E947C6B181644F0BE80B88E8F80E1
:10B12000898E98849A8EA984AB8E7E816F81988552
:10B130008985272F362F492F582FECA1602F722D8C
:10B14000832D9E2F0E94796987FD05C00E812F8077
:10B150003884B984BCA2112309F43FC37889698972
:10B160009A898B89272F362F492F582FBE81AF817F
:10B17000E885F9856B2F7A2FCF010E947C6B18161A
:10B180000CF063C20E94622564197509860997094B
:10B19000693873418105910508F457C28EA59FA5B2
:10B1A000A8A9B9A98C199D09AE09BF09B595A7959C
:10B1B000979587958093EA0D0E9462256C877D871D
:10B1C0008E879F874B015C0184189508A608B708F5
:10B1D00088A299A2AAA2BBA29888988EA988A98EB3
:10B1E000BA88BA8E8B888B8EF8C20E9462258C84B6
:10B1F0009D84AE84BF84681979098A099B096938DE
:10B2000073418105910508F41FC20E9462252B013C
:10B210003C018A849B84892809F4FCC1DC01CB01B0
:10B220008C849D84AE84BF8488199909AA09BB09BE
:10B2300088A099A0AAA0BBA0880E991EAA1EBB1E1A
:10B2400028A139A14AA15BA1281B390B4A0B5B0B32
:10B25000CA01B901A70196010E94276DA5019401B9
:10B260000E946D6D8EA59FA5A8A9B9A9280F391FA9
:10B270004A1F5B1F243131054105510524F12EA7DA
:10B280003FA748AB59AB2C3E31054105510544F071
:10B290002BEE30E040E050E02EA73FA748AB59AB83
:10B2A0008EA59FA5A8A9B9A980389105A105B105CA
:10B2B000C4F0EEEFCE2ED12CE12CF12CC81AD90A15
:10B2C000EA0AFB0A12C024E130E040E050E02EA779
:10B2D0003FA748AB59AB74E1C72ED12CE12CF12C20
:10B2E00004C0CEA4DFA4E8A8F9A88FA1E3E1FDE0A3
:10B2F00008C09091C00095FFFCCF8093C6003196A6
:10B3000084918111F6CF2AE030E04EA55FA568A9AF
:10B3100079A989EA95E00E94142888A5EBE1FDE06F
:10B3200008C09091C00095FFFCCF8093C600319675
:10B3300084918111F6CF2AE030E0B701A60189EAB5
:10B3400095E00E94142889A5E0E2FDE008C09091F4
:10B35000C00095FFFCCF8093C60031968491811187
:10B36000F6CF22E030E08CA1402F522D632D782FB4
:10B3700089EA95E00E941E298AA5E7E2FDE008C05F
:10B380009091C00095FFFCCF8093C60031968491C8
:10B390008111F6CF22E030E0F88DE98D9A8D8B8D0A
:10B3A0004F2F5E2F692F782F89EA95E00E941E2982
:10B3B0008091C00085FFFCCF8AE08093C6004A855B
:10B3C0005B85433051050CF425C1C701B6010E94CD
:10B3D0001B6A20E030E040E850E40E944E6C6C8F25
:10B3E0007D8F8E8F9F8F8CA1202F322D432D582F34
:10B3F000B88DA98DEA8D1B8D6B2F7A2F8E2F912FF3
:10B400000E949F6820ED3FE049E450E40E944E6CAA
:10B4100020E030E040E05FE30E944E6C9B01AC0115
:10B420006C8D7D8D8E8D9F8D0E948069362E072FAD
:10B43000182F9C8FC501B4010E941B6A20E030E0E8
:10B440004AE754E40E948069A62E972E282E892E62
:10B450008BA5EEE2FDE008C09091C00095FFFCCF07
:10B460008093C600319684918111F6CF22E030E0BE
:10B470008C8D432D502F612F782F89EA95E00E9403
:10B480001E298CA5E4E3FDE008C09091C00095FF63
:10B49000FCCF8093C600319684918111F6CF22E0D3
:10B4A00030E04A2D592D622D782D89EA95E00E94D1
:10B4B0001E298091C00085FFFCCF8AE08093C600E2
:10B4C0002AE939E949E15FE3EC8D632D702F812F83
:10B4D0009E2F0E944E6C362E072F182FB92E762FD6
:10B4E000272F302F412F5B2D632D702F812F9B2D08
:10B4F0000E94A0682A2D392D422D582D0E94806966
:10B500006C8F7CA38DA39EA32A2D392D422D582DFF
:10B51000632D702F812F9B2D0E944E6C20E030E018
:10B5200040E05EE30E944E6CA62E972E282E892EB8
:10B53000EAE3FDE007C09091C00095FFFCCF809347
:10B54000C600319684918111F6CF8091C00085FFAD
:10B55000FCCF8AE08093C600E7E4FDE007C090914D
:10B56000C00095FFFCCF8093C60031968491811175
:10B57000F6CF22E030E0432D502F612F7B2D89EA5A
:10B5800095E00E941E298091C00085FFFCCF8AE0D3
:10B590008093C600EDE4FDE007C09091C00095FFE8
:10B5A000FCCF8093C600319684918111F6CF22E0C2
:10B5B00030E0FC8DECA19DA18EA14F2F5E2F692F55
:10B5C000782F89EA95E00E941E298091C00085FFAE
:10B5D000FCCF8AE08093C600E3E5FDE007C09091D0
:10B5E000C00095FFFCCF8093C600319684918111F5
:10B5F000F6CF22E030E04A2D592D622D782D89EAD0
:10B6000095E00E941E298091C00085FFFCCF8AE052
:10B610008093C6008EA59FA5A8A9B9A98C0D9D1DD4
:10B62000AE1DBF1DB595A795979587958093EA0D9B
:10B630008A859B8501969B878A87088929883A880D
:10B640008B888CA211E001C010E020E030E040EADD
:10B6500051E4B889A989EA89FB896B2F7A2FCF0138
:10B660000E94A0689B01AC01BE81AF81E885F9858D
:10B670006B2F7A2FCF010E947C6B181694F4E9E5AA
:10B68000FDE007C09091C00095FFFCCF8093C600FD
:10B69000319684918111F6CF8091C00085FFFCCF57
:10B6A00098C00E9462258C889D88AE88BF886819E2
:10B6B00079098A099B09613D77408105910508F464
:10B6C0003FC00E9462256C8B7D8B8E8B9F8BE2E846
:10B6D000FDE007C09091C00095FFFCCF8093C600AD
:10B6E000319684918111F6CF60E08091E40D9091C4
:10B6F000E50D0E942854AB01BC0122E030E089EA4C
:10B7000095E00E941E29E8E8FDE007C09091C00086
:10B7100095FFFCCF8093C600319684918111F6CFBE
:10B720006091EA0D4AE050E070E089EA95E00E94FD
:10B7300025288091C00085FFFCCF8AE08093C60059
:10B740000E9462256A837B838C839D830E9462258D
:10B750008C849D84AE84BF84840C951CA61CB71C6D
:10B760002A813B814C815D81281939094A095B098D
:10B77000260F371F481F591F21383F4442415105AA
:10B7800090F0ECE8FDE007C09091C00095FFFCCF81
:10B790008093C600319684918111F6CF8091C000CC
:10B7A00085FFFCCF16C0AA85BB8516970CF48DCCFF
:10B7B000E9EAFDE007C09091C00095FFFCCF8093BF
:10B7C000C600319684918111F6CF8091C00085FF2B
:10B7D000FCCF8AE08093C60015C0788969899A8970
:10B7E0008B89272F362F492F582FBE81AF8118857F
:10B7F000F9856B2F7A2F812F9F2F0E94796987FD02
:10B80000F4CC22CFE1960FB6F894DEBF0FBECDBFC9
:10B81000DF91CF911F910F91FF90EF90DF90CF902C
:10B82000BF90AF909F908F907F906F905F904F9060
:10B830003F902F900895CF93DF931F92CDB7DEB73F
:10B8400089830E94D6570E94DF24698181112FC00D
:10B85000EAEFFDE007C08091C00085FFFCCF909328
:10B86000C600319694919111F6CF4AE050E070E015
:10B8700089EA95E00E9425288091C00085FFFCCFD1
:10B880008AE08093C600EEE2FFE007C09091C0001E
:10B8900095FFFCCF8093C600319684918111F6CF3D
:10B8A0008091C00085FFFCCF8AE08093C6000F9096
:10B8B000DF91CF910895CF93DF931F92CDB7DEB77D
:10B8C00089830E94D6570E94DF24698181112FC08D
:10B8D000EAEFFDE007C08091C00085FFFCCF9093A8
:10B8E000C600319694919111F6CF4AE050E070E095
:10B8F00089EA95E00E9425288091C00085FFFCCF51
:10B900008AE08093C600EBE5FFE007C09091C0009D
:10B9100095FFFCCF8093C600319684918111F6CFBC
:10B920008091C00085FFFCCF8AE08093C6000F9015
:10B93000DF91CF9108955A980E94DF24811121C090
:10B94000EAEFFDE007C09091C00095FFFCCF809327
:10B95000C600319684918111F6CFE8E8FFE007C078
:10B960009091C00095FFFCCF8093C60031968491E2
:10B970008111F6CF8091C00085FFFCCF8AE08093D3
:10B98000C60008951F920F920FB60F9211242F93A5
:10B990003F934F935F936F937F938F939F93AF9357
:10B9A000BF93EF93FF9380914201811106C0809174
:10B9B000EA0D8093140E81115D9A9091140E80917E
:10B9C0004201891708F05D988F5F8F77809342015D
:10B9D0008091150E833009F443C020F48130D1F0FA
:10B9E000A8F50CC0853009F457C008F453C0863060
:10B9F00009F454C0873009F05AC052C010927B003D
:10BA000087E480937C0080917A00806480937A0040
:10BA100081E019C020917800309179008091160E54
:10BA20009091170EA091180EB091190E820F931FCE
:10BA3000A11DB11D8093160E9093170EA093180EA2
:10BA4000B093190E82E08093150E31C086E4809386
:10BA50007C0080917A00806480937A0083E0F3CF49
:10BA6000209178003091790080911A0E90911B0EF0
:10BA7000A0911C0EB0911D0E820F931FA11DB11D30
:10BA800080931A0E90931B0EA0931C0EB0931D0E64
:10BA900084E0D9CF85E0D7CF86E0D5CF87E0D3CF7C
:10BAA0001092150E80911E0E8F5F80931E0E809156
:10BAB0001E0E803108F474C02FEF3FE38091160E04
:10BAC0009091170EA901481B590BCA015093E50D1F
:10BAD0004093E40D40911A0E50911B0E241B350B20
:10BAE0003093E30D2093E20D21E02093DD0D1092C1
:10BAF0001E0E1092160E1092170E1092180E109223
:10BB0000190E10921F0E1092200E1092210E1092FC
:10BB1000220E1092230E1092240E1092250E1092D7
:10BB2000260E10921A0E10921B0E10921C0E1092DE
:10BB30001D0E20913E0130913F01821793074CF07A
:10BB40001092E90D1092E80D80E00E941B5C0E94AB
:10BB5000A4242091E40D3091E50D80910C0E90917C
:10BB60000D0E821793074CF01092E90D1092E80D1C
:10BB700080E00E945B5C0E94A4242091E20D309141
:10BB8000E30D80914001909141012817390744F05D
:10BB90001092E70D1092E60D0E949B5C0E94A42477
:10BBA000FF91EF91BF91AF919F918F917F916F9195
:10BBB0005F914F913F912F910F900FBE0F901F906B
:10BBC0001895CF93DF93FC01148A178A8CE692E0D4
:10BBD000938B828B13AA16AA92AB81ABDF01A05B79
:10BBE000BF4F1C9213961C92DF01A25BBF4F8D9337
:10BBF0009C93DF01A359BF4F1C9213961C92DF0147
:10BC0000A559BF4F8D939C93DF01A857BF4F29E1E2
:10BC100011962C93119714961C92DF01A357BF4FD6
:10BC200057961C92DF01A355BF4F1C9213961C928E
:10BC3000DF01A555BF4F8D939C93DF01A853BF4FE4
:10BC40001D921D921D921C921397DF01A053BF4FAE
:10BC50001D921D921D921C921397118212821082C6
:10BC6000EF01C453DF4F188219821A821B82DF0151
:10BC7000AC52BF4F81E08C93118A108A0E946225DA
:10BC800068577C4E8F4F9F4F688379838A839B834D
:10BC9000DF91CF910895DB01FC0120E03EE24C9161
:10BCA000403229F0283009F431934C9141932F5FB1
:10BCB00011962B30A1F7108208952F923F924F9248
:10BCC0005F926F927F928F929F92AF92BF92CF922C
:10BCD000DF92EF92FF920F931F93CF93DF93CDB735
:10BCE000DEB7C158D1090FB6F894DEBF0FBECDBF85
:10BCF0008C017B01212C4A0182E0880E911C680195
:10BD0000E5EDCE0ED11C5801F6EDAF0EB11C8EE361
:10BD1000482E512C4C0E5D1E82E0480E511CE2EC68
:10BD2000FFE03490F3C09C85292F2871203109F061
:10BD300007C1F6018081813009F402C1823009F027
:10BD4000EFC0FEC069E972E0CE01855A9F4F0E94A4
:10BD50005B70B701CE01855A9F4F0E945B70BE0198
:10BD60006B587F4FCE01855A9F4F0E945B7069E9E7
:10BD700072E0CE01855A9F4F0E945B7021961FAEE4
:10BD8000219724961FAE24978CE692E09FAF8EAF4A
:10BD900021E0AE014B585F4FB401C2010E94552F04
:10BDA000811139C0F6018081811135C0832DE2EC0B
:10BDB000FFE008C09091C00095FFFCCF8093C600C3
:10BDC000319684918111F6CFABE9B2E006C0909133
:10BDD000C00095FFFCCF8093C6008D918111F7CFF5
:10BDE0008091C00085FFFCCF8AE08093C600DE0111
:10BDF000AB58BF4F06C09091C00095FFFCCF809319
:10BE0000C6008D918111F7CF8091C00085FFFCCFD6
:10BE10008AE08093C6008BE1FE01E05CFF4FDE010B
:10BE2000939601900D928A95E1F78CE692E09AA3A1
:10BE300089A3AE014F5D5F4FBE01655A7F4FC801B8
:10BE40000E945D5ECE0181960E94E924CE01CE96CD
:10BE50000E94E9245BC0853E09F458C08E3209F483
:10BE600055C08F3509F452C093FD50C081E0203198
:10BE700009F080E0F8018787811108C0898587343F
:10BE800009F044C08A858E3709F440C03801F3E0D8
:10BE90006F0E711CBE016F5F7F4FC3010E944B5E2E
:10BEA000F601808181111EC0D70106C09091C000AB
:10BEB00095FFFCCF8093C6008D918111F7CFD30100
:10BEC00006C09091C00095FFFCCF8093C6008D9175
:10BED0008111F7CF8091C00085FFFCCF8AE080936D
:10BEE000C60014C0813039F4F5018081918101963A
:10BEF000918380830BC0823049F4222D30E0F5011C
:10BF00008081918128173907F1F02394BE016F5F7A
:10BF10007F4FC4010E94C32B18160CF404CF13C02A
:10BF2000BE016F5F7F4FCE018B589F4F0E944B5ECB
:10BF30006C961FAE6C97F701808181110ACF02CFFA
:10BF40008981811188CFCF57DF4F0FB6F894DEBFBC
:10BF50000FBECDBFDF91CF911F910F91FF90EF905A
:10BF6000DF90CF90BF90AF909F908F907F906F9019
:10BF70005F904F903F902F900895EF92FF920F9314
:10BF80001F93CF93DF93CDB7DEB76D970FB6F894BD
:10BF9000DEBF0FBECDBF8C01FC01EB52FF4F108204
:10BFA0007C0184E1E80EF11C40E050E0BA01C701D9
:10BFB0000E94362C8BE1F701DE01139601900D9261
:10BFC0008A95E1F78CE692E09A838983AE014F5F10
:10BFD0005F4F65E872E0C8010E945D5ECE01019688
:10BFE0000E94E9246D960FB6F894DEBF0FBECDBF58
:10BFF000DF91CF911F910F91FF90EF900895EF92F5
:10C00000FF920F931F93CF93DF93EC011A828F89D6
:10C01000882321F0CE0144960E941D2D7E0188E8E0
:10C02000E80EF11C4FE160E0C7010E945F678111DB
:10C030001FC0E2ECFFE007C09091C00095FFFCCF6D
:10C040008093C600319684918111F6CFE8ECFFE031
:10C0500007C09091C00095FFFCCF8093C600319639
:10C0600084918111F6CF8091C00085FFFCCF76C00E
:10C070008E0103571F4F41E0B701C8010E9452359E
:10C08000811126C040E0B701C8010E9452358111DC
:10C090001FC0E5EDFFE007C09091C00095FFFCCF09
:10C0A0008093C600319684918111F6CFECEDFFE0CC
:10C0B00007C09091C00095FFFCCF8093C6003196D9
:10C0C00084918111F6CF8091C00085FFFCCF46C0DE
:10C0D000B801CE0144960E94302A81111FC0E5EDBF
:10C0E000FFE007C09091C00095FFFCCF8093C60091
:10C0F000319684918111F6CFEFEEFFE007C0909169
:10C10000C00095FFFCCF8093C600319684918111C9
:10C11000F6CF8091C00085FFFCCF20C081E08A83EC
:10C12000E2ECFFE007C09091C00095FFFCCF809348
:10C13000C600319684918111F6CFEFEFFFE007C082
:10C140009091C00095FFFCCF8093C60031968491FA
:10C150008111F6CF8091C00085FFFCCF8AE08093EB
:10C16000C6008BE1FE017496DE01D39601900D921C
:10C170008A95E1F7CE01429698AB8FA7DF91CF91D8
:10C180001F910F91FF90EF900895FC011182128290
:10C190000895FC012281222311F021E021830895DA
:10C1A000FC0121812111118208952F923F924F921B
:10C1B0005F926F927F928F929F92AF92BF92CF9237
:10C1C000DF92EF92FF920F931F93CF93DF93CDB740
:10C1D000DEB7AA970FB6F894DEBF0FBECDBF7C01C5
:10C1E0006B01342EFC018281882309F4B4C147011C
:10C1F000FDEA8F0E911CC4010E941D2DF7011182D2
:10C200001B821E828CE692E09A838983C701429644
:10C2100090AB87A7F60180818F3209F08CC06FE266
:10C2200070E0C6010E9466708C010F5F1F4F9AE09C
:10C23000292E44244394512C4C0E5D1E77C06FE28E
:10C2400070E0C8010E9466705C01009709F47BC031
:10C250000817190708F077C03C01601A710AA3019A
:10C26000B801CE014E960E948670EEE1F0E0EC0F30
:10C27000FD1FE60DF71D10828E01025E1F4FF801B3
:10C2800006C09091C00095FFFCCF8093C6008191BD
:10C290008111F7CF8091C00085FFFCCF2092C600AE
:10C2A000F70167A570A96115710519F06E5F7F4FE1
:10C2B00002C060E070E021E0AE01425E5F4FCE015F
:10C2C00003960E94552F81112BC0EAE0F0E107C0D0
:10C2D0009091C00095FFFCCF8093C6003196849169
:10C2E0008111F6CF06C09091C00095FFFCCF8093DE
:10C2F000C600F80181918F018111F5CFEEE1F0E1E7
:10C3000007C09091C00095FFFCCF8093C600319686
:10C3100084918111F6CF8091C00085FFFCCF14C1BC
:10C32000F70150AA47A685010F5F1F4F01151105A0
:10C3300009F085CF05C0C701C196F70190AB87A76B
:10C34000BC2CAD2C02C0B02EA12EF70167A570A9A0
:10C35000332009F49FC06115710519F06E5F7F4F9E
:10C3600002C060E070E021E04B2D5A2DC4010E9414
:10C37000552F882309F463C0F701E853FF4FD70115
:10C38000A355BF4F51960D911D912D913C915497FE
:10C390000083118322833383E0E2F0E107C09091B0
:10C3A000C00095FFFCCF8093C60031968491811127
:10C3B000F6CFEB2DFA2D06C09091C00095FFFCCF73
:10C3C0008093C60081918111F7CFEDE2F0E107C0C3
:10C3D0009091C00095FFFCCF8093C6003196849168
:10C3E0008111F6CFF701E853FF4F408151816281FF
:10C3F00073812AE030E089EA95E00E94012880916B
:10C40000C00085FFFCCF8AE08093C600F701E053AF
:10C41000FF4F1082118212821382E4E3F0E107C021
:10C420009091C00095FFFCCF8093C6003196849117
:10C430008111F6CF8091C00085FFFCCF85C0E2E47A
:10C44000F0E107C09091C00095FFFCCF8093C6003B
:10C45000319684918111F6CFEB2DFA2D06C0909183
:10C46000C00095FFFCCF8093C60081918111F7CF6A
:10C47000E6E5F0E107C09091C00095FFFCCF809306
:10C48000C600319684918111F6CF8091C00085FF5E
:10C49000FCCF5AC06115710519F06E5F7F4F02C065
:10C4A00060E070E026E54B2D5A2DC4010E94552F07
:10C4B00081112BC0E8E5F0E107C09091C00095FF25
:10C4C000FCCF8093C600319684918111F6CFEB2D7D
:10C4D000FA2D06C09091C00095FFFCCF8093C60056
:10C4E00081918111F7CFECE6F0E107C09091C00097
:10C4F00095FFFCCF8093C600319684918111F6CFD1
:10C500008091C00085FFFCCF1FC081E0F7018083D0
:10C51000EEE6F0E107C09091C00095FFFCCF80935C
:10C52000C600319684918111F6CFF60106C0909134
:10C53000C00095FFFCCF8093C60081918111F7CF99
:10C540008091C00085FFFCCF8AE08093C600CE01B9
:10C5500001960E94E924AA960FB6F894DEBF0FBE9A
:10C56000CDBFDF91CF911F910F91FF90EF90DF90A2
:10C57000CF90BF90AF909F908F907F906F905F9083
:10C580004F903F902F9008955F926F927F928F927D
:10C590009F92AF92BF92CF92DF92EF92FF920F9352
:10C5A0001F93CF93DF93CDB7DEB7AA970FB6F8945A
:10C5B000DEBF0FBECDBF8C016B01FC0182818823E1
:10C5C00009F408C1C80183559F4F0E941D2DF80131
:10C5D00011821B821E828CE692E09A838983C801B5
:10C5E000429690AB87A7F60180818F3209F08EC00A
:10C5F0006FE270E0C6010E94667001967C014AE01D
:10C60000542E66246394712C6C0E7D1E7AC06FE2EA
:10C6100070E0C7010E9466705C01009709F47CC05D
:10C62000E816F90608F078C04C018E189F08A4019E
:10C63000B701CE014E960E948670EEE1F0E0EC0F5D
:10C64000FD1FE80DF91D10823EE1E32EF12CEC0EEA
:10C65000FD1EF70106C09091C00095FFFCCF8093AE
:10C66000C60081918111F7CF8091C00085FFFCCF7A
:10C670005092C600F80167A570A96115710519F0FF
:10C680006E5F7F4F02C060E070E021E0AE01425E6D
:10C690005F4FCE0103960E94552F81112BC0E0E819
:10C6A000F0E107C09091C00095FFFCCF8093C600D9
:10C6B000319684918111F6CF06C09091C00095FF0C
:10C6C000FCCF8093C600F70181917F018111F5CFE6
:10C6D000E4E9F0E107C09091C00095FFFCCF8093A2
:10C6E000C600319684918111F6CF8091C00085FFFC
:10C6F000FCCF69C0F80170AA67A67501FFEFEF1AB9
:10C70000FF0AE114F10409F082CF05C0C801C19607
:10C71000F80190AB87A77601F80187A590A900974B
:10C7200011F0029602C080E090E0B7010E94123042
:10C73000882301F1E6E9F0E107C09091C00095FF80
:10C74000FCCF8093C600319684918111F6CFF7011A
:10C7500006C09091C00095FFFCCF8093C6008191E8
:10C760008111F7CFF801E053FF4F1082118212823E
:10C7700013822CC0E4EAF0E107C09091C00095FF5D
:10C78000FCCF8093C600319684918111F6CFF701DA
:10C7900006C09091C00095FFFCCF8093C6008191A8
:10C7A0008111F7CFECEBF0E107C09091C00095FF4D
:10C7B000FCCF8093C600319684918111F6CF809191
:10C7C000C00085FFFCCF8AE08093C600CE010196B1
:10C7D0000E94E924AA960FB6F894DEBF0FBECDBF23
:10C7E000DF91CF911F910F91FF90EF90DF90CF904D
:10C7F000BF90AF909F908F907F906F905F900895C3
:10C80000CF93DF93EC018A818823C1F1EEEBF0E155
:10C8100007C09091C00095FFFCCF8093C600319671
:10C8200084918111F6CFFE01E053FF4F4081518189
:10C83000628173812AE030E089EA95E00E94012854
:10C84000E0EDF0E107C09091C00095FFFCCF809330
:10C85000C600319684918111F6CFC853DF4F4881CD
:10C8600059816A817B812AE030E089EA95E00E9463
:10C8700001288091C00085FFFCCF11C0E2EDF0E1FE
:10C8800007C09091C00095FFFCCF8093C600319601
:10C8900084918111F6CF8091C00085FFFCCF8AE0A2
:10C8A0008093C600DF91CF910895CF92DF92EF92EF
:10C8B000FF920F931F93CF93DF937C01EB01EC2F3B
:10C8C000FD2FDF010D900020E9F78D0101501109C6
:10C8D0000E1B1F0BF701E355FF4F10826EE470E053
:10C8E000CE010E9466706C01009729F4F80131971F
:10C8F000EC0FFD1F0DC060E270E00E946670EC015D
:10C9000021966AE270E0C6010E946670FC013197D0
:10C910008DE081838AE082831382BE01C701855541
:10C920009F4F0E94D631F701E355FF4F8081882346
:10C9300009F1E5EDFFE007C09091C00095FFFCCF45
:10C940008093C600319684918111F6CFE2EEF0E13A
:10C9500007C09091C00095FFFCCF8093C600319630
:10C9600084918111F6CF8091C00085FFFCCF8AE0D1
:10C970008093C600DF91CF911F910F91FF90EF90B0
:10C98000DF90CF9008953F924F925F926F927F9287
:10C990008F929F92AF92BF92CF92DF92EF92FF92CF
:10C9A0000F931F93CF93DF93CDB7DEB7CC55D1094B
:10C9B0000FB6F894DEBF0FBECDBF8C01662349F0E1
:10C9C000F801EC52FF4F1082F8018281811118C0EA
:10C9D00030C0FC01EC52FF4F8081882309F4AEC0C7
:10C9E000F801E453FF4FC080D180E280F3800E94C1
:10C9F0006225C616D706E806F90608F49FC0E0CF00
:10CA0000F80181898F9380898F938EEA92E09F93BA
:10CA10008F937E01FFE3EF0EF11CFF92EF920E94D5
:10CA2000AF700F900F900F900F900F900F906701C5
:10CA300010C0C8010E94FF5FF80182818111E0CF20
:10CA40007DC0F701808190E00E942570F7018193FD
:10CA50007F01F60101900020E9F73197EC19FD09FB
:10CA6000C7018C199D098E179F075CF33801F4E10B
:10CA70006F0E711C40E050E0BA01C3010E94362CD9
:10CA8000312CEE24E394F12CEC0EFD1E5E018FE3BD
:10CA9000A80EB11C77EB472E72E0572E4E01E1E253
:10CAA0008E0E911C37C0F601808190E00E942570A7
:10CAB000F60181936F01F70101900020E9F73197AA
:10CAC000EE19FF09C6018E199F098E179F075CF3A7
:10CAD0008A858E37F9F045E050E0B501C7010E9424
:10CAE00078700097B9F4BF92AF925F924F929F9285
:10CAF0008F920E94AF70C4010E94040A8EEB92E0F4
:10CB00000E94040A0F900F900F900F900F900F90BB
:10CB100033243394B701C3010E94C32B181614F4B5
:10CB20006701C9CF311004C08FEF9FEFF80104C037
:10CB3000F801808991890196918B808BC45ADF4FCF
:10CB40000FB6F894DEBF0FBECDBFDF91CF911F911E
:10CB50000F91FF90EF90DF90CF90BF90AF909F909C
:10CB60008F907F906F905F904F903F9008950F93BC
:10CB70001F93CF93DF938C01EC01C355DF4FCE01A0
:10CB80000E94D12CCE010E941D2DF8011082DF9150
:10CB9000CF911F910F910895CF93DF93EC010E94E5
:10CBA000A3520E941853198282EC92E00E94040A58
:10CBB00080910E0D8823A1F110920E0D6091D0028C
:10CBC000E62FF0E0EE0FFF1FE851F24F80819181D8
:10CBD0000E9428542091210130912201409123018B
:10CBE000509124010E947C6B1816D4F46091D002FD
:10CBF000C62FD0E080E090E00E945853FE01EE0F77
:10CC0000FF1FE851F24F91838083FE01EE0FFF1F5B
:10CC1000EE0FFF1FE252F24F108211821282138236
:10CC2000DF91CF910895EF92FF920F931F93CF93CF
:10CC3000DF937C01EB018A01060F171F09C0699180
:10CC4000D701ED91FC910190F081E02DC70109958C
:10CC5000C017D107A1F7DF91CF911F910F91FF90DE
:10CC6000EF9008958FEF8EBD0DB407FEFDCF8EB50A
:10CC700008958EBD0DB407FEFDCF089561E0FC015F
:10CC800080810C94A626FC014281242F30E035954A
:10CC9000279520652CBD40FD03C021E0463009F4F6
:10CCA00020E02DBD60E0FC0180810C94A626CF928F
:10CCB000DF92EF92FF920F931F93CF93DF93EC01DC
:10CCC0008B017A010E9462256B0109C00E946225D6
:10CCD0006C197D096D32714010F081E108C00E942D
:10CCE00032668B838F3F91F38E3F19F08FE08983FB
:10CCF00028C0E114F104E1F081E0E81AF1088FEFB7
:10CD00008EBDF8012FEF06C00DB407FEFDCF8EB526
:10CD100081932EBDCF01801B910B8E159F05A0F333
:10CD20000DB407FEFDCF8EB5F801EE0DFF1D80831B
:10CD30000E9432660E943266CE010E943E6681E009
:10CD400004C0CE010E943E6680E0DF91CF911F912A
:10CD50000F91FF90EF90DF90CF9008950F931F9366
:10CD6000CF93DF938B010E946225EB0107C00E94E5
:10CD700062256C1B7D0B6017710730F40E943266D0
:10CD80008F3FA9F781E001C080E0DF91CF911F9133
:10CD90000F910895CF92DF92FF920F931F93CF933D
:10CDA000DF9300D000D0CDB7DEB78C01F62E2983FB
:10CDB0003A834B835C830E9443666CE271E0C80156
:10CDC0000E94AE668F2D80640E94396668E1C62E8F
:10CDD000D12C5C814B813A812981DA01C9010C2C6B
:10CDE00004C0B695A795979587950A94D2F729839D
:10CDF0003A834B835C830E94396668E0C61AD10887
:10CE000029813A814B815C8188EFC8168FEFD80663
:10CE100021F7FF2029F098E0F91621F08FEF03C0E9
:10CE200085E901C087E80E943966ECE0FE1202C085
:10CE30000E943266F12C0E943266F801838387FFDC
:10CE400005C0FFEFFF1611F0F394F5CF0F900F9090
:10CE50000F900F90DF91CF911F910F91FF90DF9076
:10CE6000CF9008950F931F93CF93DF93EC01890127
:10CE70008C81833039F0B9E0440F551F661F771F4E
:10CE8000BA95D1F79A01AB0161E1CE010E94CA6661
:10CE900081110AC040E052E0B801CE01DF91CF918C
:10CEA0001F910F910C94576684E08983CE010E94F4
:10CEB0003E6680E0DF91CF911F910F910895BF9260
:10CEC000CF92DF92EF92FF920F931F93CF93DF9356
:10CED000EC01B62E1C82198248830E9462258B01C8
:10CEE00061E088810E948A26CE010E943E6660E051
:10CEF00086E00E948A2661E085E00E948A2661E041
:10CF000087E00E948A2661E084E00E948A2661E030
:10CF100084E00E94A62685E08A8382E58CBD1DBC44
:10CF20002AE0F22E8FEF0E943966FA94D9F709C0F1
:10CF30000E946225601B710B613D774010F081E01B
:10CF400058C020E030E0A90160E0CE010E94CA662E
:10CF5000F82E8B8381E0F812EBCF2AEA31E040E033
:10CF600050E068E0CE010E94CA6682FF02C0FC82E7
:10CF70000DC094E0F92E0E9432668B83FA94D9F7A3
:10CF80008A3A11F082E035C082E08C838C81823055
:10CF900031F4C12CD12CE12C80E4F82E0DC0C12C31
:10CFA000D12C760109C00E946225601B710B613D86
:10CFB000774010F08AE01DC020E030E0A90167E36F
:10CFC000CE010E94CA66A701960169E2CE010E94C5
:10CFD000CA668B838111E7CF8C818230C9F420E04F
:10CFE00030E0A9016AE3CE010E94CA66882319F0E5
:10CFF00088E0898319C00E943266807C803C11F4ED
:10D0000083E08C830E9432660E9432660E94326600
:10D01000CE010E943E6686E08B1518F488E1898374
:10D0200006C0BA8281E004C0CE010E943E6680E064
:10D03000DF91CF911F910F91FF90EF90DF90CF90F4
:10D04000BF900895CF93DF93EC016EBD20E030E0F8
:10D050000DB407FEFDCFFA01E20FF31F80818EBDF4
:10D060000DB407FEFDCF81818EBD2E5F3F4F211590
:10D0700082E0380769F70DB407FEFDCF8FEF0E94FD
:10D0800039668FEF0E9439660E9432668B838F71FA
:10D09000853039F083E18983CE010E943E6680E0CD
:10D0A00001C081E0DF91CF9108950F931F93CF933B
:10D0B000DF93EC0189018C81833039F0E9E0440F82
:10D0C000551F661F771FEA95D1F79A01AB0168E1FA
:10D0D000CE010E94CA66882311F086E029C0A8010B
:10D0E0006EEFCE010E9422688823B9F068E572E0F5
:10D0F000CE010E94AE66811102C087E119C020E016
:10D1000030E0A9016DE0CE010E94CA6681110FC016
:10D110000E94326681110BC005C0CE010E943E669E
:10D1200080E008C0CE010E943E6681E003C086E137
:10D130008983F3CFDF91CF911F910F9108955058BC
:10D14000BB27AA270ED076C23FD230F044D220F0BF
:10D1500031F49F3F11F41EF40FC20EF4E095E7FB8B
:10D16000DCC1E92F89D280F3BA17620773078407FD
:10D17000950718F071F49EF5B8C20EF4E0950B2EE9
:10D18000BA2FA02D0B01B90190010C01CA01A00119
:10D190001124FF27591B99F0593F50F4503E68F174
:10D1A0001A16F040A22F232F342F4427585FF3CFB5
:10D1B000469537952795A795F0405395C9F77EF486
:10D1C0001F16BA0B620B730B840BBAF09150A1F0CF
:10D1D000FF0FBB1F661F771F881FC2F70EC0BA0F55
:10D1E000621F731F841F48F4879577956795B795DD
:10D1F000F7959E3F08F0B3CF9395880F08F09927D5
:10D20000EE0F979587950895DFD158F080E891E06B
:10D2100009F49EEFE0D128F040E851E059F45EEFC8
:10D2200009C0AAC162C2E92FE07826D268F3092EAC
:10D23000052AC1F3261737074807590738F00E2E7D
:10D2400007F8E02569F0E025E0640AC0EF6307F81D
:10D25000009407FADB01B9019D01DC01CA01AD01AF
:10D26000EF935DD0E7D10AD05F91552331F02BEDDC
:10D270003FE049E450FD49EC63CF0895DF93DD279B
:10D28000B92FBF7740E85FE31616170648075B071C
:10D2900010F4D92F96D29F938F937F936F93A9D336
:10D2A000ECE7F0E06CD1C6D12F913F914F915F91A7
:10D2B00001D3DD2349F09058A2EA2AED3FE049EC82
:10D2C0005FE3D0785D274DDFDF91B4C1F7D180F007
:10D2D0009F3740F491110EF409C260E070E080E8DD
:10D2E0009FE3089526F01B16611D711D811D1BC152
:10D2F00035C1EFD008F481E0089575D1E395ABC155
:10D300000CD098C168D140F05FD130F021F45F3F7C
:10D3100019F003C15111EAC12FC1AED198F399237D
:10D32000C9F35523B1F3951B550BBB27AA276217E9
:10D330007307840738F09F5F5F4F220F331F441F2E
:10D34000AA1FA9F333D00E2E3AF0E0E830D0915066
:10D350005040E695001CCAF729D0FE2F27D0660F53
:10D36000771F881FBB1F261737074807AB07B0E892
:10D3700009F0BB0B802DBF01FF2793585F4F2AF0A8
:10D380009E3F510568F0C9C0B1C15F3FECF3983EC4
:10D39000DCF3869577956795B795F7959F5FC9F705
:10D3A000880F911D9695879597F90895E1E0660F8E
:10D3B000771F881FBB1F621773078407BA0720F007
:10D3C000621B730B840BBA0BEE1F88F7E095089570
:10D3D00004D06894B1118AC1089556D188F09F573E
:10D3E00090F0B92F9927B751A0F0D1F0660F771FB1
:10D3F000881F991F1AF0BA95C9F712C0B13081F091
:10D4000074D1B1E0089571C1672F782F8827B85F74
:10D4100039F0B93FCCF3869577956795B395D9F7F1
:10D420003EF490958095709561957F4F8F4F9F4FFB
:10D430000895E89409C097FB3EF490958095709507
:10D4400061957F4F8F4F9F4F9923A9F0F92F96E950
:10D45000BB279395F695879577956795B795F111C5
:10D46000F8CFFAF4BB0F11F460FF1BC06F5F7F4F62
:10D470008F4F9F4F16C0882311F096E911C0772374
:10D4800021F09EE8872F762F05C0662371F096E87D
:10D49000862F70E060E02AF09A95660F771F881F4C
:10D4A000DAF7880F9695879597F9089507D180F058
:10D4B0009F3740F491110EF019C160E070E080E8F0
:10D4C0009FEB089526F41B16611D711D811D2BC055
:10D4D00045C0990F0008550FAA0BE0E8FEEF16169D
:10D4E0001706E807F907C0F012161306E407F50758
:10D4F00098F0621B730B840B950B39F40A2661F0CC
:10D50000232B242B252B21F408950A2609F4A1406E
:10D51000A6958FEF811D811D089597F99F6780E87B
:10D5200070E060E00895882371F4772321F098502B
:10D53000872B762F07C0662311F499270DC09051D1
:10D54000862B70E060E02AF09A95660F771F881F9F
:10D55000DAF7880F9695879597F908959F3F31F0F0
:10D56000915020F4879577956795B795880F911D11
:10D570009695879597F908959FEF80EC0895DF932E
:10D58000CF931F930F93FF92EF92DF927B018C0159
:10D59000689405C0DA2EEF018DD1FE01E894A591C3
:10D5A0002591359145915591AEF3EF01DADDFE01FC
:10D5B0009701A801DA9479F7DF90EF90FF900F912F
:10D5C0001F91CF91DF91089500240A941616170633
:10D5D00018060906089500240A9412161306140664
:10D5E00005060895C9CF50D0E8F3E894E0E0BB27E2
:10D5F0009F57F0F02AED3FE049EC06C0EE0FBB0F5D
:10D60000661F771F881F28F0B23A620773078407E6
:10D6100028F0B25A620B730B840BE3959A9572F75C
:10D62000803830F49A95BB0F661F771F881FD2F79A
:10D63000904896CF092E0394000C11F4882352F0E1
:10D64000BB0F40F4BF2B11F460FF04C06F5F7F4F2E
:10D650008F4F9F4F0895EF93E0FF06C0A2EA2AED97
:10D660003FE049EC5FEB7DDDE5DF0F90039401FCCB
:10D670009058E9EAF0E0C7C157FD9058440F551F94
:10D6800059F05F3F71F04795880F97FB991F61F044
:10D690009F3F79F087950895121613061406551FBB
:10D6A000F2CF4695F1DF08C0161617061806991F27
:10D6B000F1CF86957105610508940895E5DFA0F026
:10D6C000BEE7B91788F4BB279F3860F41616B11D62
:10D6D000672F782F8827985FF7CF8695779567957E
:10D6E000B11D93959639C8F30895E894BB27662732
:10D6F0007727CB0197F90895ECDE08F48FEF0895B2
:10D7000063DF19F068DF09F037CF07CFB901CA012D
:10D7100025CF9F775F77B0DF98F39923B9F355232F
:10D72000B9F3FF27951758F4E52FE91BED3070F793
:10D730005E3B10F0F1E41CC09034E0F40AC0E92F25
:10D74000E51BED3028F79E3B10F0F1E411C050349A
:10D7500088F4F9EA88232AF09A95660F771F881FC4
:10D76000DAF744232AF05A95220F331F441FDAF7C1
:10D770009F1B5F1BFF931F930F93FF92EF92790103
:10D780008A01BB27AB2F9B01AC0196D09701A80162
:10D79000BF937B018C01AA27BA2FB901CA018CD093
:10D7A000AF919701A801EF90FF900F911F91D9DCE5
:10D7B00041DFE1D04F9140FF0895552747FD509537
:10D7C00009C09B01AC0160E070E080E89FE398CD68
:10D7D000A4CEC4CE59DFE8F39923D9F3940F511D99
:10D7E000BBF39150504094F059F0882332F0660F0B
:10D7F000771F881F91505040C1F79E3F510544F755
:10D80000880F911D9695879597F908955F3FACF025
:10D81000983E9CF0BB27869577956795B79508F459
:10D82000B1609395C1F7BB0F58F711F460FFE8CFD3
:10D830006F5F7F4F8F4F9F4FE3CF58CF25DF58F15A
:10D840009E5758F19851A0F0E9F0983020F5092E34
:10D850009927660F771F881F991F0A94D1F712C066
:10D86000062E672F782F8827985F11F4000C07C0C9
:10D87000993FB4F38695779567959395D9F7611D90
:10D88000711D811D3EF490958095709561957F4F37
:10D890008F4F9F4F0895689429CF27CF0BD0CACEC2
:10D8A00093DE28F098DE18F0952309F036CE64CE8A
:10D8B00011241CCFE1DEA0F3959FD1F3950F50E02A
:10D8C000551F629FF001729FBB27F00DB11D639F32
:10D8D000AA27F00DB11DAA1F649F6627B00DA11DD8
:10D8E000661F829F2227B00DA11D621F739FB00D7E
:10D8F000A11D621F839FA00D611D221F749F3327EE
:10D90000A00D611D231F849F600D211D822F762F86
:10D910006A2F11249F5750408AF0E1F088234AF083
:10D92000EE0FFF1FBB1F661F771F881F91505040CF
:10D93000A9F79E3F510570F0F0CDD8CE5F3FECF3D4
:10D94000983EDCF3869577956795B795F795E795BB
:10D950009F5FC1F7FE2B880F911D9695879597F9CC
:10D9600008959F9340DE0F9007FCEE5F74CE11F494
:10D970000EF402CEF3CD88DED0F39923D9F3CEF3A3
:10D980009F57550B87FF38D00024A0E640EA90014E
:10D9900080585695979528F4805C660F771F881FEE
:10D9A00020F026173707480730F4621B730B840BEF
:10D9B000202931294A2BA695179407942025312533
:10D9C0004A2758F7660F771F881F20F0261737075A
:10D9D000480730F4620B730B840B200D311D411D81
:10D9E000A09581F7B901842F9158880F9695879556
:10D9F00008959B01AC0152CF91505040660F771FA4
:10DA0000881FD2F708959F938F937F936F93FF930F
:10DA1000EF939B01AC0142DFEF91FF91B0DD2F91BD
:10DA20003F914F915F913ACF0E94896DA59F900DD4
:10DA3000B49F900DA49F800D911D11240895B7FFF0
:10DA40000C94146D0E94146D821B930B0895DB01DE
:10DA50008F939F930E94146DBF91AF91A29F800DF1
:10DA6000911DA39F900DB29F900D1124089597FBD7
:10DA7000072E16F4009407D077FD09D00E94956D0B
:10DA800007FC05D03EF4909581959F4F08957095C1
:10DA900061957F4F0895A1E21A2EAA1BBB1BFD01C1
:10DAA0000DC0AA1FBB1FEE1FFF1FA217B307E4077D
:10DAB000F50720F0A21BB30BE40BF50B661F771FD5
:10DAC000881F991F1A9469F76095709580959095B5
:10DAD0009B01AC01BD01CF010895052E97FB16F403
:10DAE000009407D057FD0DD00E944B6D07FC09D064
:10DAF0007EF490958095709561957F4F8F4F9F4FE5
:10DB0000089550954095309521953F4F4F4F5F4F69
:10DB10000895A29FB001B39FC001A39F01D0B29FFF
:10DB2000700D811D1124911D0895AA1BBB1B51E18D
:10DB300007C0AA1FBB1FA617B70710F0A61BB70B7D
:10DB4000881F991F5A95A9F780959095BC01CD0122
:10DB50000895EE0FFF1F0590F491E02D0994A0E0C9
:10DB6000B0E0E5EBFDE60C9459738B01611571058E
:10DB700019F0FB01808391837C01F701C1907F0143
:10DB8000EF018C2D90E00E941D70892BB1F7FDE212
:10DB9000CF1204C0C990DD24D39405C02BE2C21279
:10DBA00001C0C990D12C7E0141E0E41AF10843E0A4
:10DBB00050E062E671E1C7010E942D70892BE9F403
:10DBC0007E0182E0E80EF11C45E050E065E671E17F
:10DBD000C7010E942D70892B21F47E01E7E0EE0E33
:10DBE000F11C0115110519F0F801F182E08210E035
:10DBF000D0E0C0E8D110FBC0FFC043E050E06AE6CF
:10DC000071E1C7010E942D70892B49F4011511059E
:10DC100009F4EFC02296F801D183C083EAC060E026
:10DC200070E0CB01E12CF12CEC2DE053EA3048F50B
:10DC3000FD2DF2602D2D2870D2FE06C0211127C0C7
:10DC40002FEFE21AF20A23C0222319F041E0E41A6E
:10DC5000F108A5E0B0E09B01AC010E94146D660FD5
:10DC6000771F881F991F6E0F711D811D911D6839C7
:10DC7000E9E97E078E07E9E19E0748F0FD2DF66091
:10DC800006C0EE3F39F4D3FC3DC0FD2DF860C990CD
:10DC9000DF2ECACFE53311F0E531A1F5A881AD3211
:10DCA00019F4F0E1DF2A06C0AB3221F0219621E021
:10DCB00030E004C0A981229622E030E0A053AA30CF
:10DCC00018F0C21BD30B1EC0FE0120E030E020384C
:10DCD0004CE034075CF4A901440F551F440F551F55
:10DCE000240F351F220F331F2A0F311DA191A0537E
:10DCF000EF01AA3060F3D4FE03C0319521953109BC
:10DD0000E20EF31ED1FE07C00115110521F0219787
:10DD1000F801D183C0830E94196A2D2D237023300E
:10DD200029F0162FD72FC82F092F07C0DC01CB01F0
:10DD3000B058182FD92FCA2F0B2F20E030E0A9019F
:10DD4000612F7D2F8C2F902F0E947969882309F4F1
:10DD500054C0F7FE08C0F194E194F10839E9C32EEC
:10DD600031E1D32E04C021E8C22E21E1D22E46019A
:10DD7000F8E18F1A910890E2A92EB12C15C0F60196
:10DD80004591559165917491242F352F462F572F2A
:10DD9000612F7D2F8C2F902F0E944E6C162FD72F26
:10DDA000C82F092FEA18FB08EA14FB0444F724E003
:10DDB000C21AD108B594A794C814D904A9F7612F41
:10DDC0007D2F8C2F902F282F220F292F221F2F3F9E
:10DDD00039F020E030E0A9010E94796981110DC07D
:10DDE00082E290E090932C0E80932B0E06C00FEFF2
:10DDF00004C010E0D0E0C0EC0FE7612F7D2F8C2F26
:10DE0000902FCDB7DEB7ECE00C947573A0E0B0E0D6
:10DE1000ECE0FFE60C9455732B018A016115710546
:10DE200019F0FB01808391830115110539F09801E8
:10DE3000225031092332310508F0E6C07C01F70198
:10DE4000C1917F013F018C2F90E00E941D70892BB2
:10DE5000B1F7CD3229F4F701C1913F01D1E006C0FD
:10DE6000CB3219F4F701C1913F01D0E00115110542
:10DE700009F4D8C00031110581F4D0C0F3018081CC
:10DE8000883719F0883509F0C3C0F301C181F2E089
:10DE90006F0E711CD26000E110E008301105D9F05E
:10DEA00024F402301105F9F407C00A30110551F0CD
:10DEB00000311105C1F425C0C12CD12CE12C30E476
:10DEC000F32E24C00AE010E02CECC22EDC2CEC2C4B
:10DED0002CE0F22E1BC008E010E0C12CD12CE12C6C
:10DEE00090E1F92E13C09801442737FD4095542F37
:10DEF00060E070E080E090E80E944B6D69017A017B
:10DF000005C0C12CD12CE12C88E0F82E40E060E067
:10DF100070E0CB014801AA2497FCA094BA2CEC2F06
:10DF2000E053EA3060F02C2F21542A3110F4E750EE
:10DF300006C02C2F21562A3128F5EC2FE7552E2F1D
:10DF400030E020173107F4F447FD18C0C616D70695
:10DF5000E806F90680F09B01AC01C501B4010E94FE
:10DF6000276D6E0F711D811D911D61307105810539
:10DF700020E8920710F04FEF01C041E0F301C1919A
:10DF80003F01CDCF4114510491F0442339F0F1E029
:10DF90006F1A7108F2017182608209C0D1FF1BC043
:10DFA000F2E06F1A7108F2017182608214C047FFBB
:10DFB00012C0D0FF05C060E070E080E090E804C0CF
:10DFC0006FEF7FEF8FEF9FE722E230E030932C0E70
:10DFD00020932B0E16C0D0FF08C0909580957095A9
:10DFE00061957F4F8F4F9F4F0CC097FF0AC082E211
:10DFF00090E090932C0E80932B0E6FEF7FEF8FEFBE
:10E000009FE76B017C0112C0C12CD12C76010EC0A0
:10E01000C0E30115110509F45ECF3FCFC03309F00D
:10E020003CCF2CCFC03309F04DCF28CFB601C7016C
:10E03000CDB7DEB7E0E10C947173911191C28032DB
:10E0400019F089508550D0F70895911108958154A1
:10E050008A5108F4805E855A0895FB01DC01415025
:10E06000504088F08D9181341CF08B350CF4805E2B
:10E07000659161341CF06B350CF4605E861B611198
:10E0800071F3990B0895881BFCCFFB01DC0104C0E0
:10E090008D910190801921F441505040C8F7881BA0
:10E0A000990B0895FB01DC0102C001900D924150D3
:10E0B0005040D8F70895FB01DC010D900020E9F7EE
:10E0C000119701900D920020E1F70895FC018191D4
:10E0D000861721F08823D9F7992708953197CF0122
:10E0E0000895FB01DC0101900D920020E1F70895F5
:10E0F000FB01DC014150504030F08D9101908019BE
:10E1000019F40020B9F7881B990B0895FB01DC0175
:10E110004150504048F001900D920020C9F701C0D5
:10E120001D9241505040E0F70895FB015191552355
:10E13000A9F0BF01DC014D9145174111E1F759F4F8
:10E14000CD010190002049F04D9140154111C9F3D6
:10E15000FB014111EFCF81E090E001970895A0E12C
:10E16000B0E0E5EBF0E70C9461730F89188D86E061
:10E170008C831A8309838FEF9FE79E838D83AE0183
:10E18000455E5F4F588B4F87698D7A8DCE01019622
:10E190000E94D370EF81F885E00FF11F1082609626
:10E1A000E4E00C947D73ACE0B0E0E9EDF0E70C94B2
:10E1B00053737C016B018A01FC01178216828381F3
:10E1C00081FFC7C188248394912C8C0E9D1EF7017A
:10E1D0009381F60193FD859193FF81916F018823CF
:10E1E00009F4B3C1853239F493FD859193FF819190
:10E1F0006F01853229F4B70190E00E94C972E7CF20
:10E20000712C312C20E02032A8F48B3261F028F4FC
:10E21000803251F0833271F40BC08D3239F080338B
:10E2200049F4216028C02260246025C0286023C0F2
:10E23000206121C027FD27C0382F30533A3078F4B1
:10E2400026FF06C0FAE07F9E300D1124732E13C006
:10E250008AE0389E300D1124332E20620CC08E329D
:10E2600021F426FD72C1206406C08C3611F42068AA
:10E2700002C0883641F4F60193FD859193FF8191A8
:10E280006F018111C0CF982F9554933018F09052A0
:10E29000933028F40C5F1F4FFFE3F9830DC08336E2
:10E2A00031F0833771F0833509F05EC023C0F80187
:10E2B000808189830E5F1F4F66246394712C540103
:10E2C00015C02801F2E04F0E511CF801A080B1806A
:10E2D00026FF03C0672D70E002C06FEF7FEFC5011E
:10E2E0002C870E94BE723C0182012C856FE7262E8E
:10E2F000222218C02801F2E04F0E511CF801A08024
:10E30000B18026FF03C0672D70E002C06FEF7FEF82
:10E31000C5012C870E94B3723C012C8550E8252E44
:10E32000222A820123FC1CC006C0B70180E290E0D3
:10E330000E94C9723A94832D90E068167906A8F37A
:10E340000FC0F50127FC859127FE81915F01B70180
:10E3500090E00E94C97231103A94F1E06F1A71088E
:10E360006114710471F7EEC0843611F0893641F5FD
:10E37000F80127FF07C060817181828193810C5F62
:10E380001F4F08C060817181882777FD8095982F85
:10E390000E5F1F4F4FE6642E622297FF09C09095D3
:10E3A0008095709561957F4F8F4F9F4FF0E86F2A52
:10E3B0002AE030E0A4010E94F572A82EA81844C0FB
:10E3C000853731F43FEEB32EB2222AE030E024C08C
:10E3D00099EFB92EB2228F36B9F020F4883509F0C2
:10E3E000B4C00DC0803721F0883709F0AEC002C03C
:10E3F00020E1B22AB4FE0BC084E0B82A08C024FF92
:10E4000009C0E6E0BE2A06C028E030E005C020E1F1
:10E4100030E002C020E132E0F801B7FE07C06081C1
:10E420007181828193810C5F1F4F06C06081718171
:10E4300080E090E00E5F1F4FA4010E94F572A82EAD
:10E44000A8188FE7682E6B2066FE0BC0362D3E7F26
:10E45000A71450F464FE0AC062FC08C0362D3E7E4C
:10E4600005C0BA2C362D03C0BA2C01C0B72C34FF1E
:10E470000DC0FE01EA0DF11D8081803311F4397E5B
:10E4800009C032FF06C0B394B39404C0832F8678CA
:10E4900009F0B39433FD14C030FF0FC07A2CB314CD
:10E4A00060F4730C7B18B32C08C0B70180E290E0D5
:10E4B0003C870E94C972B3943C85B314B0F304C086
:10E4C000B31410F43B1801C0312C34FF12C0B70153
:10E4D00080E390E03C870E94C9723C8532FF1EC0F9
:10E4E00031FF03C088E590E002C088E790E0B70103
:10E4F0000CC0832F867891F031FD02C080E201C00C
:10E500008BE237FD8DE2B70190E00E94C97206C030
:10E51000B70180E390E00E94C9727A94A714C0F317
:10E52000AA94F401EA0DF11DB701808190E00E94E8
:10E53000C972A110F5CF06C0B70180E290E00E9439
:10E54000C9723A943110F8CF42CEF7012681378153
:10E5500002C02FEF3FEFC9012C96E2E10C946F73DC
:10E56000992788270895FC0105906150704001109B
:10E57000D8F7809590958E0F9F1F0895FC016150EC
:10E58000704001900110D8F7809590958E0F9F1FD5
:10E5900008950F931F93CF93DF938C01EB018B8131
:10E5A00081FD03C00FEF1FEF1AC082FF0DC02E8147
:10E5B0003F818C819D812817390764F4E881F981B6
:10E5C0000193F983E88306C0E885F985802F0995D2
:10E5D000892B41F78E819F8101969F838E83C8018D
:10E5E000DF91CF911F910F910895FA01AA2728304A
:10E5F00051F1203181F1E8946F936E7F6E5F7F4F10
:10E600008F4F9F4FAF4FB1E03ED0B4E03CD0670F8B
:10E61000781F891F9A1FA11D680F791F8A1F911DDE
:10E62000A11D6A0F711D811D911DA11D20D009F42E
:10E6300068943F912AE0269F11243019305D319370
:10E64000DEF6CF010895462F4770405D4193B3E059
:10E650000FD0C9F7F6CF462F4F70405D4A3318F000
:10E66000495D31FD4052419302D0A9F7EACFB4E0B1
:10E67000A6959795879577956795BA95C9F7009769
:10E680006105710508959B01AC010A2E069457950A
:10E69000479537952795BA95C9F7620F731F841F61
:10E6A000951FA01D08952F923F924F925F926F92F7
:10E6B0007F928F929F92AF92BF92CF92DF92EF9212
:10E6C000FF920F931F93CF93DF93CDB7DEB7CA1B93
:10E6D000DB0B0FB6F894DEBF0FBECDBF09942A88BE
:10E6E000398848885F846E847D848C849B84AA8466
:10E6F000B984C884DF80EE80FD800C811B81AA81F3
:10E70000B981CE0FD11D0FB6F894DEBF0FBECDBFBD
:10E71000ED01089511E1C0EAD1E104C0FE010E94BB
:0EE72000AB6D2296C23AD107C9F7F894FFCF2D
:10E72E006400640000803B4500803B450000704360
:10E73E00000000000080BB440160EA0000CDCCCC9C
:10E74E003D0000524300007A430101010101000027
:10E75E00803FE7849145AECF1A3D00004041FF3F18
:10E76E00FF3F0171DBB64271DBB64200007A450015
:10E77E00C05A440000FA430000FA430000A04000D3
:10E78E00003442E8030000E803000032000000FA03
:10E79E000000005573696E672044656661756C7480
:10E7AE002073657474696E67733A004D31313000B1
:10E7BE002569206D696E2C202569207365630048DC
:10E7CE0020004C20004D31303420496E76616C694A
:10E7DE006420657874727564657220004D31303531
:10E7EE0020496E76616C6964206578747275646513
:10E7FE007220004D31303920496E76616C6964208B
:10E80E00657874727564657220003F006F6B00202E
:10E81E00703A0020693A0020643A0020633A0054AE
:10E82E0000496E76616C69642065787472756465F2
:10E83E0072004163746976652045787472756465FB
:10E84E00723A20004D32390058595A4500000100E5
:10E85E000F0015000E001200FFFF160017000E002D
:10E86E001300FFFF030002001A001400FFFFFFFF5A
:10E87E00FFFF0A00FFFF010000000E000D00070061
:10E88E00FFFFFFFF06002E0000000000E231D63130
:10E89E001366537465707261746520746F206869B5
:10E8AE006768203A2000504944204175746F747592
:10E8BE006E65207374617274002F0043616E6E6F0B
:10E8CE0074206F70656E2073756264697200617575
:10E8DE00746F25692E67004D3233202573004D323B
:0EE8EE0034004D383420582059205A2045005F
:00000001FF
